:1000000000800020BD01000015D10000CDD000000F
:10001000CDD00000CDD00000CDD00000CDD000006C
:10002000CDD00000CDD00000CDD0000015D1000013
:1000300015D10000CDD0000095C7000099C8000080
:1000400015D1000015D1000015D1000015D1000018
:1000500015D1000015D1000015D1000015D1000008
:1000600015D1000015D1000015D1000015D10000F8
:1000700015D1000015D1000015D1000015D10000E8
:1000800015D1000015D1000015D1000015D10000D8
:1000900015D1000015D1000015D1000015D10000C8
:1000A000D1AC0000DDAC000015D1000015D100007E
:1000B00015D1000015D1000015D1000015D10000A8
:1000C00015D1000015D1000015D1000015D1000098
:1000D00015D1000015D1000015D1000015D1000088
:1000E00015D1000015D1000015D1000015D1000078
:1000F00015D1000081F1000015D10000ADF2000023
:1001000015D10000EDDA000015D1000015D1000076
:1001100015D1000015D1000015D1000015D1000047
:1001200015D1000015D1000015D1000015D1000037
:1001300015D1000015D1000015D1000015D1000027
:1001400015D1000015D1000015D1000015D1000017
:1001500085C9000099C90000ADC90000C1C90000EF
:1001600015D1000009DE000015D1000015D10000F6
:1001700015D1000015D1000015D1000015D10000E7
:1001800015D1000015D1000015D1000015D10000D7
:1001900015D1000015D1000015D1000015D10000C7
:1001A00015D1000015D1000015D1000015D10000B7
:1001B00015D1000015D1000015D10000564B4CF2AE
:1001C000205210B51A804DF628121A8000BF00BFC9
:1001D0000CF0A4FF514B4FF010621A60504A9A6025
:1001E000504ADA60504A136813F4807304D14F49BF
:1001F0000B604FF4A85313604D4B1A78110703D5C9
:100200001A7842F008021A704A4B4B492A221A7097
:100210004A4A4B4B8B4204D252F8040F43F8040B6A
:10022000F8E7484B484900228B4202D243F8042B9E
:10023000FAE74649464A002352F8230041F82300D2
:1002400001336F2BF8D1434B434A802103F8011B44
:100250009342FBD1414B3D4A1A60414B8A221A70AE
:10026000A3F5805324225A70A0221A709A7992071B
:10027000FCD59A79D406FCD43A4A937903F00C035E
:10028000082B384BF9D103221A7140225A719A79FE
:100290009006FCD5334A9179324B4906FBD5324A58
:1002A000324911600221516020221A709A7902F0BD
:1002B0000C020C2AFAD12E4B2E4A1A602E4B2F4AD2
:1002C0001A6000225A60072243F8042C2C4AC3F813
:1002D0000C2D62B60DF0D2FA144B1B68DA0705D567
:1002E00028480DF09FF8284B284A1A60284B1B78A5
:1002F0005B0609D5244C254B22689A4204D121483B
:100300000DF090F80023236010F08AFA0CF00CFF37
:100310000CF03AFEFEE700BF0E200540308004409E
:10032000823F04000100002B10D0034014D0034092
:1003300002D0074000E00740EC9BFF1F9440010003
:100340004088FF1FEC9BFF1F04A4FF1F0082FF1FBC
:100350000000000000E400E05FE400E008ED00E0E1
:100360000050064000400640448004400000030165
:1003700004800440C010050014E000E0FF76010096
:10038000000020205EE63C5F1CE00340A5C3945AB9
:1003900000F00740FFFFFFFFFFFFFFFFFFFFFFFF32
:1003A000FFFFFFFFFFFFFFFFFFFFFFFFFFFFFFFF5D
:1003B000FFFFFFFFFFFFFFFFFFFFFFFFFFFFFFFF4D
:1003C000FFFFFFFFFFFFFFFFFFFFFFFFFFFFFFFF3D
:1003D000FFFFFFFFFFFFFFFFFFFFFFFFFFFFFFFF2D
:1003E000FFFFFFFFFFFFFFFFFFFFFFFFFFFFFFFF1D
:1003F000FFFFFFFFFFFFFFFFFFFFFFFFFFFFFFFF0D
:10040000FFFFFFFFFFFFFFFFFFFFFFFFDEF9FFFF23
:1004100010B5054C237833B9044B13B10448AFF33E
:1004200000800123237010BDEC9BFF1F0000000023
:1004300098400100084B10B51BB108490848AFF3BC
:1004400000800848036803B910BD074B002BFBD0A0
:10045000BDE81040184700BF00000000F09BFF1FE0
:1004600098400100EC9BFF1F0000000038B50446D7
:10047000104621700A491D460FF0B4FF01464FF0A7
:100480007E5010F063F807490FF0ACFFE560606044
:10049000256165610DF082F9E061204638BD00BF3D
:1004A000DB0FC9400024744938B50446104621705A
:1004B00009491D460FF096FF01464FF07E5010F09F
:1004C00045F806490FF08EFFE560606025616561C3
:1004D0000DF064F9E06138BDDB0FC94000247449B8
:1004E00038B503780446032B20D8DFE803F01A1848
:1004F0001002C16840690FF06BFE0D490546606847
:1005000010F024F80146284610F020F838BD0849BC
:10051000406810F01BF8E1680FF064FF38BDC06858
:1005200038BDC16840690FF053FE38BD002038BDAA
:100530000024744970B504460E460DF02FF90546A7
:10054000E069281A0FF0FAFEE3682361E56166614D
:10055000A061014660680FF0F9FF0146A0601048F5
:100560000FF0F4FF0FF0CAFA0EF06AFF0FF0DCFD97
:10057000054601464FF07E500FF02AFE61690FF0EC
:1005800031FF2169064628460FF02CFF0146304610
:100590000FF020FEE0602046BDE87040FFF7A0BFEE
:1005A000000080BF38B50E201C4C0CF0C7FB218822
:1005B0001B4B884205461A881DDA0023511AB1F5F3
:1005C000805FAABF1B03C3EB03330131142093FBED
:1005D000F1F10CF039FF134B1988F1B923889D42D2
:1005E00010DAC3F57F630F33282091FBF3F1BDE8E8
:1005F00038400CF029BF9042D4BFC1EB0003C1EBDF
:100600000203DBE740F6FF718D42D4BFC3EB050167
:10061000C3EB0101C1EB0131E3E738BDD89CFF1FFB
:100620009A9EFF1F489EFF1F10B504460CF088F9E4
:10063000204610BD70B44C88A04220D9012301335C
:10064000DBB21CB2660031F8144084421D46F6D37A
:10065000A04211D005F10045013D965B31F815101F
:1006600032F81530401AF21A00FB02F0641A90FBBF
:10067000F4F4E01870BC7047905B70BC70470226C1
:100680000125E5E700280CDA064A434282FB0320F5
:10069000DA17C2EB600000EB4000A3EB8000C0F172
:1006A0000C007047ABAAAA2AF0B40E8886420DD27D
:1006B00003F10043013B31F81350854202D9F0BCED
:1006C000FFF7B8BF32F81300F0BC70471088F0BCD9
:1006D000704700BF094B1B880C2B09D8084A80B211
:1006E00052F8232028B143F6FE73984203D9108CA8
:1006F0007047108870470349FFF79CBF3E9CFF1F5F
:10070000201B0100BC1C0100374A38491088384AB8
:10071000F8B5384B12881B68834248DB9342A8BF68
:10072000134698420B60C8BF002342DD101AB0F593
:10073000804FAABF9B03C3EB8333013093FBF0F0E0
:10074000FFF7C8FF2C4B2D4F1C883B68C0F3C61524
:1007500005FB04F47F2CA8BF7F249D42064608D0E9
:10076000274B1B88002B38D1264B1B88002B30D100
:100770003D60254D2B689E4205D0214B1B885A1F9A
:10078000032A1DD92E60214D2B689C420ED0204B90
:10079000188848B11A4B1F4A1B88D35C834203D088
:1007A000C0B2E1B208F000FC2C60F8BDF8BD034611
:1007B00008609A42D4BFC0EB0203C0EB0303B5E765
:1007C000144AD05C2030C0B206F07F0108F0ECFB88
:1007D000D8E7284608F05CFCCAE70E4A2946D05CF8
:1007E00008F0E2FBC0E700BFD89CFF1F109CFF1F72
:1007F0009A9EFF1F449EFF1F249CFF1F809CFF1F8B
:100800002C9EFF1FCA9CFF1F389CFF1FCC9CFF1F04
:100810003A9EFF1F048AFF1F2DE9F04F012089B087
:100820000DF0D0F9AF4B186000200DF0CBF9AE4BB6
:10083000AE4A1B8810600C2B00F03B81AC4BAD4ADC
:1008400019880093AC4B52F8214000221A70AB4B30
:10085000AB4D1B88AB4A2E88013B32F91370002E3A
:100860005CD0A94BA94A1B88A9491278013B31F9F0
:100870001380002A40F0DF8011200DF0A3F9A54B72
:100880000193D3F800A00646B24540F3DF80A24BA7
:10089000DFF8A4921B88A14A012BD9F80030B2F8E6
:1008A00000B09F4A02922046C8EB030800F09A82EB
:1008B0000FF044FD029A52F82B100FF093FD014601
:1008C00000200FF085FC0FF053FFCAEB0802B04583
:1008D000B8BFB0469042CAEB080880F2968200FB8F
:1008E0000888013298FBF2F08E4BDFF850820293B9
:1008F000D8F80030034403EBD3735B10C8F8003022
:100900002B88012B12D1884BDFF834B20393874B2D
:10091000DBF8005004934FF0000A47E07D4B019351
:10092000DFF814927F4BDFF8148202937E4B03931F
:100930001D460F200DF046F92B689842824641DA99
:10094000754A1288012A00F01D82744A05931288A4
:10095000734D049220460FF0F1FC049ADFF8E0B1E9
:1009600055F82210DBF800500FF03CFD0146002046
:100970000FF02EFC0FF0FCFEEF1B059B5745A7EB7D
:100980000302B8BF5746FF1A9042BABF013200FBBC
:100990000777474397FBF2F7D8F80020634B04939F
:1009A000BB1803EBD3735B10C8F80030604B1B8897
:1009B000013B032B00F2B082DFE813F06301A901D1
:1009C000C4008601594B04931B68984240F3C281CE
:1009D000514A1288012A00F0A682504A07931188D2
:1009E0004F4A0691204605920FF0A8FC059A0699F9
:1009F000DFF84CB152F82110DBF800500FF0F2FC98
:100A00000FF0B6FE079B2F445745A7EB0302A8BF84
:100A10005746FF1AD8F800309042BABF00FB07775C
:100A20000132474397FBF2F73B4403EBD3735B1070
:100A3000C8F80030BAE715200CF080F9354B019367
:100A4000D3F800A00646B2453FF721AF354B0293DD
:100A5000D3F800A0B24580F289812F4BDFF8D890FF
:100A60001B882E4A012BD9F80030B2F800B02C4A6E
:100A700003922046984400F070820FF05FFC039AC6
:100A800052F82B100FF0AEFC0FF072FEB045CAEB1F
:100A90000802A8BFB046CAEB08089042B6BF00FBE8
:100AA000088800FB08F8013298FBF2F0DFF88C8030
:100AB0001EE7204B1B78002B3FF4C0AE0C4B0D4AB9
:100AC000198800930C4B52F8210001221A700FF084
:100AD00035FC4FF07C510FF085FC0FF049FE0446C9
:100AE000B5E600BF709CFF1F729EFF1FBC9EFF1FDC
:100AF000769CFF1F8489FF1F1A9CFF1F108AFF1F0F
:100B0000E49DFF1F04200100608AFF1FF89DFF1F66
:100B1000741C0100689CFF1FB69CFF1F5C9CFF1F9C
:100B20001C200100A49CFF1F649EFF1FD89DFF1F77
:100B30005A89FF1F2E9CFF1F089CFF1F7C9EFF1FD2
:100B4000609EFF1F28460FF0F9FBB2490FF04AFCE8
:100B5000054650460FF0F2FBAF490FF043FC01464B
:100B600028460FF037FB0FF003FE0546CBF8005088
:100B7000D9F800000FF0E2FBA6490FF033FC07465E
:100B800030460FF0DBFBA4490FF02CFC0146384641
:100B90000FF020FB0FF0ECFDC9F800009F4AA04BBE
:100BA000168819889F4AA04B12681B889F4FC6EB76
:100BB000050E3544039EC6F800E0461A0844049921
:100BC0000D6001990E6002993E8808609A4280F299
:100BD00089810025C3EB060E954974450F6880F2A4
:100BE0007681611C9F4205FB01F50EF1010E95FB1C
:100BF000FEF5C0F2BE81BE42A8BF3E46F61A01FB1A
:100C000006F494FBFEF49A4200F33681BB42C0F234
:100C10003381884C20680FF091FB87490FF0E2FB8D
:100C200086490FF0D7FA0FF0A3FDA0F5FF531C3B48
:100C3000082B98BF4FF40050D8F800301844002813
:100C40002060C0F24281B0F5804F80F252817C4B2F
:100C50001B781BB1B0F5005F40F05381794D2B78C4
:100C6000002B40F05481784D20682B68714C9842DD
:100C700004D080B208F076FA23682B6009B0BDE892
:100C8000F08F28460FF05AFB70490FF0ABFB05467A
:100C900050460FF053FB6E490FF0A4FB0146284667
:100CA0000FF098FA0FF064FD0546CBF80050D9F824
:100CB00000000FF043FB65490FF094FB07463046F8
:100CC0000FF03CFB62495FE728460FF037FB5A49BB
:100CD0000FF088FB054650460FF030FB5D490FF0E2
:100CE00081FB014628460FF075FA0FF041FD0546DD
:100CF000CBF80050D9F800000FF020FB4E490FF060
:100D000071FB074630460FF019FB52493CE7284675
:100D10000FF014FB50490FF065FB054650460FF0ED
:100D20000DFB4E490FF05EFB014628460FF052FACC
:100D30000FF01EFD0546CBF80050D9F800000FF06B
:100D4000FDFA45490FF04EFB074630460FF0F6FA24
:100D5000424919E7D8F80030DFF810B103EBD3733C
:100D60005B10DBF80050C8F800301FE6DFF80081A8
:100D7000DFF80091D8F8003003EBD3735B10C8F8AC
:100D80000030BDE5364A06931188364A0591204663
:100D90000492DFF8D8B00FF0D1FA049A0599DBF885
:100DA000005052F821100FF01DFB0FF0E1FCEF1B7B
:100DB000069B5745A7EB0302B8BF5746FF1AD8F862
:100DC00000309042BABF013200FB0777474397FBE0
:100DD000F2F73B4403EBD373234A04925B10C8F849
:100DE0000030E3E50FF0AAFA029A52F82B100FF048
:100DF000F9FA0FF0BDFCCAEB0802B045B8BFB04627
:100E00008242CAEB08083FF76AAD00FB08F898FB7E
:100E1000F2F069E5CDCC4C3FCDCC4C3E128AFF1FA1
:100E20005889FF1F709CFF1F409EFF1F549CFF1F8F
:100E3000BC9EFF1FB889FF1F9A99193FCDCC4C4526
:100E4000729FFF1FC89CFF1F2089FF1F3333733F12
:100E5000CDCC4C3DCDCCCC3E6666663FCDCCCC3DBA
:100E60005C9CFF1F1C200100D89DFF1F609EFF1F80
:100E70007C9EFF1F089CFF1F009B1B88002B3FF4DC
:100E8000C8AE2B1B002BB8BF5B42092B47DD05F515
:100E900000500130001B0FF051FA3B493B4C0FF062
:100EA000A1FA054620680FF049FA39490FF09AFA7D
:100EB000014628460FF08EF90FF05AFCD8F80030A2
:100EC000184400282060BFF6BEAE002213E09F4207
:100ED00005FB04F5B8BF002195FBFEF54BDA91FB4D
:100EE000FEF490E6B242D4BFC3EB0205C3EB0605A5
:100EF00070E643F6FF72274B22601B78002B3FF40D
:100F0000ADAE05F0D3FA244B01221A70ABE605F022
:100F1000C9FA00232B70A6E6D9F800003EE64FF48C
:100F200000501A4C88E61D491D4A069320460D883C
:100F300005920FF003FA059ADFF868B052F8251011
:100F4000DBF800500FF04EFA014600200FF040F998
:100F50000FF00EFC2F44069B56E50FF0EFF9039AB5
:100F600052F82B100FF03EFA014600200FF030F936
:100F70008AE51E4642E6B742D4BFC3EB0701C3EB86
:100F8000060104FB01F1AAE7CDCCCC3EB889FF1FD6
:100F90009A99193F729FFF1FC89CFF1F5C9CFF1FFF
:100FA0001C200100609EFF1F08B5244B1B88FBB16D
:100FB000234B1B78FBB1234B1B78E3B1224B1B78EF
:100FC000CBB1224B1B78B3B1214B22481A78C2B95E
:100FD000214A22490088128809680244B1EB620F55
:100FE00009DD01221A706420BDE8084005F072BADC
:100FF000174A117801B908BD1370BDE8084008F020
:101000007BB8154A16490088128809680244B1EB7A
:10101000620FF0DD00221A7008F06EF8642005F00F
:1010200059FA642005F056FA642005F053FA4FF49B
:101030001670BDE808400CF0D3BB00BFE69DFF1F53
:10104000969EFF1F979EFF1F989EFF1F999EFF1F52
:101050003C9CFF1F549CFF1F409EFF1F709CFF1F66
:10106000BC9EFF1F38B5114C232025780BF066FE7F
:101070000F4A42F82500131F02F1C400002253F862
:10108000041F83420A44FAD123780A4907480A4CCC
:101090000133DBB2322B81FB025108BF0023D21790
:1010A000C2EB21120370226038BD00BF269CFF1FD7
:1010B000E89CFF1F1F85EB513C9EFF1F2DE9F04F61
:1010C000B84CB94D2068B94F83B00FF037F9B84923
:1010D0000FF088F9064610200CF074FD0FF02EF981
:1010E000B4490FF07FF931460FF074F80FF040FB70
:1010F0002988206088423B8843DA9E465B1A7F2B12
:101100004FF0000247DDD2015E1C92FBF6F2AA4EC0
:10111000DFF8C882B6F800C0C8F80020BCF1190F8B
:1011200000F0DF80BCF11A0F00F01781BCF11E0F38
:1011300000F020810126B146A04A1288002A00F062
:101140009D808842C0F207817045D4BFC1EB00008A
:10115000C1EB0E009A42BABF02FB000001335043BC
:1011600090FBF3F3964A1360964B1888C0B9964AE1
:101170001288AAB9954B197801B11A7003B0BDE86D
:10118000F08F9842D4BFC1EB0002C1EB03029E4630
:101190005B1A7F2BB7DCC2EBC21292FBF3F2B6E70D
:1011A0002988D4F800E0DFF80082DFF8F8A1714563
:1011B0006CDCDFF818C29CF80020002A2ED14FF01A
:1011C000010B04288CF800B028D1002E40F0948147
:1011D0007D4B18880028D1D0B9F1000FCED02368FC
:1011E0002C883A88A34280F265810023141B7E2C50
:1011F000774DD5BFC3EB8313C3EBC3135B0001343F
:1012000093FBF4F42B680134A34203D0C0B2E1B2E3
:1012100007F0CAFE2C6003B0BDE8F08F012800F093
:10122000F680022800F0EB800328D1D1694B1B889F
:10123000092BCDD0002ECBD023682E883A88B3421C
:1012400080F27B810023961B7E2EDFF88CA1D5BF18
:10125000C3EB8313C3EBC3135B00013693FBF6F6BA
:10126000DAF800300136B34203D0F1B24A2007F079
:101270009BFECAF80060ABE716469146BCF11E0F14
:101280007FF472AF0022DFF858817EE04F4B1A786E
:10129000002A3FF473AF002401281C7000F0A480E2
:1012A000022840F00E81002E00F0A3804A4D2B68EA
:1012B000002B00F09E800420214607F075FE424B73
:1012C0002C60188800283FF459AFB9F1000F3FF4A3
:1012D00055AFC0B2002107F067FE3D4B00221A60F7
:1012E0004CE7DFF8FC8098F80020C2B1DFF8D89016
:1012F000B9F800A0BAF1000F11D0DFF8E89099F822
:1013000000B0934578D05FFA8AF07F2107F04CFE59
:1013100098F80030B6F800C089F8003010E0DFF827
:10132000C49099F800A0924566D0274B0021187808
:1013300007F03AFE98F80030B6F800C089F800309F
:101340001E4B1A88002A97D0BCF11E0F40F0068170
:101350000026B14619E00020FCE6DFF8848098F80A
:101360000020002A0BBF012600264FF000094FF095
:101370000109E1E6DFF86880104B98F800601A88F0
:10138000B6FA86F676094FF0000998F80030002B7F
:101390003FF4E8AE2988B7F800E02068C1EB0E03FF
:1013A000CFE600BF649CFF1FEC9DFF1FE89DFF1F61
:1013B0009A99193FCDCCCC3E729EFF1FA09EFF1F75
:1013C000E09CFF1F6E9CFF1F829EFF1F779EFF1FEA
:1013D000489CFF1F2C9EFF1FE49CFF1F589EFF1F71
:1013E0002E9CFF1F2A9CFF1F1EB1614D2B68002BF6
:1013F0007BD1604B188865E70026B1469CE6002E3D
:101400003FF4E6AEDFF868A1DAF800202EE0002E07
:101410003FF4DEAEB7F80080F045D4BFC1EB080260
:10142000C1EB0E02C1EB0808B8F17E0FDFF840A156
:10143000D5BFC2EB8212C2EBC212520008F1010802
:1014400092FBF8F8DAF8002008F10108424506D0CE
:101450005FFA88F10120009307F0A6FD009B188831
:10146000CAF8008002287FF4DFAE42462168B5F852
:1014700000803888414559DA0021C8EB0008B8F1EE
:101480007E0FD3BFC1EB8111C1EBC11108F101087F
:10149000490091FBF8F808F10108904506D05FFA81
:1014A00088F10420009307F07FFD009B1888CAF89C
:1014B0000080B9E69342D4BFC4EB0303C4EB02033C
:1014C00094E6032827D12C4B1B88092B91D0002EA2
:1014D0008FD0274D2B68002B8BD04A20214607F058
:1014E00063FD244B2C601888ECE6214607F05CFD78
:1014F000204B2C601888E5E640207F218DE80C0009
:1015000007F052FD019B009A188858451CD002280C
:101510007FF48AAE76E704287FF46BAF002E3FF4A9
:1015200068AF2146402007F03FFD62E78142D4BF0B
:10153000C8EB0101C8EB00019FE79342D4BFC6EBA3
:101540000303C6EB02037EE6B8F80010DAF800E009
:10155000B7F800808E45FFF665AF5DE72988B7F8DC
:1015600000E020680026C1EB0E03B146E9E500BFAC
:10157000E49CFF1F829EFF1F2C9EFF1F08B5114B8E
:101580001B88022B09D0052B07D0032B15D0042B69
:101590000BD00D4B01221A7008BD7F21412007F0AE
:1015A00003FD094B01221A7008BD7F21092007F0B5
:1015B000FBFC054B01221A7008BD4021092007F0F1
:1015C000F3FCE6E7DE9CFF1F929CFF1F38B5244B1F
:1015D0001B881D2B40D0234B1B88012B25D0224A72
:1015E000224B14881B68224AA342128828DB214917
:1015F00009889342D4BFC4EB0303C4EB0203121B5C
:10160000914224DA01FB0333541C93FBF4F41A4B8C
:101610001A4D1B88052B06D02B689C4203D0E1B2E3
:10162000052007F0C1FC2C6038BD154B154A1B681E
:101630001488154AC3F53B630833A3421288D6DAEF
:101640000C490988121B91424FF00003DADB03FBBF
:1016500001F393FBF2F4DAE7064B1C88D7E700BFEF
:10166000729EFF1FE49DFF1F8E9CFF1F1C9CFF1F8F
:10167000709EFF1F789EFF1FDE9CFF1F149CFF1FA4
:10168000F09DFF1FDC9CFF1F5C9EFF1F38B5124DB5
:10169000124C2B88052B12D022684AB9022B0ED08F
:1016A000033B012B13D90E4A00231370236038BD6E
:1016B0000021052007F078FC2B88022B04D10021A3
:1016C000412007F071FCEEE7052BE9D1F7E7002197
:1016D000092007F069FCE6E7DE9CFF1F149CFF1F52
:1016E000929CFF1F08B5284B1B78ABB115200BF05F
:1016F00025FB264A264B128818601D2A15D0254A3C
:101700001288DAB1012A2BD0234B1B78002B3AD058
:10171000BDE80840FFF7BABF11200CF053FA1B4A8E
:101720001B4B128818601D2AE9D11C4B1B88002B0B
:10173000EAD01B4B1B78002BE6D008E0174A128832
:10174000002AE1D0174A1B6812889A42DCDC124B4F
:101750001B780BB9FFF712FFBDE80840FFF736BF53
:101760000F200CF02FFA0D4B0F4A1B88106033B17D
:101770000E4BC0F53B601B8808309842E7DA064BF9
:101780001B78002BC4D108BDF89DFF1F729EFF1F60
:101790001C9CFF1FE49DFF1F929CFF1FDE9CFF1FF0
:1017A0002E9CFF1F8E9CFF1FF09DFF1FDC9CFF1FC8
:1017B000F8B510200CF006FAC830B0F5FA7FC0F288
:1017C0009780B0F57A6F0146A8BF4FF47A6101F5B2
:1017D0001673B3F57A6FA8BF4FF47A639BB289B2E0
:1017E000914A924C11802220238007F061FD2188CC
:1017F0008F4D904C242007F05BFD0E200BF09EFADD
:1018000040F6FF71C8308842A8BF084620EAE07061
:1018100000F5FA6283B28A42A8BF0A46022019463E
:1018200022802B8007F044FD2188042007F040FD32
:1018300001200CF0C7F9044600200CF0C3F9A042C7
:10184000B8BF204600F1C801B1F5FA7FC0F2D280DE
:10185000B1F57A6FA8BF4FF47A6101F54873B3F51B
:101860007A6FA8BF4FF47A639BB289B2724A734C05
:1018700011800A20238007F01BFD21880C2007F02F
:1018800017FD0F200CF09EF9C0F53F610E31B1F548
:10189000AF6FC0F2AC80B1F5FA6FA8BF4FF4FA6138
:1018A00089B2C0F54460664B0E30B0F5AF6F198059
:1018B000C0F29A80B0F5FA6FA8BF4FF4FA6083B215
:1018C000604CA420238007F0F3FC2188A62007F0B9
:1018D000EFFC15200BF032FA00F59671B1F52F7F71
:1018E0000BDB41F25C23994240F38980194608E002
:1018F00040F24C434FF4FA7172E740F214534FF444
:101900002F71514A1180514C514D2380062007F010
:10191000CFFC21884F4E082007F0CAFC00274FF467
:10192000AF74F9B24C4809F047FA55F8043BC3F5D7
:10193000967300FB03F086FB0023C017C0EB631017
:10194000844207F10107A8BF0446062FE9D1434F9F
:10195000404E0025E9B2424809F02EFA57F8043B00
:10196000C3F5967300FB03F086FB0023C017C0EBA2
:101970006310844205F10105A8BF04460C2DE9D18E
:10198000384F344E0025E9B2374809F015FA57F8B8
:10199000043B304AC3F5967300FB03F086FB00134B
:1019A000C017C0EB6310844205F10105A8BF0446CF
:1019B0000C2DE8D1A4F11401312931DD40F23A7344
:1019C000A4F5B97403FB04F482FB0432E417A4EB1E
:1019D000621289B232322548254B01801A602A20D2
:1019E000BDE8F84007F064BC4FF4AF6368E74FF41C
:1019F000AF6156E740F214534FF4FA7136E7124ADA
:101A000000F5617089B2B0F52F7F1180B8BF4FF437
:101A10002F73FFF678AF8342A8BF03469BB272E7ED
:101A200040F26C723221D6E7EC9DFF1FE89DFF1F4C
:101A3000D89CFF1F9A9EFF1F409EFF1F549CFF1FB4
:101A4000DC9CFF1F5C9EFF1F8E9CFF1F709EFF1F74
:101A5000488AFF1FB5814E1B409CFF1F188AFF1F3D
:101A6000749CFF1F2889FF1FD09CFF1F949EFF1F9F
:101A7000008AFF1F2DE9F84F0C200BF02BF90C20EA
:101A80000BF0E0FDBF4914200BF0ECFDBE49BF4850
:101A900008F024FE022103200BF07AFE022104202C
:101AA0000BF076FE022105200BF072FE02210620CB
:101AB0000BF06EFE01210A200BF06AFE01210920C5
:101AC0000BF066FE01210D200BF062FE01212820A3
:101AD0000BF05EFE012114200BF05AFE01211620AE
:101AE0000BF056FE172001210BF052FE04200BF0E4
:101AF00041FE00283DD005200BF03CFE04460028A6
:101B00003ED000242046A24D287005F0E9FF2E7833
:101B10005EBB204607F0F6FB9E4B9F491B880F8853
:101B20009E4ADFF8DCE29E4DA3F5AF7140F23A73B6
:101B300003FB01F382FB0312DB17A3EB62133233C7
:101B400001210D20CEF800302F700BF00DFE642027
:101B50000BF046FE4FF416710A200BF075FC5D2168
:101B6000904809F065F990B9FEE7BDE8F84F08F034
:101B7000C5BC06200BF0FEFD0028BCD10124C2E745
:101B800003200BF0F7FDB0FA80F04009BBE76420BA
:101B90000BF026FE31460A200BF056FC4FF49671EE
:101BA00009200BF051FC5C217F4809F041F900B994
:101BB000FEE764200BF014FE314609200BF044FCD4
:101BC0004FF4967116200BF03FFC5B21774809F02B
:101BD0002FF900B9FEE764200BF002FE3146162013
:101BE0000BF032FC4FF4967117200BF02DFC6420A3
:101BF0000BF0F6FD314617200BF026FC64200BF0AD
:101C0000EFFD31460D200BF0AFFD694A69481268BF
:101C1000DFF8F0B1DFF8A4A1674FDFF8EC91DFF84F
:101C2000EC8100230121FEF73FFC0123CAF800608C
:101C30003E60C9F800608BF8003004260F200BF0DE
:101C4000C1FFD9F8003003440E20C9F800300BF072
:101C500075F8DAF800309BF800200344CAF8003029
:101C60001520002A7DD00BF069F83B6818443860D5
:101C700006F0010080F0010004F01CFCB8F8003010
:101C8000002B14BF4B20DC200BF0AAFD013ED5D168
:101C9000D9F80030DAF8002048493868DFF870E1F8
:101CA000474E002BB8BF0333002AB8BF033292104F
:101CB0000A604449444A098812880028B8BF0330A2
:101CC0009B10801038605F1A19443160CEF80070A4
:101CD0003E4E3F4F3F49C9F80030C2EB000E024470
:101CE000C7F800E032600B600CB1FFF761FDB8F897
:101CF00000305BB94FF4FA7004F0ECFB04F0D6FB53
:101D000006F0F6F94FF4AF600BF06AFD324B012498
:101D100004201C600BF02EFD10B9304B28701C7095
:101D20002F4B1B881C2B23D02E4C04F1C8052320DD
:101D30000BF004F844F8040F01200BF051FDA5420C
:101D4000F5D1294A294B1078187007F0E5F904F00D
:101D5000A9FB45F6BF5226492648BDE8F84F0AF0D0
:101D6000A5BD11200BF02EFF3B68184438607FE7BB
:101D7000214B18880028D7D0204BC0B2197807F023
:101D800013F9D1E7001B374640420F00F890FF1FC0
:101D9000449CFF1F949EFF1F049EFF1FB5814E1B96
:101DA000A09CFF1F409CFF1FD09CFF1F749CFF1F27
:101DB0002489FF1F089EFF1F089CFF1F209CFF1FF8
:101DC000D89DFF1F128AFF1F5889FF1FA49CFF1F69
:101DD000689CFF1FA89EFF1F6C9EFF1F2F9CFF1F6C
:101DE000729EFF1FE49CFF1FF49DFF1FD39DFF1FEA
:101DF000A50500008C9EFF1FA89CFF1F609CFF1F75
:101E0000008AFF1FF89DFF1F609EFF1F369EFF1F69
:101E1000649EFF1F2DE9F04FAC4C2678012E95B043
:101E200000F04582C0F0FB81022E00F0CB80A84973
:101E3000A84A91F800801178A74ADFF82CE3A74D53
:101E4000A74FA848A84B0292A84A0092A84A9EF819
:101E500000B001922D78A74A3F7890F800E01B78F7
:101E6000DFF80CA3DFF80CC3DFF80C930392012E0C
:101E700084BF00222270A04AA0481370A04A80F8B4
:101E800000B015709F48A04A077082F800809F48F4
:101E90009F4A03709CBF013626701170BEF1000F7F
:101EA00040F009819B4A10880D2800F0A9819A4CC6
:101EB00000202070024604462DB196480088002874
:101EC00040F0AA810546954806882544002E40F03A
:101ED00057819348934C019E0078367824780130DE
:101EE000A0EB4600002C40F04682039C94F800E0F2
:101EF000CEEB0004BEF1000F40F066820026DFF852
:101F000064E202989EF800E00078A41BA4EB4E0463
:101F10003C44CBEB040410B1B7FA87F040099CF8BD
:101F200000602718BC1B1EB11EF1000618BF012659
:101F3000009F99F8000097F800909AF800C07A4F37
:101F4000C6EB040EC0EB0E00A0EB49008044C3EBCF
:101F50000803A3EB41010C2313FB0C113960734BF5
:101F6000734C744E1B887448248837680088734EFD
:101F7000033B03EB4303C4EBC40401EB83033C4486
:101F800003440C3B56F824001D4405440AB16C4B35
:101F900019606C4B1A68954200F02E816A4A6B48B2
:101FA0001168079107990160126808926848089AB9
:101FB00000881D60521A824284BF664A156015B0BF
:101FC000BDE8F08FDFF8B481634E08AF0025E9B2B9
:101FD000624808F0F1FE58F8043BC3F5967300FB25
:101FE00003F086FB00230135C017C0EB63100C2DF6
:101FF00047F8040BEBD15A4B3D4D01953D4DB3F8DD
:1020000000C00395109D09980F99464EDFF8D4A0A3
:10201000DFF8C890DFF8D080654511AA8CCAAE46BB
:10202000ACBF4FF0000E4FF0010E8445D4BF00202E
:10203000012030708C452E480B9D254E8AF800E01B
:10204000D4BF00210121017094452A49DFF820A165
:10205000D4BF002201220A709C45424AD4BF00230B
:102060000123BC45AB46D4BF002701271370AC4504
:102070001B4B0C9D1F70D4BF4FF0000B4FF0010B9A
:10208000394B154A0292AC45DFF848C0174A83F82D
:1020900000B0D4BF0025012589F8005098F8003021
:1020A0009CF8001096F80080DFF8C8C02678DFF8AA
:1020B000C8900092DBE62D4A174814880122182C9C
:1020C000027040F260810024F6E600BFD29DFF1F3F
:1020D000289EFF1F2A9EFF1FB89CFF1FC49EFF1F44
:1020E000909CFF1FC99EFF1F299EFF1F759EFF1F0B
:1020F000859EFF1F869EFF1FC39EFF1FEB9DFF1F38
:10210000C59EFF1FC69EFF1FC79EFF1FC89EFF1FC5
:10211000769EFF1FCA9EFF1F2E9CFF1F189CFF1F4D
:10212000148AFF1FB49EFF1F309EFF1F4C9EFF1F8F
:10213000689EFF1FE09CFF1F289CFF1F341E0100AC
:10214000AC9EFF1F889CFF1FB09FFF1F789CFF1F46
:10215000809EFF1FB89EFF1FB5814E1BD09CFF1FA6
:10216000949EFF1F879EFF1F919CFF1F729EFF1F63
:10217000DD9DFF1FC29EFF1F749EFF1F2889FF1F4A
:10218000012E00F08F81022E00F0EE81032EA74B6E
:1021900000F01F811E78009B9CF800E01C78019BDA
:1021A00099F800C01878029B93F80080039B1F7871
:1021B000A6EB4E03A4EB8404CCEB030CC0EB8076BF
:1021C0000CEB0403C0EB8600034403EB480303EB72
:1021D000810327B196490978002940F060820126E1
:1021E0009AF800109348C1F1060101EB4101334414
:1021F00003EB81010160B2E68F49904A0968D3E69A
:10220000002D3FF454AE8E4A8E4E14880122182CB5
:10221000327040F2B8807446A0F10D0553E6DFF845
:102220007092894F0DF120080025E9B2874808F027
:10223000C3FD59F8043BC3F5967300FB03F087FB1D
:1022400000230135C017C0EB6310062D48F8040BBE
:10225000EBD17F4BDFF83CA219880D9B00228B420B
:102260008AF8002080F2A2807A4B8AF800507A49DE
:102270007A4A7B4891F8008011787A4A1D70029260
:102280000378794ADFF810C2DFF810920092774A9B
:10229000774E784D784892F800E0784A0192784A73
:1022A00096F800B02D78077826780392DFE5DFF8FE
:1022B000F081654E08AF0025E9B2724808F07CFD58
:1022C00058F8043BC3F5967300FB03F086FB00232C
:1022D0000135C017C0EB63100C2D47F8040BEBD190
:1022E0005B4B0C9D1F885F4B02935F4B00930B9BD6
:1022F0000A98099ADFF8A0C1089EDFF8A0910F990B
:10230000BB429E46ACBF4FF0000E4FF0010EAF42F5
:10231000D4BF002501258742109B8CF80050D4BF04
:1023200000200120504D89F800009742D4BF0022C0
:102330000122B742D4BF4FF000084FF001082A70C5
:102340009F42474A4448474E80F80080D4BF00234C
:1023500001231370129A414886F800E08F42D4BFDF
:1023600000210121974201701ADC00224648DFF863
:1023700024A102708BE7039C46B12678002E40F022
:102380006081441EBBE50C3C012295E594F800E019
:102390000138CEEB0004BEF1000F7FF4B0ADADE527
:1023A000119A9742D4BF00220122DFE70C9A374BE3
:1023B0009142CCBF012200221A7040F345810525CD
:1023C0008AF80050234B52E7002E3FF497AD0126C8
:1023D00095E51C78009B029893F80080019B9CF87F
:1023E00000601B7890F800C099F800700398A4EB87
:1023F0004604E71B90F800E0C3EB8374A8EB880069
:102400003844C3EB8403034403EB4C0303EB810325
:10241000BEF1000F40F0488101269AF800100548EF
:1024200033440C2414FB0131016098E5148AFF1F2A
:10243000879EFF1F309EFF1F789CFF1FB09FFF1FCE
:10244000729EFF1F2E9CFF1FB5814E1B409CFF1FDD
:10245000949EFF1FEA9DFF1F289EFF1F2A9EFF1FBD
:10246000299EFF1FB89CFF1F759EFF1FC99EFF1F5F
:10247000919CFF1FC49EFF1F909CFF1F859EFF1F06
:10248000869EFF1F749CFF1F5A9CFF1F999EFF1F73
:10249000488AFF1FDD9DFF1FC29EFF1F749EFF1F06
:1024A000188AFF1FA34CDFF89CE2207805909EF865
:1024B000004001980494059C007801900134A4EB3D
:1024C00040040498002840F0AF80039890F800E0A2
:1024D0000498261ACEEB06000390BEF1000F40F0E0
:1024E0009E8074460298944E007802900398367845
:1024F0000496041BA4EB460402983C44CBEB040472
:10250000002800F08780B7FA87F040099CF8006047
:102510002044871B1EB10498061C18BF0126009C8E
:1025200099F800002478BE1B301AA0EB44008044C8
:102530000198C3EB0803A3EB4103002867D1BEF168
:10254000000F40F0BB807344002C5ED100290CBF0B
:1025500000206FF009009AF80010784C03440C201A
:1025600010FB01312160FAE4039E019C367803964A
:10257000009E2478019434786F4E714899F800E0F9
:10258000009496F800906F4C9DF80C6086709DF852
:102590000460067080F806E09DF8006080F8039003
:1025A0009CF800C02478DFF8B491DDF804E080F8EE
:1025B0000880077180F805C0C671417244704FF001
:1025C00000080120009500215D4C0D465FFA88FC53
:1025D0004F46764607E0022809D00A290BD014F8A6
:1025E000016F17F8010F864201F10101F3D10135A6
:1025F0000A29EDB2F3D1092D72D808F10108B8F11A
:10260000100F36D019F80A0FDDE70020A3E74FF0CE
:10261000000E98E7029879E7CEEB0400039001984A
:10262000041C18BF01245DE7019800284ED00398D0
:1026300090F800E0BEF1000FEED1601E03907446EA
:1026400050E7841B01265AE40B9A3F4B9142CCBFC2
:10265000012200221A703EDC0A9A3C4B9142CCBF08
:10266000012200221A7052DD03258AF80050384BEF
:10267000FDE5304837490478C86B0299009D097818
:1026800001342044CBEB0000084400219AF80040BC
:102690002A4B401A0C2111FB040119605FE41BF165
:1026A000000618BF01269BE52349097800293FF45D
:1026B000B3AE1BF1000618BF0126AEE60498002851
:1026C0000CBF4FF0000E4FF0090E3CE7039890F856
:1026D00000E03046FDE604258AF800501C4BC6E5B4
:1026E00014481C49047851F828000299009D097883
:1026F00001342044CBEB000066460844002BC4D0D4
:10270000002EC2D1BBF1000FBFD00121BEE7099A54
:10271000114B9142CCBF012200221A7004DD022528
:102720008AF800500A4BA2E5089B994218DD012562
:102730009AE500BF148AFF1F879EFF1F309EFF1F70
:10274000AC9CFF1FB49EFF1F989EFF1F979EFF1F0C
:10275000EA9DFF1FC089FF1F969EFF1FE01C01001E
:10276000134B1D78012D21D9124A8AF80050128886
:10277000002A3FF47CAD104A1288013A92B2062A30
:102780003FF675AD0D4A1278002A3FF470AD0C4A41
:102790001268012A7FF46BAD0A4A0B4E10680C22B6
:1027A00090FBF2F102FB1102328060E535465EE5F6
:1027B000EA9DFF1FC09EFF1FF69DFF1FDA9CFF1FB3
:1027C0006C9EFF1FB89EFF1F349EFF1F2DE9F04F28
:1027D0003A4B1B788BB0002B6BD10E200AF0AEFA6F
:1027E0000DF0ACFD01463648364E374DFDF7A2FEE2
:1027F0003348FDF775FE0DF0BBFF80F30C00306031
:10280000FFF708FB2C68012C7AD0022C00F09D8287
:10281000032C00F0AB832D4E2D4C33682D4A2E4EE9
:102820000993099B316812882360591A013A914231
:10283000274F00F28582294E32689A1A0D2A00F23B
:102840007882274E32689A1A132A00F26D82254E3A
:1028500032689A1A252A1AD9234B1B88002B40F07C
:102860005481224B1B78002B40F04F81FEF7FAFB7E
:102870001F4B1B881B3B9BB2022B04D81D4B1B78A4
:10288000002B40F0458103F037FE236833601A4D7A
:102890002A689B1A502B00F20382184B1B88012BCD
:1028A00000F01B8206F014FC06F042FA0BB0BDE803
:1028B000F08F07F0ABFC0BB0BDE8F08F449CFF1F1E
:1028C000089EFF1F449EFF1F6C9EFF1FB09FFF1FAF
:1028D000009EFF1FBC89FF1FD49CFF1FC09CFF1FD1
:1028E000989CFF1F9C9CFF1FE69DFF1F3C9CFF1FA9
:1028F000729EFF1F2E9CFF1FE09DFF1F489EFF1F23
:10290000DFF80C939C4AB9F800001378834204D096
:10291000C3B21846137006F017FBDFF8F082974A2F
:10292000B8F800301178994204D0954F39780029D1
:1029300040F0DA86934A33681288934E9A42C0F286
:10294000F180924A1278002A40F0EC80DFF8C4A2AD
:10295000BAF8003023B98E4B1B88002B00F0E384BB
:102960008C4A8D4B11881B888C4A0B4412685B1073
:1029700093428B4A126880F2858400219342B4BF4F
:1029800001230B4604910093ACBF4FF0010B8B4623
:1029900005910E200AF0D2F9824B834A1B68176812
:1029A00003930133A7F25232002B8446029240F384
:1029B000C286802BA8BF80237C4A7D491278019172
:1029C000002A00F0B9800978914200F0B580B8F88B
:1029D0000010DFF838E2994201F0D7806849AEF87C
:1029E0000030744B4FF0010E81F800E01978DFF8E9
:1029F00028E2019B8EF800101A70009B002B00F05B
:102A00000D81BAF80030002B00F008816A4B1B687A
:102A10005A1C002A40F39386802A00F38F86674C65
:102A2000674968482488098800682144B0EB610F31
:102A3000C1F22083A3F148020F2A02D8473BA9F82C
:102A400000300E200AF07AF96FF454731F44874265
:102A500002DC5D4B00221A705C4B1B88002B00F0DF
:102A600009845B4B5B4A1B781178994240D0002B5C
:102A70003ED059490C78002C00F01D87574991F839
:102A800000C0BCF1000F40F01487554F0097554F20
:102A900055480297524F007887F800C0514F4FF0C9
:102AA000010E87F800C081F800E0002841F0C480E2
:102AB0004E490978002900F0E0874D4903910C4602
:102AC0000978002940F0D6874A48464F0078397087
:102AD00001210297217058B14148404900900020DF
:102AE00008700099029F0870039901243C700870D7
:102AF0001370414B1B88A3F11B02012A40F2B885D9
:102B00001D2B00F002863D4C87E6FEF74DFAADE640
:102B10003B4B1B78002B3FF4B6AE2B68012B7FF4A8
:102B2000B2AEB2E63168374A06910698364910606F
:102B300002220B602A6009E71E49DFF8DCE0097811
:102B400000293FF456AF9EF8000081423FF451AF98
:102B500003984B2840F3E0871833802BB8F8000027
:102B6000A8BF802398423FF444AF2848038004481C
:102B7000012303703DE700BFD39DFF1FA09CFF1FF3
:102B80002F9CFF1FD89CFF1FB09FFF1F3C9CFF1F67
:102B9000C69CFF1F549CFF1F409EFF1F709CFF1F81
:102BA000BC9EFF1FAC9EFF1F209CFF1FA29EFF1F0D
:102BB000849CFF1FA39EFF1F309EFF1FEC9DFF1FE5
:102BC000E89DFF1F649CFF1FDC9DFF1FF69DFF1FFC
:102BD0005A9CFF1F0C9CFF1FC69EFF1F389EFF1FA5
:102BE000849EFF1FDA9CFF1FC79EFF1FC39EFF1F0F
:102BF0000D9CFF1F2E9CFF1F729EFF1F009EFF1F3C
:102C0000769EFF1F949CFF1FFC9DFF1F049EFF1FCD
:102C1000F49DFF1F8C9CFF1F859CFF1F029B9C4502
:102C2000BFF60FAF864B1B88002B3FF40AAFBBF1FA
:102C3000000F7FF4EBAE834B1B881BB1059B002B71
:102C40007FF4E4AE049B002B3FF4FBAE7E4B1A787E
:102C5000002A7FF4F6AEDFF8649299F80040012272
:102C60001A70002C40F02C83784B1B78002B02F05C
:102C7000C680774B1B78002B02F09A83754B1B782C
:102C8000002B7FF4DEAE744B1B78002B3FF4D9AEE3
:102C9000B8F8003071490A3BA8F800300A70D0E655
:102CA00004F066FF6E4B1B7873B96E4B1B785BB9F3
:102CB0006D4B1B7843B96D4B1B782BB96C4B1B7854
:102CC00013B903F0EFFB01E003F0F8FB23682B607E
:102CD000684B1B88012B7FF4E5AD674A674B116891
:102CE00067481A78A1F118032A2101FB03F101605A
:102CF000002A00F0A982634C2368994200F35283B2
:102D000010DA61480278002A40F07C875F4A106838
:102D1000D0F17F0048BF0330801001301B1A994268
:102D200042F3BF86216091E2FEF7DCFC236833604A
:102D30008DE5FDF771FDFEF7C1F92368336080E58D
:102D4000FDF7E2FC3B68336075E5514A3468118851
:102D5000A14204DB464B1B78002B00F05D834D4EF7
:102D60004D48336807934D4B079A00681B88121A29
:102D70009A4200F2A980002B00F0A680484B1A88E6
:102D8000002A3FF4C0AE474B47481B680088A34267
:102D9000B8BF2346994241F36681444B1960DFF87E
:102DA000208188F80020344FFDF7AEFC38687F287A
:102DB00040F371853E4B7F3883FB0032C317C3EB72
:102DC000620303EB4303A0EB83007330394B0193A1
:102DD0001B883860002B40F0CA86234B00931B7879
:102DE000002B00F0C683344C2378002B00F0C18305
:102DF000DFF8D090DFF8B8A04FF0000B0CE003F143
:102E00007300C0B298F8001006F0F6F823780BF1C2
:102E1000010B5B4540F3AD833B6859F8040F184440
:102E2000A0F17F038AFB0321DA17C2EB610202EBF8
:102E300042027F28A3EB8203E1DCFDF723FCE0E7FD
:102E4000C69CFF1FFA9DFF1FDC9DFF1FC39EFF1F37
:102E5000EB9DFF1FC59EFF1FC69EFF1F2F9CFF1FE0
:102E6000DA9CFF1F389EFF1F849EFF1F0D9CFF1FD3
:102E70003C9CFF1F489EFF1FB89EFF1F929CFF1F98
:102E80009C9EFF1F349CFF1F889EFF1F149CFF1FEA
:102E9000D89CFF1FB09FFF1F949CFF1FC49CFF1F67
:102EA0002C9CFF1FFC9DFF1F9A9EFF1F109CFF1F65
:102EB000ABAAAA2A6C9CFF1F8089FF1FDD9DFF1F04
:102EC000B99CFF1F5889FF1F554B564A1B68108835
:102ED000554AA342B8BF2346994200F37A82534C25
:102EE00012888342A8BF03462360002A7FF457AFAD
:102EF0009942C8BF134640F37382401AB0F5804F21
:102F0000AABF9B03C3EB8333013093FBF0F0FDF7C3
:102F1000E1FBC0F3C6100DF011FA454B04461888CA
:102F20000DF00CFA4349074620460DF05BFA0146C6
:102F300038460DF057FA21460DF04CF94FF07E510E
:102F400004460DF0EDFB002841F071803A4920461F
:102F50000DF004FC002840F0698620460DF02EFCA0
:102F6000C0B2DFF8F48088F800001CE7334B346807
:102F70001988A14274DD324B1B78002B70D1DFF829
:102F8000DC9099F800007F2840F33886A3F1553390
:102F90007F3803F1004383FB0032C317C3EB6203A6
:102FA00003EB4303A0EB83007330264B01931B8894
:102FB000C0B289F80000002B41F03580224B00930D
:102FC0001B78002B00F0A484204C2378002B00F009
:102FD0009F841F4FDFF87C804FF0000A0AE003F166
:102FE0007300C0B206F030F823780AF1010A5345A5
:102FF00040F38E8457F8043F99F800001844A0F17C
:103000007F0388FB0321DA17C2EB610202EB420265
:103010007F28A3EB8203E2DCFDF734FBE1E700BF8E
:10302000FC9DFF1F9A9EFF1F2C9CFF1F109CFF1FE3
:10303000A49EFF1FCDCCCC3D0000FE42D89CFF1FBC
:103040003C9CFF1F6C9CFF1F849EFF1F8089FF1FFD
:103050005889FF1FABAAAA2AB99CFF1F2E9EFF1FEB
:10306000B34F38687F2800F3C281FDF70BFBDFF810
:10307000249399F800A0824500F02182AD4B1B8873
:10308000002B43D1AC4AAD4812680088914205DC60
:103090008242D4BFC1EB0203C1EB0003411AB1F578
:1030A000804FA6BF9B030131C3EB833393FBF1F049
:1030B000FDF710FBC0F3C6100DF040F9A04B04461D
:1030C00018880DF03BF99F49804620460DF08AF99B
:1030D000014640460DF086F921460DF07BF84FF091
:1030E0007E5104460DF01CFB002840F08F87964966
:1030F00020460DF033FB002840F0958520460DF06A
:103100005DFBC0B2DFF8908288F80000BAF17F0F53
:1031100040F3BD838D48AAF17F0A80FB0A304FEA55
:10312000EA73C3EB600000EB4000AAEB8000733051
:10313000874B00931B78C0B289F80000002B40F049
:103140001A83844B03931B78002B40F04B85824BF2
:1031500002931B78002B40F07E87804B0193029BEB
:103160001B78FBB17E4B1B88012B00F0C385022B23
:1031700001F05380032B01F09281042B01F09D8319
:10318000052B01F03E84062B01F00D86072B01F084
:10319000C187082B02F07880092B02F08C810A2B62
:1031A00002F0C283009B1B78002B00F07684019B09
:1031B0006A4C1988002900F0FD8438687F2840F3A4
:1031C0006383624B7F3883FB0032C317C3EB620318
:1031D00003EB4303A0EB830073303860002940F019
:1031E000AC84009B1B78002B00F075815D4C23782C
:1031F000002B00F07081DFF8A4A1DFF89C814FF074
:10320000000B0CE003F17300C0B298F8001005F059
:10321000F3FE23780BF1010B5B4540F35C813B68C7
:103220005AF8040F494A1844A0F17F0382FB032196
:10323000DA17C2EB610202EB42027F28A3EB8203A2
:10324000E0DCFDF71FFADFE7474B1960474B1B68CF
:10325000A92202FB03F3002BBCBF03F57F533F33CE
:103260009B13543B194481F30C0128200AF0ECF81D
:10327000FFF718BB384C3E483549364A2370037077
:103280000B7035E493424FF0000B80F2BD800123B8
:10329000CDF800B0CDF814B00493FFF77ABB354BEE
:1032A0001B78002B7FF4CDAB039B334A243B83F385
:1032B0004703D9B25B20136005F076FE99F8004011
:1032C000032C30D1DFF8D88098F80030002B42F082
:1032D000BE812A4F3B78002B42F0AC81254C2378ED
:1032E000002B42F09A81264B1B78002B42F08881FC
:1032F000244A1380244B1B78002B42F04E820D4B46
:103300007F221A8098F800306BB93B785BB923783C
:103310004BB91E4A7F210720138005F045FE7F210F
:103320000B2005F041FE1A4B1F68FFF78ABB00BF58
:10333000B89EFF1F2C9CFF1F109CFF1F9A9EFF1F13
:10334000A49EFF1FCDCCCC3D0000FE42ABAAAA2A12
:10335000849EFF1F0D9CFF1FDA9CFF1F6C9CFF1FAC
:10336000F69DFF1F8089FF1F349CFF1FB889FF1F38
:10337000389EFF1FC69EFF1F509CFF1FC59EFF1F4C
:10338000EB9DFF1FCA9CFF1FC79EFF1F2C9EFF1FA8
:10339000209CFF1F2E9EFF1FB99CFF1F5889FF1FF7
:1033A000C39EFF1FBA4A1078002840F05983B94ADB
:1033B0001268D2F17F0248BF033203EBA202531C12
:1033C000B54A23609942B8BF1160FFF63FAF194676
:1033D0003CE7B24B12881960002A7FF4E0AC0B4640
:1033E0009842D4BFC1EB0003C1EB030385E5AC4BAE
:1033F0007F3883FB0032C317C3EB620303EB430345
:10340000A0EB8300733032E60123CDF810B0CDF885
:1034100000B00593FFF7BDBA01232B60A14EA24C6B
:10342000FFF7FBB9029B1B78FBB1A04B1B88012B5C
:1034300000F0E284022B00F06F86032B01F0A580E0
:10344000042B01F05F82052B01F05283062B01F063
:10345000A284072B01F00685082B01F04C87092B6D
:1034600002F04A800A2B02F02882019B1B88002B65
:1034700000F06C83009B1B783BB9039B1B7823B93E
:10348000029B1B78002B01F00080894B1B78002BDE
:1034900000F0288187490B78082B00F223818648A9
:1034A0003A680068854C0133DBB25F1E101A44F89D
:1034B00027000B70824B3468198889F80020A142DC
:1034C000784EBFF620AB32687E4B0892089A764C55
:1034D0001A60FFF7A2B9039B1B78002BA2D03B68B0
:1034E000A3F10C007F2840F36C836D488B3B80FB7D
:1034F0000320DA17C2EB600000EB4000A3EB80036F
:1035000003F17300DFF8D081C0B298F8001005F025
:1035100073FD009B1B78002B84D0664C2378002B16
:1035200080D0DFF8B8A14FF0000B0CE003F173007E
:10353000C0B298F8001005F05FFD23780BF1010B85
:103540005B457FF76FAF3B685AF8040F544A184445
:10355000A0F18B0382FB0321DA17C2EB61020C3866
:1035600002EB42027F28A3EB8203DFDCFDF78AF83F
:10357000DEE74F4B1B78002B40F0EE823B68524A4F
:103580001278002A45D0A3F10C007F2840F3338342
:10359000434A8B3B82FB0321DA17C2EB610202EB49
:1035A0004202A3EB820303F17300C0B298F800104B
:1035B00005F022FD009B1B7853B33E4C23783BB3B0
:1035C000DFF81891DFF8D8A04FF0000B0BE003F103
:1035D0007300C0B298F8001005F00EFD23780BF1CF
:1035E000010B5B4514DD3B6859F8040F1844A0F14A
:1035F0008B038AFB0321DA17C2EB61020C3802EB62
:1036000042027F28A3EB8203E1DCFDF73BF8E0E711
:103610003B682E4A1278FAB1244A1288012A00F037
:103620007284022A00F07786032A01F02F80042A90
:1036300001F08C81052A01F0CE82062A01F0D883A0
:10364000072A01F0B484082A01F0CD86092A01F086
:1036500098870A2A02F0F980019A1288002A00F05D
:103660008D821B4A104C137003232B60FFF7D5B8D3
:10367000DFF86C8098F80030002B40F01081154F77
:103680003B78002B40F0F984074C3B70FFF7C5B83E
:10369000889EFF1F149CFF1F349CFF1F109CFF1F60
:1036A000ABAAAA2AB09FFF1F009EFF1FF69DFF1F17
:1036B000389EFF1F8089FF1F309CFF1F5C89FF1F02
:1036C000D89CFF1F5C9FFF1F0D9CFF1FDA9CFF1FF4
:1036D0002E9EFF1F2A9CFF1FB99CFF1F5889FF1FAA
:1036E0002E9CFF1F3A68E5E6DBB21846137005F022
:1036F00039FCAC4BAC491A46AC4B184600230B7056
:103700003B7013700370FFF715B9DFF8BC8298F8AF
:103710000030002B40F0CF81A54F3B78002BB3D079
:10372000A44BA54C1988A22005F0C2FD98F80030E2
:103730003B70FFF772B80123FFF73EB980249F4921
:103740009F4BA04A09881B8812680B44B2EB630F99
:10375000BFF677A99C4B1B78002B40F01C82B8F871
:1037600000309A4AA3423FF46CA9994B148001227D
:103770001A70FFF766B9974B01931B88002B42F034
:103780008A818A4B0393944B0293944C23786BB3B6
:10379000DFF85C82DFF848A24FF0000B09E003F18C
:1037A0007300C0B205F050FC23780BF1010B5B45B0
:1037B0001CDD58F8043F99F800001844A0F17F037D
:1037C0008AFB0321DA17C2EB610202EB42027F2877
:1037D000A3EB8203E3DCFCF755FFE2E77E4B0293A9
:1037E00005F032FC009B1B78002BCED1039B1B788D
:1037F000002B3FF4B4AC99F80030A3F10C007F2803
:1038000040F3ED8176488B3B80FB0320DA17C2EB57
:10381000600000EB4000A3EB800303F17300C0B233
:1038200005F012FC009B1B78002B00F0CD816B4C47
:103830002378002B01F0C082DFF8B481DFF8A0A16B
:103840004FF0000B0AE003F17300C0B205F0FCFB7F
:1038500023780BF1010B5B457FF781AC58F8043FEF
:1038600099F800001844A0F18B038AFB0321DA17B2
:10387000C2EB61020C3802EB42027F28A3EB820309
:10388000E1DCFCF7FFFEE0E7FCF7FCFEA5E45046B8
:10389000FCF7F8FE4CE4FCF7F5FEFFF797BA514A47
:1038A0001278002A40F0D581414F434C3B70FEF71F
:1038B000B4BF002008704C49087840B139490091E4
:1038C0000978002900F0B581009F0021397047492F
:1038D000097800297FF4F1A8002C40F0CE80002860
:1038E00040F0CB80384C2F4F94F800E02F4C0394DD
:1038F000394C02942D4C2C492070374C009708709D
:1039000038702070BEF1000F7FF4E9A8FFF7F0B81F
:10391000264B1B78002B6DD099F80030A3F10C00DA
:103920007F2840F3CC832E4A8B3B82FB0321DA179E
:10393000C2EB610202EB4202A3EB820303F17300CC
:10394000C0B205F081FB009B1B78002B52D0234CAA
:103950002378002B4ED0264FDFF884804FF0000AEA
:1039600009E003F17300C0B205F06EFB23780AF1A1
:10397000010A53453EDD57F8043F99F8000018440A
:10398000A0F18B0388FB0321DA17C2EB61020C382C
:1039900002EB42027F28A3EB8203E2DCFCF772FE1B
:1039A000E1E700BF849EFF1F389EFF1F0D9CFF1F95
:1039B0002A9CFF1F789EFF1F009EFF1FEC9DFF1F8C
:1039C000E89DFF1F649CFF1F2E9CFF1F049EFF1F8E
:1039D0002F9CFF1F6C9CFF1FDA9CFF1F8089FF1F1D
:1039E000ABAAAA2A769EFF1FC79EFF1FC39EFF1F7A
:1039F0005889FF1FA84B1B78FBB1A84B1B88012BD4
:103A000000F0D486022B00F0CF87032B01F04A810F
:103A1000042B01F0E481052B01F01B84062B01F03F
:103A2000DA84072B01F01F86082B01F0DD86092BB5
:103A300001F0C9870A2B01F0A687019B1B88002B88
:103A400000F0EC82964B1B78002B40F0E282954B05
:103A5000954A198834680020012310602B602EE5F8
:103A60000130C0B2022886BF0021117010701946C3
:103A7000FFF7ECBB0398002101708C4909780029FD
:103A80003FF436A8844902910978002900F0B287F2
:103A9000029800210170FFF72BB8039B1B78002BC5
:103AA0007FF485AB029B1B78002B7FF480AB019BDE
:103AB0001988FFF782BB7E4A1278002A3FF4F4AEE1
:103AC0007C4F387802F082FD7B4B1B78002B00F096
:103AD000BB8439887E2900F2B784784CDFF80C92D9
:103AE0002368D9F800209B1A0F2B40F29680744B64
:103AF00001311B8889B239802BB1052B03D0C9B2A3
:103B0000052005F051FA6F4F226898F80030C9F887
:103B100000203B70FEF781BE243B002BB8F800006C
:103B200040F3788498423EF464AF9BB26648A8F8AC
:103B3000003001230370FEF75CBFDFF89081C0B254
:103B400098F8001005F058FAFFF74BBB5F4B387838
:103B5000197805F051FA8DE47F21402005F024FA10
:103B60005B495C4A3B680B600021117007E5C0B2FD
:103B700098F8001005F040FAFFF72FB9D8B298F87E
:103B8000001005F039FA3B686BE5534BDFF860E154
:103B90001978FEF72EBF4B2C40F34C821834802C42
:103BA000B8F800304D4AA8BF8024A3427FF4DDADB1
:103BB000FEF747BF99F8000005F046FA2188FFF7A5
:103BC000FCBAFCF75FFD9DE4029B1B78002B7FF4A1
:103BD000C9AA039B1B78002B7FF4E9AA67E7FCF7CF
:103BE00051FD1CE63E4B01931B88002B7FF4F6AD84
:103BF000294B0293FFE5FCF745FDD6E4FCF742FDB7
:103C0000FFF7D3B90132D2B2022A40F25E8200221B
:103C100002701946FFF71ABB284C2A4F98F800305B
:103C20003B70FEF7FABD7F20FFF76CBA7F20FFF7ED
:103C300098B9194F1A4902974FF0000C81F800C04B
:103C4000009F02994FF0010E87F800E081F800C054
:103C50003DE6244F387802F0B9FC174B1B78002B57
:103C600000F03A8239887E2900F23682134CDFF860
:103C70007C902368D9F800209B1A0F2BCDD91A4BC2
:103C80000131188889B23980002800F04182C9B218
:103C9000C0B205F089F936E7DA9CFF1FF69DFF1FD9
:103CA000389EFF1FD89CFF1F109CFF1F2E9CFF1FDC
:103CB000769EFF1F789EFF1FC89EFF1F009EFF1F5E
:103CC000DE9CFF1F2A9CFF1F2F9CFF1FB99CFF1F1C
:103CD000309CFF1F8089FF1FA39EFF1F049EFF1FB4
:103CE0006C9CFF1F609CFF1FA89CFF1FB09EFF1FC6
:103CF000859CFF1FDFF8B4A399F80000BAF80030E4
:103D0000E34AE44CC31A82FB031ED917C1EB6E01D0
:103D100001EB4101A3EB810303EB430354F8233090
:103D200018447F2840F3AE847F3882FB0032C317EB
:103D3000C3EB620303EB4303A0EB83007330DFF8B4
:103D400070B3C0B205F080F9BBF80030022B7FF6EB
:103D500029AA99F80010BAF80030CD4ACB1A82FB94
:103D6000030ED817C0EB6E0000EB4000A3EB8003FE
:103D700003EB430304EB8303586808447F2840F3B4
:103D800020877F3882FB0032C317C3EB620202EB4D
:103D90004202A0EB82007330C0B205F055F9BBF8C7
:103DA0000030032B7FF6FEA999F80010BAF8003016
:103DB000B74ACB1A82FB030ED817C0EB6E0000EB9C
:103DC0004000A3EB800303EB430304EB8304A068F0
:103DD00008447F2840F370817F3882FB0032C3178C
:103DE000C3EB620202EB4202A0EB82007330C0B26E
:103DF00005F02AF9FFF7D6B9DFF8B0A23868BAF8AB
:103E00000030A34AA34CC31A82FB031ED917C1EB8F
:103E10006E0101EB4101A3EB810303EB430354F873
:103E2000233018447F2840F329847F3882FB0032F6
:103E3000C317C3EB620303EB4303A0EB83007330B0
:103E4000DFF87082DFF868B298F80010C0B205F0B1
:103E5000D3F8BBF80030022B7FF607AB3968BAF80D
:103E600000308B4ACB1A82FB030ED817C0EB6E00D2
:103E700000EB4000A3EB800303EB430304EB83035D
:103E8000586808447F2840F398867F3882FB0032C8
:103E9000C317C3EB620202EB4202A0EB8200733055
:103EA000C0B298F8001005F0A7F8BBF80030032B5B
:103EB0007FF6DBAA3968BAF80030754ACB1A82FB64
:103EC000030ED817C0EB6E0000EB4000A3EB80039D
:103ED00003EB430304EB8304A06808447F2840F30A
:103EE000F8807F3882FB0032C317C3EB620202EB1B
:103EF0004202A0EB8200733098F80010C0B205F0C7
:103F00007BF8FFF7B2BADFF8A4A16149BAF8002044
:103F1000604C9A1A81FB020ED017C0EB6E0000EBCA
:103F20004000A2EB800202EB420254F82200184447
:103F30007F2840F32284A0F17F0381FB0321DA175D
:103F4000C2EB610000EB4000A3EB80007330DFF8B0
:103F500060B198F80010C0B205F04EF8BBF8003020
:103F6000022B50D93968BAF80030494ACB1A82FB83
:103F7000030ED817C0EB6E0000EB4000A3EB8003EC
:103F800003EB430304EB8303586808447F2840F3A2
:103F900085867F3882FB0032C317C3EB620202EBD7
:103FA0004202A0EB82007330C0B298F8001005F016
:103FB00023F8BBF80030032B25D93868BAF8003055
:103FC000334AC31A82FB031ED917C1EB6E0101EB02
:103FD0004101A3EB810303EB430304EB8304A368D8
:103FE00018447F286EDD7F3882FB0032C317C3EB95
:103FF000620202EB4202A0EB82007330C0B298F87A
:10400000001004F0F9FF3B68FFF726BB0120FFF723
:1040100079B80021402004F0C7FF18E599F80000A6
:1040200005F012F80EE505F00FF8FEF7C7BF012006
:10403000FEF797BF243C002CB8F8003040F3C5854C
:10404000A3423EF4FEACA4B2134BA8F800400122F8
:104050001A70FEF7F6BC114B01931B88002B7FF4FE
:10406000BFABFFF77CB80E498342A8BF03460B6085
:10407000FEF795BE1446FFF76DBB0A4B0A4C198834
:104080006A2005F015F998F800303B70FEF7C5BBC3
:10409000ABAAAA2AE41B01002F9CFF1F6C9CFF1FE8
:1040A000109CFF1F609CFF1F009EFF1F349EFF1F80
:1040B000429CFF1FB99CFF1FFCF7E4FA97E6FCF750
:1040C000E1FA3DE4FCF7DEFA98E702701946FFF7E3
:1040D000BDB8FCF7D7FA0FE7D14B1B78002B3FF4A4
:1040E0009BAD3B88CF4F002B3FF496ADCE4CDFF815
:1040F00048932268D9F80010521A0F2A7FF68DAD26
:10410000CA4A013B108899B2398000287FF4BFADBC
:10411000C8B204F0BDFFF6E4DFF820A33868BAF8AF
:104120000030C34AC34CC31A82FB031ED917C1EB2C
:104130006E0101EB4101A3EB810303EB430354F850
:10414000233018447F2840F325847F3882FB0032D7
:10415000C317C3EB620303EB4303A0EB830073308D
:10416000DFF8DC82DFF8DCB298F80010C0B204F0AF
:1041700043FFBBF80030022B7FF677A93968BAF805
:104180000030AB4ACB1A82FB030ED817C0EB6E008F
:1041900000EB4000A3EB800303EB430304EB83033A
:1041A000586808447F2840F30E867F3882FB00322F
:1041B000C317C3EB620303EB4303A0EB830073302D
:1041C000C0B298F8001004F017FFBBF80030032BC2
:1041D0007FF64BA93868BAF80030954AC31A82FBBB
:1041E000031ED917C1EB6E0101EB4101A3EB810363
:1041F00003EB430304EB8304A36818447F287FF791
:1042000068AF7F3882FB0032C317C3EB620303EB56
:104210004303A0EB830073306EE6DFF820A299F829
:104220000000BAF80030824A824CC31A82FB031E97
:10423000D917C1EB6E0101EB4101A3EB810303EB45
:10424000430354F8233018447F2840F3A7837F3872
:1042500082FB0032C317C3EB620303EB4303A0EB03
:1042600083007330DFF8DCB1C0B204F0EDFEBBF8C0
:104270000030022B7EF696AF99F80010BAF80030A5
:104280006B4ACB1A82FB030ED817C0EB6E0000EB13
:104290004000A3EB800303EB430304EB8303586864
:1042A00008447F2840F393857F3882FB0032C31790
:1042B000C3EB620303EB4303A0EB83007330C0B294
:1042C00004F0C2FEBBF80030032B7EF66BAF99F80A
:1042D0000010BAF80030564ACB1A82FB030ED817EA
:1042E000C0EB6E0000EB4000A3EB800303EB430345
:1042F00004EB8304A06808447F287FF7DDAE7F3895
:1043000082FB0032C317C3EB620303EB4303A0EB52
:10431000830073306BE5DFF824A14549BAF800202B
:10432000444C9A1A81FB020ED017C0EB6E0000EBD2
:104330004000A2EB800202EB420254F82200184433
:104340007F2840F32E83A0F17F0381FB0321DA173E
:10435000C2EB610000EB4000A3EB80007330DFF89C
:10436000E4B098F80010C0B204F046FEBBF800308C
:10437000022B7FF648AE3968BAF800302C4ACB1AC7
:1043800082FB030ED817C0EB6E0000EB4000A3EBDE
:10439000800303EB430304EB8303586808447F283E
:1043A00040F319857F3882FB0032C317C3EB6203E9
:1043B00003EB4303A0EB83007330C0B298F8001006
:1043C00004F01AFEBBF80030032B7FF61CAE3868F1
:1043D000BAF80030164AC31A82FB031ED917C1EB84
:1043E0006E0101EB4101A3EB810303EB430304EBFB
:1043F0008304A36818447F287FF764AE7F3882FB6C
:104400000032C317C3EB620303EB4303A0EB83004B
:104410007330F3E501283EF4ECAA0123FFF786BBD5
:10442000C79EFF1F609CFF1F009EFF1FA89CFF1FD1
:10443000ABAAAA2AC01E0100B09EFF1F349EFF1F18
:10444000B99CFF1F429CFF1FCE4B1B78002B3FF4F3
:10445000E3AB3B88CC48002B3FF4DEABCB4CDFF822
:104460003C932268D9F80010521A0F2A7FF6D5AB78
:10447000C74A013B128899B20180002A3FF443AB3E
:10448000052A7FF43CABFFF73EBB4FF47A43013B78
:10449000FDD199F8000004F0D7FDFEF7F6BFDFF874
:1044A00000A399F80000BAF80030BA4ABA4CC31A0F
:1044B00082FB031ED917C1EB6E0101EB4101A3EB97
:1044C000810303EB430354F8233018447F2840F35F
:1044D000E8817F3882FB0032C317C3EB620202EB34
:1044E0004202A0EB82007330DFF8B8B2C0B204F031
:1044F000ABFDBBF80030022B7EF654AE99F80000FD
:10450000BAF80030A34AC31A82FB0321DA17C2EBC0
:10451000610202EB4202A3EB820303EB430304EBD1
:1045200083035B6818447F2840F31F847F380C2284
:1045300090FBF2F302FB13007330C0B204F084FD71
:10454000BBF80030032B7EF62DAE99F80000BAF8C8
:104550000030904AC31A82FB0321DA17C2EB6102D2
:1045600002EB4202A3EB820303EB430304EB83045D
:10457000A36818447F287FF79FAD7F380C2290FBFB
:10458000F2F302FB1300733031E4DFF814A2386851
:10459000BAF800307F4A804CC31A82FB031ED91739
:1045A000C1EB6E0101EB4101A3EB810303EB43037C
:1045B00054F8233018447F2840F370817F3882FB01
:1045C0000032C317C3EB620202EB4202A0EB82008F
:1045D0007330DFF8D481DFF8CCB198F80010C0B2A6
:1045E00004F00AFDBBF80030022B7EF63EAF3868BF
:1045F000BAF80030674AC31A82FB0321DA17C2EB0C
:10460000610202EB4202A3EB820303EB430304EBE0
:1046100083035B6818447F2840F3AB837F380C2208
:1046200090FBF2F302FB13007330C0B298F8001055
:1046300004F0E2FCBBF80030032B7EF616AF3868BE
:10464000BAF80030534AC31A82FB0321DA17C2EBCF
:10465000610202EB4202A3EB820303EB430304EB90
:104660008304A36818447F287FF733AD7F380C227A
:1046700090FBF2F302FB130073303DE4FCF702F809
:10468000FFF7DEBBFBF7FEFFFFF759BBDFF810A11A
:104690004049BAF80020404C9A1A81FB020ED0170C
:1046A000C0EB6E0000EB4000A2EB800202EB420286
:1046B00054F8220018447F2840F3F680A0F17F03CD
:1046C00081FB0321DA17C2EB610101EB4101A3EB8E
:1046D00081007330DFF8CCB098F80010C0B204F05D
:1046E0008BFCBBF80030022B7FF68DAC3868BAF833
:1046F0000030284AC31A82FB0321DA17C2EB610299
:1047000002EB4202A3EB820303EB430304EB8303BC
:104710005B6818447F2840F338837F380C2290FB75
:10472000F2F302FB13007330C0B298F8001004F0EB
:1047300063FCBBF80030032B7FF665AC3868BAF831
:104740000030144AC31A82FB0321DA17C2EB61025C
:1047500002EB4202A3EB820303EB430304EB83046B
:10476000A36818447F287FF7ADAC7F380C2290FBFC
:10477000F2F302FB1300733040E4FBF783FFFFF713
:10478000E6BB00BFC79EFF1F789EFF1F009EFF1F56
:10479000DE9CFF1FABAAAA2A501F0100B09EFF1F7C
:1047A000349EFF1F429CFF1FB99CFF1FDFF838A3F8
:1047B00099F80000BAF80030C34AC44CC31A82FB0F
:1047C0000317D917C1EB670101EB4101A3EB81038B
:1047D00003EB430354F8233018447F286ADD7F3805
:1047E00082FB0032C317C3EB620202EB4202A0EB72
:1047F00082007330DFF8F4B2C0B204F025FCBBF8DD
:104800000030022B7FF619A999F80000BAF80030A1
:10481000AD4AC31A82FB0321DA17C2EB610202EB35
:104820004202A3EB820303EB430304EB83035B68C5
:1048300018447F2840F3AC827F380C2290FBF2F3BF
:1048400002FB13007330C0B204F0FEFBBBF8003073
:10485000032B7FF6F2A899F80000BAF800309A4AC4
:10486000C31A82FB0321DA17C2EB610202EB420298
:10487000A3EB820303EB430304EB8304A368184414
:104880007F2814DD7F380C2290FBF2F302FB13002B
:104890007330C0B204F0D8FBFFF7CFB8FBF7F2FEDD
:1048A00097E6FBF7EFFE1FE6FBF7ECFE12E7FBF7E0
:1048B000E9FEEEE7FBF7E6FE9CE7DFF82CA299F8AD
:1048C0000000BAF80030804A814CC31A82FB031EF4
:1048D000D917C1EB6E0101EB4101A3EB810303EB9F
:1048E000430354F8233018447F28DADD7F3882FBF5
:1048F0000032C317C3EB620303EB4303A0EB830057
:104900007330F1E5DFF8E0A13868BAF800306E4A9C
:104910006F4CC31A82FB031ED917C1EB6E0101EB6A
:104920004101A3EB810303EB430354F82330184404
:104930007F28B3DD7F3882FB0032C317C3EB6203ED
:1049400003EB4303A0EB8300733042E6DFF898A14A
:104950005D49BAF800205E4C9A1A81FB020ED0170E
:10496000C0EB6E0000EB4000A2EB800202EB4202C3
:1049700054F8220018447F2896DDA0F17F0381FBC4
:104980000321DA17C2EB610000EB4000A3EB8000CB
:1049900073309FE6FBF776FEFFF7E2BBFBF772FE94
:1049A00060E4FBF76FFEDAE4DFF83CA199F8000061
:1049B000BAF80030444A474CC31A82FB0317D91790
:1049C000C1EB670101EB4101A3EB810303EB43035F
:1049D00054F8233018447F287FF76CAF7F3882FB70
:1049E0000032C317C3EB620303EB4303A0EB830066
:1049F0007330FFE638480090384839490390FEF795
:104A00006EB8DFF8E4A099F80000BAF800302E4A3A
:104A1000344CC31A82FB0321DA17C2EB610202EBAA
:104A20004202A3EB820303EB430354F82330184400
:104A30007F2840F3A7817F380C2290FBF2F302FB22
:104A400013007330DFF8A4B0C0B204F0FDFABBF875
:104A50000030022B19D999F80000BAF800300C2266
:104A6000C11A91FBF2F302FB131302FB03435B68D1
:104A700018447F2840F385847F3890FBF2F302FBD3
:104A800013007330C0B204F0DFFABBF80030032B20
:104A90007EF688ABBAF8003099F800000C22C11AF3
:104AA00091FBF2F302FB131302FB0344A3681844C7
:104AB0007F287FF701AB7F3890FBF2F302FB1300F6
:104AC0007330FFF794B900BFABAAAA2AE41B010018
:104AD000D4200100C01E0100849EFF1F0D9CFF1FFB
:104AE000389EFF1F801D0100349EFF1F429CFF1F48
:104AF000DFF864A33868BAF80030CE4ACE4CC31A47
:104B000082FB0321DA17C2EB610202EB4202A3EB44
:104B1000820303EB430354F8233018447F2840F307
:104B20002E817F380C2290FBF2F302FB13007330CE
:104B3000DFF82883DFF828B398F80010C0B204F03B
:104B40005BFABBF80030022B1AD93868BAF800308B
:104B50000C22C11A91FBF2F302FB131302FB034375
:104B60005B6818447F2840F3C3837F3890FBF2F3DF
:104B700002FB13007330C0B298F8001004F03CFA46
:104B8000BBF80030032B7EF670ACBAF80030386802
:104B90000C22C11A91FBF2F302FB131302FB034434
:104BA000A36818447F287FF794AA7F3890FBF2F31C
:104BB00002FB13007330FFF79FB9FBF763FDFFF7AC
:104BC0006FB9FBF75FFDFFF7E7B8012B3DF439AF95
:104BD0000124FFF739BADFF880A29649BAF800201D
:104BE000954C9A1A81FB0210D117C1EB600101EBC1
:104BF0004101A2EB810202EB420254F82200184468
:104C00007F2840F3B980A0F17F030C2093FBF0F2E2
:104C100000FB12307330DFF848B298F80010C0B2D1
:104C200004F0EAF9BBF80030022B1AD93868BAF858
:104C300000300C22C11A91FBF2F302FB131302FBAA
:104C400003435B6818447F2840F34F837F3890FB11
:104C5000F2F302FB13007330C0B298F8001004F0B6
:104C6000CBF9BBF80030032B7FF6CDA9BAF80030A2
:104C700038680C22C11A91FBF2F302FB131302FBFA
:104C80000344A36818447F287FF71CAA7F3890FB51
:104C9000F2F302FB13007330FFF7B0B9FBF7F2FC3D
:104CA000FFF782B9DFF8B0A199F80000BAF8003038
:104CB000604A624CC31A82FB0321DA17C2EB61021D
:104CC00002EB4202A3EB820303EB430354F82330CD
:104CD00018447F2846DD7F380C2290FBF2F302FB5C
:104CE00013007330DFF878B1C0B204F0ADF9BBF84F
:104CF0000030022B19D999F80000BAF800300C22C4
:104D0000C11A91FBF2F302FB131302FB03435B682E
:104D100018447F2840F38B807F3890FBF2F302FB2E
:104D200013007330C0B204F08FF9BBF80030032BCE
:104D30007EF683AEBAF8003099F800000C22C11A52
:104D400091FBF2F302FB131302FB0344A368184424
:104D50007F287FF7ACAD7F3890FBF2F302FB1300A6
:104D6000733096E5FBF78EFCBCE7FBF78BFCFFF797
:104D7000E4BBFBF787FC58E4FBF784FC4BE7FBF74D
:104D800081FCD5E6FBF77EFC5CE6FBF77BFCCBE425
:104D9000FBF778FC57E5DFF8C0A03868BAF80030B8
:104DA000244A274CABE6DFF8B0A099F80000BAF827
:104DB0000030204A224C2CE6029B1B78002B7EF40C
:104DC000D1A9FEF7F4B9FBF75DFCFFF7F9B9FBF7E2
:104DD00059FCFFF774BAFBF755FCFFF7EEBADFF8A2
:104DE00078A099F80000BAF80030124A154C61E733
:104DF000DFF864A00F49BAF80020114CF1E6124B1D
:104E00001B78002B00F0C182104B1B78002B7DF427
:104E100018AE0F4B1B78002B3DF413AEB8F80030E2
:104E20000C490A33A8F800300A70FDF70ABEFBF7F8
:104E300029FC77E7ABAAAA2A801D0100501F0100B8
:104E400044200100D4200100EB9DFF1FC59EFF1FE1
:104E5000C69EFF1F2F9CFF1F349EFF1FB99CFF1F84
:104E6000429CFF1FA44C2388002B40F0BE83DFF838
:104E7000A0B2A249A24A0988D7F80080B2F800E09F
:104E8000A048C1EB080C0C229CFBF2F102FB11C103
:104E90004FF0900C0CFB0EFE02FB01E16FF00B0ECD
:104EA000405880440EFB03807F2840F30285A0F128
:104EB0007F0393FBF2F002FB10307330924BC0B2D1
:104EC000197804F099F8BBF8002023881344022BCA
:104ED00023DD8A4A8A4B11883868B3F800C0DFF8AE
:104EE00024E2411A0C2291FBF2F302FB13119023EE
:104EF00003FB0CF302FB013373445B6818447F2807
:104F000040F3AD857F3890FBF2F302FB1300733062
:104F10007D4BC0B2197804F06FF8BBF800202388ED
:104F20001344032B23DD754A754B11883868B3F899
:104F300000C0DFF8D0E1411A0C2291FBF2F302FB32
:104F40001311902303FB0CF302FB013373449B68A2
:104F500018447F2840F35D857F3890FBF2F302FB15
:104F600013007330684BC0B2197804F045F8BBF8F1
:104F7000002023881344042B7EF777AA634B1B88F9
:104F8000012B7EF472AA3A68A2F10C007F2840F34C
:104F90008F828B3A0C2092FBF0F300FB13207330CE
:104FA000594BC0B2197804F027F8FEF75EBA524C9C
:104FB0002288002A00F0D7825449DFF854B10988CA
:104FC000BBF800000331884227DD4C484C4900887B
:104FD000B1F800E0DFF82CC1181A0C2190FBF1F9B0
:104FE00001FB19004FF0900909FB0EFE01FB00E0E8
:104FF0006FF00B0E5CF8000003440EFB02307F28BC
:1050000040F3B7847F3890FBF1F301FB130073305A
:10501000C0B298F8001003F0EFFFBBF8002023881F
:105020001344022B23DD354B354A38681B88B2F810
:1050300000C0DFF8D0E0C31A0C2193FBF1F201FBB2
:105040001232902303FB0CF301FB023373445B68C1
:1050500018447F2840F3E4847F3890FBF1F301FB90
:1050600013007330C0B298F8001003F0C5FFBBF80E
:10507000002023881344032B23DD204B204A38686B
:105080001B88B2F800C0DFF87CE0C31A0C2193FB48
:10509000F1F201FB1232902303FB0CF301FB02330C
:1050A00073449B6818447F2840F3C1847F3890FB89
:1050B000F1F301FB13007330C0B298F8001003F055
:1050C0009BFFBBF8002023881344042B7EF79BAF83
:1050D0000E4B1B88012B7EF496AF3A68A2F10C00B0
:1050E0007F287EF7EFAF8B3A0C2092FBF0F300FBAA
:1050F00013207330FEF782BFBC9CFF1F349EFF1F3E
:10510000DE9DFF1FE0180100B99CFF1F5E9CFF1F82
:10511000429CFF1FCE4C2388002B40F02782DFF8F3
:1051200064B3CC49CC4A098899F80000B2F800E091
:10513000DFF85483C1EB000C0C229CFBF2F102FB64
:1051400011C14FF0900C0CFB0EFE02FB01E16FF061
:105150000B0E58F8011008440EFB03007F2840F3A3
:105160000484A0F17F0393FBF2F002FB1030733054
:10517000C0B203F069FFBBF8002023881344022B60
:1051800022DDB44AB44B118899F80000B3F800C08E
:10519000DFF8F4E2411A0C2291FBF2F302FB131147
:1051A000902303FB0CF302FB013373445B68184448
:1051B0007F2840F3E5837F3890FBF2F302FB130076
:1051C0007330C0B203F040FFBBF8002023881344C3
:1051D000032B22DD9F4AA04B118899F80000B3F8F9
:1051E00000C0DFF8A4E2411A0C2291FBF2F302FBAB
:1051F0001311902303FB0CF302FB013373449B68F0
:1052000018447F2840F302847F3890FBF2F302FBBE
:1052100013007330C0B203F017FFBBF800202388DF
:105220001344042B7DF7BEAF8C4B1B88012B7DF400
:10523000B9AF99F80020A2F10C007F287EF73CAFAF
:105240008B3A0C2092FBF0F300FB13207330FEF737
:10525000CEBDDFF800A299F80000BAF80030804C0B
:10526000C11A0C2291FBF2F302FB131302FB03F3AE
:10527000E35818447F287FF775AD7F3890FBF2F331
:1052800002FB130073302DE5764B1B88182B12D0D0
:1052900099F800201344A3F118007F2840F3DC8321
:1052A0000C20973B93FBF0F200FB123303F17300E9
:1052B000C0B203F0C9FE6C4A6C4B127833F812305E
:1052C000182B3DF46FAF99F800201344A3F1180098
:1052D0007F287EF7F1AE0C20973B93FBF0F200FBAA
:1052E000123303F17300FEF782BDFBF7CBF9B3E491
:1052F000FBF7C8F93FE45B4B1A88182A13D03B68C8
:105300001344A3F118007F2840F37D830C20973BC2
:1053100093FBF0F200FB123303F17300544BC0B265
:10532000197803F069FE504B50491A78022A94BF4D
:10533000013200221A701A7831F81200182810D1A0
:105340000424022A02F10100C2B288BF002231F80F
:105350001200182804D1013CF3D11A70FEF785B869
:105360001A703B680344A3F118007F2840F3A08023
:105370000C20973B93FBF0F200FB123303F1730018
:105380000EE6FBF77FF9FFF77DBB3A4B1B78002B4E
:105390007DF485AF384B1B78002B3DF452ABB8F849
:1053A000003036490133A8F800300A70FDF749BBD8
:1053B000304B1B78002B7DF444AB2F4B1B78002B1C
:1053C0003DF43FABB8F800302C49013BA8F8003061
:1053D0000A70FDF736BBDFF87CA099F80000BAF838
:1053E0000030274C3CE71F4A1288182A12D0134479
:1053F000A3F118007F2840F3C0820C20973B93FB59
:10540000F0F200FB123303F17300C0B298F8001001
:1054100003F0F2FD144B15491A78022A94BF0132A9
:1054200000221A701A7831F8120018282FD104249B
:10543000022A02F10100C2B288BF002231F8120034
:10544000182823D1013CF3D11A703B68FEF704B948
:10545000BC9CFF1F349EFF1FDE9DFF1F5E9CFF1F35
:10546000801D01004E9CFF1FBA9CFF1F509EFF1F16
:10547000B99CFF1FC59EFF1FC69EFF1F2F9CFF1FCD
:1054800044200100429CFF1FE01801001A703B6895
:105490000344A3F118007F287EF714AE0C20973B3D
:1054A00093FBF0F200FB123303F17300FEF7A6BD8D
:1054B000FBF7E8F874E5BF4B1B88182B12D099F85E
:1054C00000201344A3F118007F2840F3AD820C2084
:1054D000973B93FBF0F200FB123303F17300C0B271
:1054E00003F0B2FDB44AB54B127833F81230182BE2
:1054F0007FF4E9AEFDF756BEAE4B1A88182A13D0DA
:105500003B681344A3F118007F2840F386820C20E7
:10551000973B93FBF0F200FB123303F17300A84BAF
:10552000C0B2197803F068FDA34BA4491A78022A87
:1055300094BF013200221A701A7831F8120018282C
:105540007FF40FAF0424022A02F1010294BFD2B209
:10555000002231F8120018287FF402AF013CF2D18A
:105560001A70FDF782BFDFF87CB22EE5954ADFF8AE
:1055700074B21288BBF80010033291427FF7FBAD82
:10558000CFE58C4A1288182A12D01344A3F11800D0
:105590007F2840F35E820C20973B93FBF0F200FBE8
:1055A000123303F17300C0B298F8001003F024FD29
:1055B000814B82491A78022A94BF013200221A7064
:1055C0001A7831F8120018287FF461AF0424022AF7
:1055D00002F1010294BFD2B2002231F81200182861
:1055E0007FF454AF013CF2D12EE7764ADFF8F4B1F4
:1055F0001288BBF80010033291427FF764AC38E4A4
:10560000714B01227F2107201A8003F0CDFC7F21FE
:105610000B2003F0C9FCFDF76DBE6C4B04227F210B
:1056200007201A8003F0C0FC00210B2003F0BCFC13
:10563000FDF759BE654B02227F2107201A8003F037
:10564000B3FC7F210B2003F0AFFCFDF747BE5F4B9F
:10565000002107201C8003F0A7FC7F210B2003F012
:10566000A3FCFDF736BE5A4C2388002B40F0E681A0
:10567000DFF870B1574999F80000574A0988178830
:10568000DFF858E1411A0C2291FBF2FC02FB1C11DD
:105690004FF0900C0CFB07F702FB01716FF00B074A
:1056A0005EF80110014407FB03107F2840F3C3811B
:1056B0007F3890FBF2F302FB13007330C0B203F0AB
:1056C000C3FCBBF8002023881344022B21DD414B8F
:1056D000414A99F800001B88B2F800E03F4FC31A16
:1056E0000C2193FBF1F201FB1232902303FB0EF32A
:1056F00001FB02333B445B6818447F2840F3C881B8
:105700007F3890FBF1F301FB13007330C0B203F05C
:105710009BFCBBF8002023881344032B21DD2D4B79
:105720002D4A99F800001B88B2F800E02B4FC31AED
:105730000C2193FBF1F201FB1232902303FB0EF3D9
:1057400001FB02333B449B6818447F2840F39D8152
:105750007F3890FBF1F301FB13007330C0B203F00C
:1057600073FCBBF8002023881344042B7EF765A943
:10577000144B1B88012B7EF460A999F80020A2F13C
:105780000C007F287FF793A88B3A0C2092FBF0F354
:1057900000FB13207330FFF77CB8114B00227F21F0
:1057A00007201A8003F000FC7F210B2003F0FCFB94
:1057B000FDF7A8BD569CFF1FBA9CFF1FC09DFF1F91
:1057C000B99CFF1F5E9CFF1FCA9CFF1F2C9EFF1FE2
:1057D000BC9CFF1F349EFF1FDE9DFF1FE0180100D1
:1057E0002C9CFF1F429CFF1FB04B1B88182B12D014
:1057F00099F800201344A3F118007F2840F33C815E
:105800000C20973B93FBF0F200FB123303F1730083
:10581000C0B203F019FCA64AA64B127833F8123036
:10582000182B3EF40AA999F800201344A3F118009C
:105830007F287FF73CA80C20973B93FBF0F200FBFE
:10584000123303F17300FFF724B89B4A1288182A19
:1058500012D01344A3F118007F2840F307810C20D5
:10586000973B93FBF0F200FB123303F17300C0B2DD
:1058700098F8001003F0C0FB8D4B90491A78022A6B
:1058800094BF013200221A701A7831F812001828D9
:105890007FF4FDAD0424022A02F1010294BFD2B2CA
:1058A000002231F8120018287FF4F0AD013CF2D14B
:1058B000CAE5FAF7E7FEFFF701BB7F4B1A88182A03
:1058C00013D03B681344A3F118007F2840F3DA801B
:1058D0000C20973B93FBF0F200FB123303F17300B3
:1058E000774BC0B2197803F087FB714B73491A7874
:1058F000022A94BF013200221A701A7831F812007D
:1059000018287FF42EAD0424022A02F1010294BF6C
:10591000D2B2002231F8120018287FF421AD013CE8
:10592000F2D11A70FDF7A1BD634B1B88182B12D062
:1059300099F800201344A3F118007F2840F39380C6
:105940000C20973B93FBF0F200FB123303F1730042
:10595000C0B203F079FB564A584B127833F8123034
:10596000182B7FF4B0ACFDF71DBCFAF78BFEFFF7E8
:10597000FFBBFAF787FEFFF74BBBFAF783FE44E560
:10598000FAF780FE1DE44C4B1B88182B11D099F8B8
:1059900000201344A3F118007F286ADD0C20973BF8
:1059A00093FBF0F200FB123303F17300C0B203F07B
:1059B0004BFB3F4A414B127833F81230182B7FF4DF
:1059C00032AFFEF73AB83F4B1B88182B11D099F82D
:1059D00000201344A3F118007F2850DD0C20973BD2
:1059E00093FBF0F200FB123303F17300C0B203F03B
:1059F0002BFB2F4A344B127833F81230182B7FF4DC
:105A000012AFFEF71AB8FAF73DFE87E4FAF73AFE4E
:105A100000E4FAF737FEFFF7A5BAFAF733FE7EE5A2
:105A2000FAF730FEFFF71EBBFAF72CFE57E5FAF740
:105A300029FEFFF741BBFAF725FE3FE6234ADFF8D0
:105A400098B01288BBF80010033291427FF739AE4C
:105A500010E6FAF717FEA6E5FAF714FE28E4FAF7BF
:105A600011FEFFF755BAFAF70DFE71E7FAF70AFED5
:105A7000FDE6FAF707FE99E7FAF704FEC8E6FAF73B
:105A800001FEB3E7FAF7FEFD2AE7FAF7FBFD65E64C
:105A9000FAF7F8FD3AE60E4B03930E4B0293FDF72F
:105AA0009FBE23601946FDF7D1BB00BF4E9CFF1F70
:105AB000BA9CFF1F509EFF1F589CFF1FC89DFF1FD1
:105AC000B99CFF1F569CFF1FC09DFF1F5E9CFF1FC0
:105AD0000D9CFF1FDA9CFF1F429CFF1F38B507F08B
:105AE000C9F90E4805F000F90D4805F0FDF80D481C
:105AF00005F0FAF800234FF07E5201210A48FAF728
:105B0000B5FC0A4B0A4A0B49802400251C71184633
:105B10001D60BDE838400AF071BE00BF409CFF1F09
:105B2000749CFF1FD09CFF1F089EFF1F8C9EFF1FB1
:105B30001C89FF1F2906000010B50446A4206368D5
:105B4000198803F0B5FBE368A6201988BDE810406A
:105B500003F0AEBB43682A20198803F0A9BB00BF3D
:105B600010B5044622206368198803F0A1FBE3689E
:105B700024201988BDE8104003F09ABB10B50446F4
:105B80000A206368198803F093FBE3680C201988E6
:105B9000BDE8104003F08CBB10B5044606206368D6
:105BA000198803F085FBE36808201988BDE81040D8
:105BB00003F07EBB10B5044602206368198803F029
:105BC00077FBE36804201988BDE8104003F070BB40
:105BD00070B50E4C84B012250422012306460390B2
:105BE000029320468DE824001423102106F080FA49
:105BF000062209230293039601952046009214235E
:105C0000102106F075FA04B070BD00BFF89EFF1FAA
:105C10002DE9F041224D82B0012602B284B20092F9
:105C2000284601967823192106F0A8F904F10C0200
:105C300012B28DE844002846A7197823192104F1EF
:105C4000020806F09BF93FB20FFA88F819233A468A
:105C5000284619460196CDF8008006F08FF9782382
:105C60003A4628461946CDF80080019604F10A0705
:105C70000B3406F083F93FB224B278233A46284623
:105C800019468DE8500006F079F9192300943A4638
:105C900001962846194606F071F902B0BDE8F08178
:105CA000F89EFF1F2DE9F0411E4682B01446002ADF
:105CB0006AD0099B4D4A00EBC305012C6F892989E5
:105CC0006868A7EB010382FB03E21A444FEAE3731F
:105CD000C3EBA21302887BD0042C38D112FA83F3D1
:105CE000994203DC9F423946A8BF1946089A0180B1
:105CF000B6F90030BDF920803D48971D4FF0000EE9
:105D00003FB2194642460097CDF804E006F036F956
:105D100029896A896B68521A1B885C2AA3EB0103E4
:105D200059DD03EB43030132C3EB431393FBF2F35F
:105D300003F11B0213B20120328019464246019042
:105D400000972B4806F01AF92A4B00221A702A4BAA
:105D5000022CB3F9001045D0082C31D100221A8052
:105D600091422DD0089AB6F900302148063201241C
:105D700012B2009219460194BDF9202006F0FEF8F7
:105D8000204602B0BDE8F0811C4D1D4A2B68126808
:105D9000CB1A93420F4617D9164A33881178144804
:105DA000012918BF01241470089A06321BB212B2DE
:105DB0008DE814001946BDF9202006F0DFF82F60A9
:105DC000012002B0BDE8F081204602B0BDE8F081BC
:105DD0009BB2D31A84E75C2101FB03F393FBF2F23D
:105DE0001B32A7E74A1C12B21A80B9E7C94216B2A1
:105DF000F89EFF1F719FFF1FD69EFF1F5C9FFF1F16
:105E00004431010030B583B000230C4605B2009345
:105E100026225B231C210C4805F000FE29460123A5
:105E20002622094805F00AF9002C24B205DB214698
:105E300001232622044805F001F9044A044B158089
:105E40001C8003B030BD00BFF89EFF1F628AFF1F99
:105E5000648AFF1F2DE9F041B44C237882B01BB156
:105E6000B34B4FF6FF721A80B24BB3F90030CBB987
:105E7000B14AAF4B1068B3F9002080F30C005B23EC
:105E800003FB00F000131C30824244D04FF0FF317E
:105E9000FFF7B8FFA94805F025FE0023237002B0E4
:105EA000BDE8F081012B1BD0022B53D0032B38D03F
:105EB000042B00F08C80052BEFD10F2007F082FE21
:105EC000C0F53B600830B0F5AF6F41DBB0F5FA6F5D
:105ED000A8BF4FF4FA60A0F5AF625B2398482EE0AC
:105EE000984B1A68B2F52F7F32DB41F25C23934264
:105EF000A8BF1346A3F52F735B22934802FB03F35D
:105F000080FB0320DB17C3EBA0201C30884BB3F9C8
:105F100000308342BAD18D4BB3F900300133B5D193
:105F2000BBE78B4B1B68B3F5FA7F11DBB3F57A6FD8
:105F3000A8BF4FF47A638748A3F5FA725B2303FB8B
:105F400002F380FB0320DB17C3EB20201C30DDE7CE
:105F50001C20DBE7804B1B68B3F5FA7F33DBB3F51E
:105F60007A6FA8BF4FF47A63A3F5FA7279485B237E
:105F700003FB02F380FB0320DB17C3EB20201C3064
:105F8000764B1B68B3F5FA7F1FDBB3F57A6FA8BFBA
:105F90004FF47A63A3F5FA726E495B2303FB02F3B5
:105FA00081FB0321DB17C3EB21211C31604BB3F9CB
:105FB000003083427FF46CAF644BB3F900308B4206
:105FC0007FF466AF69E71C20DAE71C21EEE72522A3
:105FD00000258DE8240076231C215848604E614F2F
:105FE000DFF8988105F0CAFF16E0B0F5AF7FA8BFD3
:105FF0004FF4AF70323802FB00F088FB0031C0175D
:10600000C0EB61111C3109B201231D4425224B480C
:1060100005F014F80C2D14D0E9B2534804F0CCFE6E
:1060200056F8043BC3F5967300FB03F087FB00139F
:10603000C017C0EB631031284FF05B02D5DC1C2188
:10604000E2E7262200258DE8240076231C213B4828
:10605000464E444FDFF8248105F090FF16E0B0F57E
:10606000AF7FA8BF4FF4AF70323802FB00F088FB5F
:106070000031C017C0EB61111C3109B201231D446E
:1060800026222E4804F0DAFF0C2D14D0E9B238484D
:1060900004F092FE56F8043BC3F5967300FB03F040
:1060A00087FB0013C017C0EB631031284FF05B0271
:1060B000D5DC1C21E2E7272200258DE82400762389
:1060C0001C211E482B4E274FDFF8B08005F056FFED
:1060D00017E0B0F5AF7FA8BF4FF4AF70323802FBC6
:1060E00000F088FB0031C017C0EB61111C3109B210
:1060F00001231D442722114804F0A0FF062D3FF480
:10610000C9AEE9B21C4804F057FE56F8043BC3F58B
:10611000967300FB03F087FB0013C017C0EB6310FE
:1061200031284FF05B02D4DC1C21E1E7CC9EFF1F3D
:10613000628AFF1FD29EFF1F449EFF1FF89EFF1F13
:1061400037800B6D1C9CFF1FD3058541648AFF1FA0
:10615000649CFF1F011FB812709CFF1FBC9EFF1F95
:10616000188AFF1FB5814E1B749CFF1F2889FF1FD3
:10617000D09CFF1F488AFF1F409CFF1F4B48371BC6
:106180002DE9F04FDFF8EC82B74CB8F900604D789C
:1061900054F8264087B08246039305B10D78DFF8A6
:1061A000FCB2002A34D19BF800308BBBAF4EB6F95D
:1061B0000000002800F0CE80012800F0248101209A
:1061C00032232A46019000935146A94B2046FFF7FF
:1061D00069FD00250746B6F90030022B40F3F48034
:1061E00000233380B8F90030A24A002BC0F2F880B7
:1061F000052BC4BF00231380039B002B40F0F680C7
:10620000002D0CBF38464FF0FF3007B0BDE8F08FCF
:10621000964EE368226898480493002705923780D9
:106220008BF8007005F052FB1120FFF7F1FC4FF0E6
:10623000010919232821CDF8049000912422194640
:106240008D4805F09BFE782328212422CDF8049068
:1062500000918948194605F091FE4946864806F0A6
:1062600023FA02221921844806F01AFADDF8149064
:1062700048460BF085F8494602467F4806F0AAFBDF
:106280007D4806F0BDFB394614227B4806F008FA2B
:1062900003227A49784806F09DFB774806F0B0FB68
:1062A00039462322744806F0FBF9032274497248E8
:1062B00006F090FB704806F0A3FB049B002B72D104
:1062C0000123704A18461370FFF782FC2089638906
:1062D0006768191A5C293A885BDC131A5C2202FB96
:1062E00003F292FBF1F31B33674A634813800127E3
:1062F0001BB21A2219468DE88400142205F03EFED6
:10630000049BDBB1218A638AE768581A5C283A88C3
:106310006FDD521A02EB4202C2EB4212431C92FBA7
:10632000F3F31B33524A54481380012738221BB21F
:106330008DE884001946322205F020FE534A544B62
:10634000B6F90000012111704FF6FF721A80002883
:106350007FF432AFDFF848914E4AD9F80030126826
:10636000C3EB0A0393424CD9464B1A78012A18BF53
:10637000012018700127FFF72BFCC9F800A0012DA0
:106380004ED0042D59D0022D60D0082D64D00025A8
:1063900021E7121A02EB4202C2EB42124B1C92FBA3
:1063A000F3F31B33A0E72F20FFF732FC39463222EC
:1063B000314806F075F9032237492F4806F00AFBE9
:1063C0002D4806F01DFB7BE77FF40CAFE368002B44
:1063D0003FF406AFB8F90030264A002BBFF608AFED
:1063E00005231380039B002B3FF40AAFFFF732FD18
:1063F00006E7511A5C2202FB01F292FBF0F31B3319
:1064000090E70746BBE7002714238DE888002A465B
:1064100051461D4B2046FFF745FC3D460746DAE650
:10642000B8F800308BF800500133A8F800306369E9
:1064300083B1002520469847CDE6B8F80030012208
:10644000013BA8F800308BF80020F0E701233380EF
:106450000025C7E61D46BEE66369002232804FF084
:10646000FF35002BE6D1BDE6688AFF1FD69EFF1FD1
:10647000D09EFF1FD29EFF1FF89EFF1F3C220100EF
:1064800040220100719FFF1FCE9EFF1FCC9EFF1F69
:10649000628AFF1F4431010044220100D49EFF1F85
:1064A0005C9FFF1F01210D2007F05EB900210D2028
:1064B00007F05AB901460D2007F056B908B50D206E
:1064C00007F058F9B0FA80F149090D20BDE80840FD
:1064D00007F04AB910B5002144080D2007F044F92F
:1064E000204607F07DF90D20012107F03DF92046F7
:1064F000BDE8104007F074B92D4A2E4B10881B6878
:10650000984210B549DA2C4A1288141A9A42A8BF48
:106510001A46B4F5157F36DA121A40F2532303FBFC
:1065200002F393FBF4F105310A2006F08DFF234BB3
:106530001978C9B3224B23491B6840F2271283F311
:10654000070302FB03F381FB03211944DB17C3EBB1
:10655000A1110531092006F077FF1B4B1968F1B135
:1065600081F3070140F22712164802FB01F380FB7A
:1065700003211944DB17C3EBA11105311620BDE837
:10658000104006F061BF131A4FF41572611C02FB34
:1065900003F393FBF1F10531C6E70021C4E71620B0
:1065A000BDE8104006F050BF092006F04DFFD4E7CB
:1065B000D89CFF1F109CFF1F9A9EFF1F929CFF1FDD
:1065C000149CFF1F09040281589EFF1F7F2838B5C5
:1065D000A8BF7F200F4C4FF4167202FB00F284FB21
:1065E00002311144D2170546C2EBA1110A2006F070
:1065F0002BFF7F3D4FF4967303FB05F384FB0321D0
:106600001944DB17A3EBA1110920BDE8384006F0BF
:106610001BBF00BF09040281C368B3F9003030B565
:1066200083EAE374A4EBE374002BA0B218DB01232C
:1066300000E0134603EB830252009442F9DA0A4D5C
:1066400090FBF3F285FB03E403FB1200DB1730320F
:10665000D3EBA40380B201F8012BF1D10B7030BD54
:106660002D230B700131E2E76766666638B5094D88
:106670008224204602F036FE35F8021B00B2884222
:10668000204601D002F014FE0234A4B28A2CF0D1CC
:1066900038BD00BFC89DFF1F024B8020198802F043
:1066A00007BE00BF589CFF1F38B5094D782420460F
:1066B00002F018FE35F8021B00B28842204601D0D5
:1066C00002F0F6FD0234A4B2802CF0D138BD00BF38
:1066D000C09DFF1F024B7620198802F0E9BD00BF64
:1066E000569CFF1F38B5094D4624204602F0FAFD9E
:1066F00035F8021B00B28842204601D002F0D8FDD6
:106700000234A4B24E2CF0D138BD00BF509EFF1F02
:10671000024B4420198802F0CBBD00BF4E9CFF1FE6
:10672000024B4E20198802F0C3BD00BF6C9CFF1FB6
:10673000024B9A20198802F0BBBD00BFBC9CFF1F12
:10674000024B9820198802F0B3BD00BF5E9CFF1F6A
:10675000024B8C20198802F0ABBD00BFDE9DFF1FED
:10676000024B9C20198802F0A3BD00BF429CFF1F72
:10677000024BA020198802F09BBD00BFC09EFF1FE6
:10678000024B9620198802F093BD00BF349EFF1F74
:10679000024B8A20198802F08BBD00BFF69DFF1FB7
:1067A00008B5034B1020198802F082FD012008BDB6
:1067B000F49DFF1F024B1020198802F079BD00BF25
:1067C000F49DFF1F024B2C20198802F071BD00BF01
:1067D0003E9CFF1F024B1E20198802F069BD00BFBE
:1067E0005C9CFF1FC3680E20198802F061BD00BFCA
:1067F000024B2820198802F05BBD00BF4C9EFF1F92
:10680000024B6420198802F053BD00BF489EFF1F51
:10681000024B5A20198802F04BBD00BF249CFF1F79
:10682000024B1620198802F043BD00BF2C9CFF1FAD
:10683000024B2E20198802F03BBD00BFC49CFF1FF5
:10684000024B3020198802F033BD00BFA49EFF1F09
:10685000024B9E20198802F02BBD00BFBC89FF1F90
:10686000024B1820198802F023BD00BFDE9CFF1FD9
:10687000024BA220198802F01BBD00BF789EFF1FAB
:10688000024B1A20198802F013BD00BF769CFF1F2F
:10689000024B1C20198802F00BBD00BF6E9CFF1F2D
:1068A000024B6620198802F003BD00BF829EFF1FC5
:1068B000024B7220198802F0FBBC00BFA09EFF1F94
:1068C000024B2020198802F0F3BC00BF809EFF1FFE
:1068D000024B3220198802F0EBBC00BF729EFF1FF2
:1068E000024B6820198802F0E3BC00BFA89CFF1F80
:1068F000024B6C20198802F0DBBC00BF189CFF1F04
:10690000024B6E20198802F0D3BC00BFCA9EFF1F45
:10691000024B5220198802F0CBBC00BF5A89FF1FDE
:10692000024B5020198802F0C3BC00BF108AFF1F21
:10693000024B5420198802F0BBBC00BF128AFF1F13
:10694000024B5C20198802F0B3BC00BF608AFF1FB5
:10695000024B5E20198802F0ABBC00BF5889FF1FB4
:10696000024B6020198802F0A3BC00BFE49DFF1F0A
:10697000024B5620198802F09BBC00BFB69CFF1F3B
:10698000244B1B880B2B43D8DFE803F00B10151AA0
:106990001F24292E33383D06084604221E490AF0DA
:1069A000ADBD084604221D490AF0A8BD08460422D0
:1069B0001B490AF0A3BD084604221A490AF09EBDED
:1069C0000846042218490AF099BD084604221749CE
:1069D0000AF094BD0846042215490AF08FBD084606
:1069E000042214490AF08ABD0846042212490AF01A
:1069F00085BD0846042211490AF080BD08460422DC
:106A00000F490AF07BBD084604220E490AF076BD04
:106A1000704700BF349EFF1FF82D0100AC2B010012
:106A2000602A0100482B0100642A0100042F0100A4
:106A3000682A01006C2A0100E02C0100702A010084
:106A4000042E0100742A0100064B074A10B41C886A
:106A5000064B0846002C14BF11461946042210BCF0
:106A60000AF04CBD8C9CFF1F782A01007C2A010093
:106A7000064B074A10B41C88064B0846002C14BF6E
:106A800011461946042210BC0AF038BDC69CFF1FEF
:106A9000782A01007C2A0100064B074A10B41C88A2
:106AA000064B0846002C14BF11461946042210BCA0
:106AB0000AF024BDE69DFF1F782A01007C2A010010
:106AC000064B074A10B41C88064B0846002C14BF1E
:106AD00011461946042210BC0AF010BD369EFF1F55
:106AE000782A01007C2A0100064B074A10B41C8852
:106AF000064B0846002C14BF11461946042210BC50
:106B00000AF0FCBCCA9CFF1F782A01007C2A010005
:106B10001B4B1B880A2B0AD8DFE803F00A0E12165B
:106B20001A1E22262A2E0600164B18680860704787
:106B3000154B186808607047144B18680860704758
:106B4000134B186808607047124B1868086070474C
:106B5000114B186808607047104B18680860704740
:106B60000F4B1868086070470E4B18680860704734
:106B70000D4B1868086070470C4B18680860704728
:106B8000F69DFF1FA42A01007C2A0100802A010033
:106B9000842A0100882A01008C2A0100902A010021
:106BA000942A0100982A01009C2A0100A02A0100D1
:106BB000F0B52B4E2B4FDFF8C4E005460FCE87B063
:106BC0006C460FC496E803003B68274A274F44F8F9
:106BD000040B40F6CC308342C8BF3A46BEF8006092
:106BE0002180012E11889278ADF80D108DF80F20BC
:106BF0002AD032D340F6CA02022E18BF00229A428F
:106C000026DAA3F698031A491A4AC3EB031381FB49
:106C100003011944DB17C3EB6123243382FB0321F7
:106C2000DA17C2EBA10202EB8201A3EB410330337E
:106C300030328DF813308DF811206946284616221F
:106C40000AF05CFC07B0F0BD40F698029A42D8DB2F
:106C5000094B1868CDF81100EFE740F6FC02CEE7CB
:106C6000B82A01003C9EFF1FAC2A0100A82A01009F
:106C70003B773B9867666666B02A0100D09DFF1F90
:106C8000F8B5174C174E2278174D33782F888E465B
:106C9000003218BF012201467046FFF771FA002347
:106CA00098423370237015DB14BF012000202B881D
:106CB0009F420ED040F23A72A3F5AF730B490C4CD1
:106CC00002FB03F381FB0312DB17A3EB62133233E6
:106CD0002360F8BD0749012218460A702270E6E7D2
:106CE000348BFF1FE99EFF1F949EFF1FB5814E1B33
:106CF000008AFF1F709FFF1F014B187802F070BAC7
:106D0000589FFF1F014B187802F084BADC90FF1FD8
:106D1000134BB3F9003030B583EAE374A4EBE374AA
:106D2000002BA0B218DB012300E0134603EB830223
:106D300052009442F9DA0B4D90FBF3F285FB03E429
:106D400003FB1200DB173032D3EBA40380B201F84F
:106D5000012BF1D10B7030BD2D230B700131E2E717
:106D6000DC90FF1F67666666144BB3F9003070B5A0
:106D700083EAE375A5EBE375002BACB21ADB0123C4
:106D800000E0034603EB830040008542F9DA0C4E35
:106D900094FBF3F086FB03E503FB1044DB17303074
:106DA000D3EBA503A4B201F8010BF1D105480B7098
:106DB000106070BD2D230B700131E0E7249CFF1F94
:106DC00067666666D02A0100134BB3F9003030B510
:106DD00083EAE374A4EBE374002BA0B218DB012375
:106DE00000E0134603EB830252009442F9DA0B4DA4
:106DF00090FBF3F285FB03E403FB1200DB17303258
:106E0000D3EBA40380B201F8012BF1D10B7030BD9C
:106E10002D230B700131E2E7BC89FF1F67666666B0
:106E2000134BB3F9003030B583EAE374A4EBE37499
:106E3000002BA0B218DB012300E0134603EB830212
:106E400052009442F9DA0B4D90FBF3F285FB03E418
:106E500003FB1200DB173032D3EBA40380B201F83E
:106E6000012BF1D10B7030BD2D230B700131E2E706
:106E7000789EFF1F67666666134BB3F9003030B526
:106E800083EAE374A4EBE374002BA0B218DB0123C4
:106E900000E0134603EB830252009442F9DA0B4DF3
:106EA00090FBF3F285FB03E403FB1200DB173032A7
:106EB000D3EBA40380B201F8012BF1D10B7030BDEC
:106EC0002D230B700131E2E75A89FF1F6766666662
:106ED000134BB3F9003030B583EAE374A4EBE374E9
:106EE000002BA0B218DB012300E0134603EB830262
:106EF00052009442F9DA0B4D90FBF3F285FB03E468
:106F000003FB1200DB173032D3EBA40380B201F88D
:106F1000012BF1D10B7030BD2D230B700131E2E755
:106F2000108AFF1F67666666134BB3F9003030B5F1
:106F300083EAE374A4EBE374002BA0B218DB012313
:106F400000E0134603EB830252009442F9DA0B4D42
:106F500090FBF3F285FB03E403FB1200DB173032F6
:106F6000D3EBA40380B201F8012BF1D10B7030BD3B
:106F70002D230B700131E2E7128AFF1F67666666F8
:106F8000134BB3F9003030B583EAE374A4EBE37438
:106F9000002BA0B218DB012300E0134603EB8302B1
:106FA00052009442F9DA0B4D90FBF3F285FB03E4B7
:106FB00003FB1200DB173032D3EBA40380B201F8DD
:106FC000012BF1D10B7030BD2D230B700131E2E7A5
:106FD000608AFF1F67666666134BB3F9003030B5F1
:106FE00083EAE374A4EBE374002BA0B218DB012363
:106FF00000E0134603EB830252009442F9DA0B4D92
:1070000090FBF3F285FB03E403FB1200DB17303245
:10701000D3EBA40380B201F8012BF1D10B7030BD8A
:107020002D230B700131E2E75889FF1F6766666602
:1070300008B5702002F056F9044B1988884204D034
:107040007020BDE8084002F033B908BDD09DFF1F95
:1070500008B5742002F046F9044B1988884204D020
:107060007420BDE8084002F023B908BD689EFF1FE8
:10707000054B1B880846042213B904490AF03EBA9E
:1070800003490AF03BBA00BF6C9CFF1FD82A0100DD
:10709000D42A01000E4B1B88032B17D8DFE803F01E
:1070A000110C0702084604220A490AF027BA0846CA
:1070B000042209490AF022BA0846042207490AF0C4
:1070C0001DBA0846042206490AF018BA704700BFE4
:1070D000DE9DFF1FE82A0100E42A0100E02A0100EA
:1070E000DC2A010010B40A4B0A4C0A4693E803005C
:1070F00083B0238802AC04E9030004EB8303104649
:1071000053F8081C052203B010BC0AF0F7B900BF01
:10711000D8220100489EFF1F30B40A4B0A4D0C468E
:1071200093E8070084B02B8804AD05E9070005EB60
:107130008303204653F80C1C042204B030BC0AF030
:10714000DDB900BFE0220100D09DFF1FF0B40C4D5F
:107150000C4F0E460FCD8CB001AC0FC40FCD0FC439
:1071600095E807003B8884E807000CAA02EB83033C
:10717000304653F82C1C04220CB0F0BC0AF0BEB907
:10718000EC2201002C9EFF1FF0B40B4D0B4F0E465E
:107190000FCD86B06C460FC495E803003B8884E8A9
:1071A000030006AA02EB8303304653F8181C04229E
:1071B00006B0F0BC0AF0A2B918230100DE9CFF1F44
:1071C000F0B40A4D0A4F0E460FCD86B001AC0FC485
:1071D0002A683B88226006AA02EB8303304653F8F4
:1071E000141C0C2206B0F0BC0AF088B93023010050
:1071F0006E9CFF1FF0B40A4D0A4F0E460FCD86B0AD
:1072000001AC0FC42A683B88226006AA02EB830304
:10721000304653F8141C042206B0F0BC0AF06EB9D4
:1072200044230100689EFF1F164B1B880BB31BB243
:1072300083EAE370A0EBE370002B30B584B21DDB72
:10724000012300E0134603EB830252009042F9DA77
:107250000D4894FBF3F280FB03E503FB1244DB17BC
:107260003032D3EBA503A4B201F8012BF1D10B709E
:1072700030BD0846042205490AF040B92D230B70A1
:107280000131DDE7A89CFF1F67666666EC2A0100F6
:10729000F0B40A4D0A4F0E460FCD86B001AC0FC4B4
:1072A0002A683B88226006AA02EB8303304653F823
:1072B000141C042206B0F0BC0AF020B958230100C7
:1072C000189CFF1F054B1B881BB9054B18680860ED
:1072D00070470846042203490AF010B9C09EFF1FF8
:1072E0007C2A0100782A0100164B1B880BB31BB2C5
:1072F00030B583EAE374A4EBE374002BA0B21CDB8B
:10730000012300E0134603EB830252009442F9DAB2
:107310000D4D90FBF3F285FB03E403FB1200DB173A
:107320003032D3EBA40380B201F8012BF1D10B7002
:1073300030BD064B1868086070472D230B70013173
:10734000DEE700BF5C9CFF1F676666667C2A010063
:10735000164B1B880BB31BB230B583EAE374A4EB66
:10736000E374002BA0B21CDB012300E0134603EB07
:10737000830252009442F9DA0D4D90FBF3F285FB43
:1073800003E403FB1200DB173032D3EBA40380B21B
:1073900001F8012BF1D10B7030BD064B1868086065
:1073A00070472D230B700131DEE700BF3A9EFF1FAF
:1073B000676666667C2A0100164B1B880BB31BB2FE
:1073C00030B583EAE374A4EBE374002BA0B21CDBBA
:1073D000012300E0134603EB830252009442F9DAE2
:1073E0000D4D90FBF3F285FB03E403FB1200DB176A
:1073F0003032D3EBA40380B201F8012BF1D10B7032
:1074000030BD064B1868086070472D230B700131A2
:10741000DEE700BF2C9CFF1F67666666F02A01004E
:10742000174B1B881BB31BB270B583EAE375A5EB42
:10743000E375002BACB21EDB012300E0034603EB37
:10744000830040008542F9DA0E4E94FBF3F086FB90
:1074500003E503FB1044DB173030D3EBA503A4B2E4
:1074600001F8010BF1D108480B70106070BD074B9B
:107470001868086070472D230B700131DCE700BFEE
:10748000C49CFF1F67666666F42A01007C2A01001F
:10749000164B1B880BB31BB230B583EAE374A4EB25
:1074A000E374002BA0B21CDB012300E0134603EBC6
:1074B000830252009442F9DA0D4D90FBF3F285FB02
:1074C00003E403FB1200DB173032D3EBA40380B2DA
:1074D00001F8012BF1D10B7030BD064B1868086024
:1074E00070472D230B700131DEE700BFA49EFF1F04
:1074F000676666667C2A0100164B1B880BB31BB2BD
:1075000030B583EAE374A4EBE374002BA0B21CDB78
:10751000012300E0134603EB830252009442F9DAA0
:107520000D4D90FBF3F285FB03E403FB1200DB1728
:107530003032D3EBA40380B201F8012BF1D10B70F0
:1075400030BD064B1868086070472D230B70013161
:10755000DEE700BF829EFF1F676666667C2A010029
:10756000164B1B880BB31BB230B583EAE374A4EB54
:10757000E374002BA0B21CDB012300E0134603EBF5
:10758000830252009442F9DA0D4D90FBF3F285FB31
:1075900003E403FB1200DB173032D3EBA40380B209
:1075A00001F8012BF1D10B7030BD064B1868086053
:1075B00070472D230B700131DEE700BFA09EFF1F37
:1075C000676666667C2A0100174B1B881BB31BB2DB
:1075D00070B583EAE375A5EBE375002BACB21EDB57
:1075E000012300E0034603EB830040008542F9DA03
:1075F0000E4E94FBF3F086FB03E503FB1044DB1710
:107600003030D3EBA503A4B201F8010BF1D1084847
:107610000B70106070BD074B1868086070472D2311
:107620000B700131DCE700BF809EFF1F6766666656
:10763000F42A01007C2A0100074B1B88022B06D08C
:10764000012B0CBF054B064B186808607047054BB3
:1076500018680860704700BFE49DFF1FFC2A010006
:10766000002B0100F82A0100054B1B881BB1054BBC
:10767000186808607047044B18680860704700BFBE
:10768000B69CFF1F082B0100042B0100184B1A8821
:1076900052B3184A128830B50A80B3F90030002B73
:1076A00083EAE374A4EBE374BCBF2D238B70A0B218
:1076B000ACBF02310331012300E0134603EB830228
:1076C00052009442F9DA0C4D90FBF3F285FB03E48F
:1076D00003FB1200DB173032D3EBA40380B201F8B6
:1076E000012BF1D10B7030BD044B18680860704756
:1076F000769CFF1F0C2B0100676666667C2A0100E2
:1077000070B53C4D2B780646002B35D11C4673785E
:107710000BB9204670BDFAF77DFB374A374B384826
:10772000127831781B78007802EB43034A1E03EB92
:1077300080030E2AEDD801A050F822F0A5770000B2
:10774000C777000013770000A577000013770000CB
:107750001377000013770000937700001377000081
:1077600013770000137700001377000013770000F1
:10777000137700008F770000AE21224803F056FEF9
:10778000204804F0A3F800232B700124BFE706F083
:1077900039FBAF211B4803F049FE1B4A012313703C
:1077A0002B70B6E783B91948038804294FF6FF7197
:1077B00003F1FF320CBF01230B46134403F07F0398
:1077C000013303800FE073B1013B114A32F81330EB
:1077D0004BB10E4E0F481049104A3380012300264A
:1077E00006700B701370084A0221012311702B7070
:1077F000204670BD348BFF1F859EFF1F869EFF1F96
:10780000879EFF1FF89EFF1F709FFF1F049EFF1F94
:10781000B09DFF1FA09CFF1F2F9CFF1F739FFF1F8A
:1078200010B5064B064C1A882046012101F02EFDAA
:1078300021884220BDE8104001F03ABD8C9CFF1F1A
:107840004C9CFF1F10B5064B064C1A88204602219F
:1078500001F01CFD21884220BDE8104001F028BD48
:10786000C69CFF1F4C9CFF1F10B5064B064C1A8888
:107870002046042101F00AFD21884220BDE8104085
:1078800001F016BDE69DFF1F4C9CFF1F10B5064B77
:10789000064C1A882046002101F0F8FC218842207D
:1078A000BDE8104001F004BD369EFF1F4C9CFF1F39
:1078B00008B5122001F016FD054B1988884206D044
:1078C000122001F0F5FCBDE8084001F009BC08BD3C
:1078D0002C9EFF1F08B5582001F004FD054B1988A8
:1078E000884206D0582001F0E3FCBDE8084001F0D2
:1078F000F7BB08BD3A9EFF1F08B5142001F0F2FC4B
:10790000054B1988884206D0142001F0D1FCBDE84F
:10791000084001F0E5BB08BDCA9CFF1FF0B480EA37
:10792000E075A5EBE0750028ACB21FDB1DBF2B2373
:107930000B704E1C0E46012300E0134603EB83023E
:1079400052009542F9DA0B4F94FBF3F287FB0305E3
:1079500003FB1244DB173032D3EBA503A4B206F8C5
:10796000012BF1D133700846F0BC70472D230B700A
:107970004E1CE0E767666666084B188828B10D283C
:1079800007D00D3800B2FFF7C9BF054A106808607C
:107990007047044A10680860704700BFCA9EFF1F06
:1079A0007C2A0100102B0100174B18880C2813D0DB
:1079B000192815D01A2817D01B2819D01C281BD01D
:1079C0001D281DD01E2803D00C3800B2FFF7A6BF1B
:1079D0000E4A1068086070470D4A106808607047CA
:1079E0000C4A1068086070470B4A106808607047BE
:1079F0000A4A106808607047094A106808607047B2
:107A0000084A106808607047729EFF1F2C2B010007
:107A1000142B0100182B01001C2B0100202B01004E
:107A2000242B0100282B0100034B1888A0EB8000B9
:107A3000400000B2FFF772BF589FFF1F024B18882B
:107A4000033800B2FFF76ABF4C9EFF1F024B188835
:107A50000C3800B2FFF762BF289CFF1F024B18884A
:107A6000183800B2FFF75ABF589CFF1F024B188806
:107A7000183800B2FFF752BF569CFF1F024B188800
:107A8000183800B2FFF74ABF4E9CFF1FC368188822
:107A9000183800B2FFF742BF054B1B881BB9054BD6
:107AA00018680860704708460422034909F026BD9B
:107AB0005E9CFF1F7C2A0100782A0100054B1B8871
:107AC0001BB9054B18680860704708460422034933
:107AD00009F014BDBC9CFF1F7C2A0100782A01001C
:107AE00030B5134C85B001252B463C22022120469F
:107AF000009503F011FD204603F0E8FE002240212E
:107B0000802320460191009311460A4B029504F010
:107B10008BFB204603F0E6FF07480849084A00238C
:107B2000036083800B608B801360938005B030BD51
:107B3000F89EFF1FE4250100D89EFF1FF09EFF1F47
:107B4000609FFF1F10B500EBC00000F10F02D2B222
:107B500093B284B09C1E981C3D2303918DE81900BC
:107B60003921024804F0C4FA04B010BDF89EFF1F8A
:107B7000014B01221A707047E99EFF1FF0B5694B57
:107B8000694C6A4F6A4E6B4D85B004228DE80C003B
:107B900002932046684B4022802103F0C5FA20461C
:107BA000664A6749674C08F029FE674A674B976148
:107BB000674FD761674F9F61674FDF61674FB7615D
:107BC000674FF761674FAF61674FEF61674FA7611D
:107BD0006748684FE761684F87616849684FC761C8
:107BE000684F8F61684A694FCF61694F9761694BF0
:107BF000694FD761694F9F61694E6A4FDF616A4F74
:107C00006A4DB7616A4FF7616A4F6B4CAF616B4F5A
:107C1000EF616B4F6B48A7616B4FE7616B4F6C492E
:107C200087616C4FC7616C4F6C4A8F616C4FCF613D
:107C30006C4F6D4B97616D4FD7616D4F6D4E9F616E
:107C40006D4FDF616D4FB7616D4D6E4FF7616E4FD8
:107C5000AF616E4C6E4FEF616E4FA7616E486F4F14
:107C6000E7616F4F87616F496F4FC7616F4F8F61DA
:107C70006F4A704FCF61704F9761704B704FD761F3
:107C8000704F9F61704E714FDF61714FB761714DE1
:107C9000714FF761714FAF61714C724FEF61724F6D
:107CA000A7617248724FE761724F73498761734FE2
:107CB000C761734F734A8F61734FCF61734F744BBA
:107CC0009761744FD761744F744E9F61744FDF6139
:107CD000744F754DB761754FF761754F754CAF6156
:107CE000754F76487649EF61764F774DA761DFF89B
:107CF00008E2E561754F764D764C774A774B8761A0
:107D0000C5618C61764E774F774D784CC1F81CE099
:107D1000774878499761D5619C61D861B16005B0B9
:107D2000F0BD00BF40420F00F89EFF1F4D7A0000DB
:107D3000A48EFF1F9C8CFF1FF890FF1F1C89FF1F44
:107D400081B10000588FFF1FBC8DFF1F348FFF1FB4
:107D5000E56700003D7A0000F1670000496A000015
:107D600021780000716A000045780000996A0000DF
:107D7000988DFF1F69780000E5700000088DFF1FD7
:107D800001680000C16A0000748DFF1F8D7800003B
:107D9000297A0000508DFF1FF96C0000116D000062
:107DA000108FFF1F056D000019710000308CFF1F40
:107DB000317000004D710000C48FFF1FB1780000CA
:107DC00051730000E48CFF1FD5780000696D00003E
:107DD000EC8BFF1F11680000E96A00003090FF1F64
:107DE000F9780000B9730000C08CFF1F2168000003
:107DF00021740000E08DFF1F3168000091740000C5
:107E0000788CFF1F41680000C96D00005C8BFF1F6C
:107E10005168000089710000C88AFF1F6168000076
:107E2000216E00002C8DFF1F716800008D76000010
:107E3000EC8EFF1F81680000C1710000B890FF1F29
:107E400091680000F9740000808EFF1FA168000097
:107E500061750000808BFF1FB1680000F5710000A4
:107E6000E88FFF1F51700000C9750000C88EFF1F0A
:107E7000C1680000A9790000A48BFF1FD168000031
:107E800029720000388BFF1FE1680000917200002A
:107E9000808AFF1FF1680000797900008890FF1F39
:107EA00001690000796E0000548CFF1F1169000009
:107EB000D16E0000108BFF1F21690000C88BFF1FCF
:107EC0007C8FFF1F296F000031690000816F000067
:107ED00041690000D96F0000EC8AFF1FA48AFF1FD0
:107EE000AC90FF1F397600006169000069760000E0
:107EF000716900008184000051690000F0B5461CE2
:107F000083B00D460127032336B22AB20446314618
:107F10008DE888002448ADB204F080F80C23AA1C38
:107F200012B200930197052321B21F4804F076F89E
:107F30001E4A1F4B12881B68BA422AD023D3022A3A
:107F400010D11C4CA3F6CA0384FB03241C44DB178A
:107F5000C3EB24140A2CA8BF0A2424EAE474A2B2B6
:107F600023B202E000231A461C460D35AA1A01204E
:107F70000093019012B2314603230B4803F0CCFF6B
:107F8000204603B0F0BD0C4CA3F6FC0384FB032495
:107F9000DDE7084CA3F6980384FB03241C44DB179D
:107FA000C3EBE404D6E700BFF89EFF1FD09DFF1F80
:107FB0003C9EFF1F898888881F85EB512DE9F0437F
:107FC0008FB283B0DFF84C80BD1D461D2DB204B2C8
:107FD00036B24FF001090AB22346314640460095B9
:107FE000CDF8049003F0CAFF2A46334621464046A6
:107FF0008DE8200203F0C2FF07F10C020095334622
:1080000012B22146CDF80490404603F0B7FF03B00A
:10801000BDE8F083F89EFF1F2DE9F043804685B050
:10802000002956D10121304804F03EFB2F4998F831
:10803000062098F8083011F80290994522DA4FEAA4
:1080400089064D460C24D8F80C3027489B595F68A8
:1080500022B2002104F024FB384609F091F9394698
:108060000246214804F0B6FC1F4804F0C9FC98F809
:10807000083001350934AB42A4B206F1040601DD33
:10808000422CE0D1B9F1000F13D109F1060999454D
:108090000CDA3C2301213B220391029300930192CD
:1080A00039233F223A21104804F022F805B0BDE8F8
:1080B000F0830F2301213B2203910293009301924D
:1080C00039230C223A21084804F012F898F80830B5
:1080D000DBE700213423009301913F230C22024867
:1080E00003F01AFF9EE700BFF89EFF1FF09EFF1FE0
:1080F00010B5104C0121204604F0DCFA2046012185
:1081000004F0D2FA20463422552104F0C9FA204660
:108110000222094904F05EFC20460522074904F0CA
:1081200059FC204604F06CFC2046BDE8104003F0EA
:10813000D9BC00BFF89EFF1F302B0100342B01007B
:1081400070B50D46064609F01BF900EB40008400AF
:10815000002D36D0284609F013F900EB400040000E
:1081600023185B1003F16001091A282209B217488D
:10817000C3F1600404F094FA0121144804F094FA65
:10818000284609F0FDF829460246104804F022FC72
:108190000E4804F035FC02210C4804F085FA21B2A7
:1081A00021220A4804F07CFA304609F0E9F8314609
:1081B0000246064804F00EFC0448BDE8704004F096
:1081C0001FBC6410C4F16004E5E700BFF89EFF1F08
:1081D000184B70B5B3F9003083EAE374A4EBE37491
:1081E000002B82B0A1B21EDB68466D46012300E081
:1081F000134603EB830252009442F9DA0E4E91FBD0
:10820000F3F286FB03E403FB1211DB173032D3EBEE
:10821000A40389B205F8012BF1D119462B70FFF7A1
:108220008FFF02B070BD2D238DF800300DF10105D8
:108230006846DBE7F49DFF1F6766666610B50D4B69
:108240001B5C51F82340237884B013B1012004B0A3
:1082500010BD04AA01A942F8103D2046A369984721
:10826000A38A9B07F2D401A80099FFF769FF0120B8
:1082700004B010BDD89EFF1F2DE9F04F2F4DDFF841
:10828000CCB0DFF8C4A0DFF8C8900FCD91B003AC3C
:108290000FC40FCD0FC40FCD0FC42B682360002572
:1082A000A8462F462E4600E09846BAF800302449EA
:1082B0005BF8232028461123F8F7F6F900EBC004F9
:1082C00000EB840089FB00340444C017C0EB643425
:1082D000C4F13C00C6F13C0207F14101012600B2A5
:1082E00008F1410300901BB2019612B209B2154881
:1082F00003F044FE08EB060305F211153C2B26465D
:10830000ADB24746D0D134226B210E4804F0C8F9F3
:1083100000210C4804F0C8F90B4B1B8810AA02EB93
:10832000830353F8344C204609F02AF802460548E6
:10833000214611B0BDE8F04F04F04CBB6C230100A6
:10834000BC1C0100F89EFF1F3E9CFF1F201B01006C
:108350000900028010B5424C424882B003F0B6FAE0
:108360002378C3B906213F4804F09EF92378012BF6
:1083700037D90A22022B11463A486BD004F090F903
:1083800039490322374804F025FB364802B0BDE8DE
:10839000104004F035BB354B1A7801210523002A23
:1083A00035D10191009311462E4803F037FE304B32
:1083B0001A78002A36D00523012201920093002268
:1083C0000A21284803F0A8FD2A4B1A78002A35D143
:1083D00001210523019100931421224803F01EFE80
:1083E000C0E7254C2388092B32D9632B8CBF0A2187
:1083F0001F210A221B4804F053F92188194804F070
:108400004FFB184802B0BDE8104004F0F9BA002252
:10841000019100931146134803F07EFD144B1A7826
:10842000002AC8D105230121019100930A210D489A
:1084300003F0F4FD0F4B1A78002AC9D0012205235E
:108440000192009300221421064803F065FD89E79C
:108450003021CEE704F024F90322084992E700BF57
:10846000739FFF1FF89EFF1F402B0100859EFF1F7B
:10847000869EFF1F879EFF1F049EFF1F3C2B01004F
:10848000F8B56D4D287840B96C4B1B6899425CD3A8
:108490006B4A012313702B70F8BD0C460026694807
:1084A000664F03F013FA04F6AC53324665483B605E
:1084B00031212E7004F0F4F801216248624D04F07D
:1084C000F9F831465F4804F0EFF805225F495D484E
:1084D00004F080FA5B4804F093FA0C22102159480A
:1084E00004F0DEF80B225A49564804F073FA0522CC
:1084F0005849544804F06EFA524804F081FA564B39
:1085000050481C68A4F69803C3EB031385FB0325AE
:108510001D441021DB172022C3EB652504F0C0F8B1
:1085200040F6CC339C4205F124054FF022014FF078
:1085300004000BDCFFF7E2FC484B1C88064674B3D2
:10854000012C46D0022C41D00120F8BDFFF736FDAA
:10855000092243493B4804F03DFA2A2210213948B8
:1085600004F09EF83F4C374884FB0534EB17C3EB0F
:10857000A404214604F094FA01223B49314804F056
:1085800029FA04EB8401A5EB41012E4804F088FA96
:10859000012236492B4804F01DFA0120F8BD344968
:1085A0001022284804F016FA264804F029FA2A2254
:1085B0001021244804F074F83146224804F070FA7F
:1085C00007222C491F4804F005FACBE70C222A4960
:1085D000E7E70C2229491B4804F0FCF9194804F08C
:1085E0000FFA2A221021174804F05AF8314615488C
:1085F0001C4E04F055FA07221E49124804F0EAF90D
:1086000086FB0536EB17C3EBA60631460D4804F092
:1086100047FA224614490B4804F0DCF906EB8601C0
:10862000A5EB4101074804F03BFA22460F490548F3
:1086300004F0D0F92046F8BD348BFF1FE09EFF1FE9
:10864000709FFF1FF89EFF1F3B773B98442B010054
:108650004C2B0100342B01003C9EFF1FD09DFF1FBF
:10866000582B010067666666D03201004032010077
:10867000642B0100782B0100902B0100802B01005E
:108680002DE9F041754C2278002A05460F4614BFAB
:108690004FF001084FF000084ED1714E3368CB1AED
:1086A000B3F5FA6F04D86B78A3B94046BDE8F08102
:1086B0006C4B6D486D49DFF8D0E11A7001230370EF
:1086C0000988237026208EF8002000F0F1FD6B78D9
:1086D000002BEAD03760F9F79DFB654A654B664988
:1086E000127828781B78097802EB4303421E03EBCB
:1086F00081030E2AD9D801A151F822F0ED8700009C
:10870000B9870000AB860000ED870000AB86000053
:10871000AB860000AB860000A1870000AB8600009E
:1087200053870000AB860000AB860000AB860000DC
:10873000AB8600004F870000AF215048484E02F042
:1087400075FEFFF707FE002337602370ABE705F0E7
:1087500059FB4A4803F0BAF80221484803F0A4FF45
:108760000F222321454803F09BFF0522444943483B
:1087700004F030F9414804F043F91E2223213F4818
:1087800003F08EFF05223F493C4804F023F93B48A3
:1087900004F036F9394803F0A5F900F0ADFC84E7A0
:1087A000394D2B78012B50D9304B2620198800F0F9
:1087B0007FFD00232B7078E7002B3FF476AF013B61
:1087C000324A32F81330002B3FF46FAF274C304859
:1087D00025492D4A23804FF001080023037081F8BA
:1087E000008082F80080FFF7B5FD5EE793B1013BA2
:1087F000264A32F8131019B31C4B254D1A4C224A45
:1088000019800026012326202E702370137000F09B
:108810004FFD15E0154C1E4922880B7004284FF6B9
:10882000FF7002F1FF310CBF012202460A440E4ED6
:10883000154D02F07F0201320121228031702B7030
:10884000FFF788FD4FF001082FE70649064A01238C
:108850000020087013702370A6E700BF348BFF1F41
:108860006C9FFF1F709FFF1F2F9CFF1F049EFF1F09
:10887000859EFF1F869EFF1F879EFF1FF89EFF1F7E
:10888000A02B0100A82B0100739FFF1FB09DFF1FAD
:10889000A09CFF1F2DE9F04F05468BB00F46AD4859
:1088A0000121164603F006FFAA8812F0010440F0E9
:1088B000B080DFF8CC8298F80030002B7DD1AB7906
:1088C000A54AD15CA1B9DFF8BCA279781AF8039067
:1088D00041B339780139072900F2B780DFE811F098
:1088E000F1005401B5006C01B500B500B500E90018
:1088F0007C78002C00F0CA800139EC68387854F894
:108900002170FC68411EB4F80080072900F2A7809E
:10891000DFE811F074015901A5006C01A500A50064
:10892000A5009F00DFF854A2DAF80020B21AB2F5D1
:10893000967F75D9894A107801281ABF01201070D6
:108940001170874A18BF0146D05CC0EB0900C0B265
:10895000FFF7F8F80124CAF80060AB889B0770D5D0
:108960007B78002B6DD0F9F755FA7E4B7E4A7F4815
:108970001B78127839780078022515FB02330A2912
:1089800003EB800300F04E810C295AD1002B58D004
:1089900003F11900764E774A013B0021400080B276
:1089A00026F813100123157088F8003000F080FCC1
:1089B000714B032220461A702FE0664802F086FFB2
:1089C0000121644803F070FE62482246214603F00C
:1089D00067FEAB88580725D42C68204608F0D0FCE9
:1089E000214602465B4803F0F5FF5A4804F008F8B8
:1089F000092201238DE80C0000217F23554803F054
:108A0000BDFA00212846FFF707FB002388F8003055
:108A100055E7AB683146384698470BB0BDE8F08F54
:108A20000846FAE72B6804A8984704A808F0A8FCB1
:108A300004A90246474803F0CDFF464803F0E0FF93
:108A4000D6E720460BB0BDE8F08F00240AF803906B
:108A500083E70021D1543846FB699847FC68A4F8A5
:108A60000080002725223C238DE884004121182224
:108A7000384803F051FAE968A879FFF7DFFB374A75
:108A80003E4B17701E600BB0BDE8F08F3B490A6883
:108A9000B21AB2F5967FD4D9304F0E603E78012ECF
:108AA00000F0B480E968184601233B70FFF7C6FB6D
:108AB000B3E7304AE9791170012288F800200024D8
:108AC000C4E72A7A013A4A45BFDD09F10104E4B25C
:108AD000A145BAD0224E16F803B0CBEB0900C0B2C4
:108AE0000021FFF72FF82B7A052BD9461BD9CBEBAA
:108AF0000402042A40F3AE80A4F1040BBBF1000F82
:108B0000C0F2B080063B5B45A8BF5B465FFA83F9C5
:108B1000AA791348B15C994205D000F8029001216E
:108B20002846FFF779FAC9EB0400C0B201210B4EC9
:108B3000FFF708F8002134230191009305483170B4
:108B400040230B223F21A14603F0E6F90124AB7933
:108B50007CE700BFF89EFF1F609FFF1F719FFF1FF4
:108B6000F09EFF1F859EFF1F869EFF1F879EFF1F93
:108B7000B09DFF1F709FFF1F739FFF1F5C9FFF1F14
:108B8000348BFF1FD89EFF1F0FFA89F1E868604CF5
:108B900050F821602168049134785E490498086097
:108BA000002C71D0012C7FF450AF5B4A317A88F8E9
:108BB00000401170002449E7B9F1000F50D009F1CD
:108BC000FF34E4B284E7B98A01F0040189B20029D4
:108BD0003FF440AF3B6A03929847039A00283FF462
:108BE0003DAFAB79FC680021D15438E77B8A43451F
:108BF0003CD908F101081FFA88F830E73B8A434561
:108C00003BD208F1FF381FFA88F828E725238DE8C2
:108C1000180042483C703C231822412103F07CF9A3
:108C20003046FAE6002B3FF40CAF3D4A3D4E11882A
:108C3000394A03F11900013B400080B226F81310B5
:108C4000012388F80030157000F032FB364B2046C7
:108C50001D70E2E6002A3FF755AF04F1FF3B4DE7F8
:108C60004C46F3E64FF000094B4651E7BB8ADA0762
:108C70007FF5F5AEB7F81080F1E6BB8AD9077FF52E
:108C8000EEAEB7F81280EAE62849C85CC0EB0900EE
:108C900009F1010EC0B201214FF0340B02F803E0DC
:108CA000FEF750FFB6681D48019440230B223F2178
:108CB0000124CDF800B003F02FF940230B223F210F
:108CC0001648CDF800B0019403F0A8F921461348E6
:108CD00003F0EAFC304608F053FBA0EB800000F103
:108CE0005F0109B20F220D4803F0DAFC304608F0AC
:108CF00047FB31460246094803F06CFE074803F083
:108D00007FFEE968A879FFF799FAAB799EE600BF84
:108D1000B09FFF1F5C9FFF1F709FFF1FF89EFF1FEC
:108D2000049EFF1FB09DFF1F739FFF1FF09EFF1F3C
:108D30002DE9F047DFF808926D4B99F800601B6849
:108D4000DFF800A282B0003601934FF0030018BF95
:108D50000126019F9AF8008004F00CFD05460420CE
:108D600004F008FD0446052004F004FD800040EAFC
:108D70004404062004F0FEFC2C4364B25D4944EA3E
:108D8000C0000A7880F00F03DBB29A425A4A3CD006
:108D90001760002259480B7003788DF800808DF819
:108DA000012053B3564A12684EF66021BA1A8A421D
:108DB00019D8022B59D0012B5FD0062B48D0032B9A
:108DC00063D0042B69D0052B77D0072B7DD0082BDF
:108DD00000F08380092B68D016B14A4802F082FE69
:108DE00002B0BDE8F087484A484C002301212370B7
:108DF00003701360938089F800103A46694644482E
:108E0000FFF748FD3043C6B2E6E71268BA1A1E2AD9
:108E10006BD99AF80020934222D0394C3D488AF809
:108E20000030012B276082EA030207609846B1D028
:108E3000042BAFD137480068381AB0F5C87FA9D9DC
:108E4000354C2068381A3228A4D927601A46A1E781
:108E50003A4669463148FFF71DFD3043C6B2BBE7CD
:108E6000012B4FF00002E3D1E4E73A4669462C4873
:108E7000FFF710FD3043C6B2AEE73A4669462948CF
:108E8000FFF708FD3043C6B2A6E73A4669462648D2
:108E9000FFF700FD3043C6B29EE73A4669462348D5
:108EA000FFF7F8FC3043C6B296E73A4669462048D9
:108EB000FFF7F0FC3043C6B28EE73A4669461D48DC
:108EC000FFF7E8FC3043C6B286E73A4669461A48DF
:108ED000FFF7E0FC3043C6B27EE73A4669461748E2
:108EE000FFF7D8FC3043C6B276E7002252E700BF56
:108EF000B09FFF1F749FFF1FE49EFF1F709FFF1F07
:108F0000689FFF1FF89EFF1F609FFF1F729FFF1F3C
:108F1000B4250100789FFF1FEC9EFF1FE42901008C
:108F20000C25010010240100AC2301009031010048
:108F30000024010068240100F0240100AC90FF1F10
:108F4000348BFF1FE89EFF1F28B11028044BA8BFD9
:108F5000102018607047024B01201860704700BF56
:108F60007C9FFF1F38B50F4D2B78013B01381B024A
:108F7000C4B203F47063200443F4404343F00C0391
:108F800000F4FE00184305F05DFD2868013860F02C
:108F90003F00C0B204F084FD2046BDE8384004F034
:108FA0007FBD00BF7C9FFF1F70B5124D2B78013B2A
:108FB0001B0203F47063064643F430430806320490
:108FC00000F0FE4043F00B03034302F4FE0018439D
:108FD0000C4605F037FD2868013860F04F00C0B23C
:108FE00004F05EFD304604F05BFD2046BDE87040B5
:108FF00004F056BD7C9FFF1F70B5124D2B78013BCE
:109000001B0203F47063064643F41043080632045F
:1090100000F0FE4043F00903034302F4FE0018434E
:109020000C4605F00FFD2868013860F06F00C0B2F3
:1090300004F036FD304604F033FD2046BDE87040B4
:1090400004F02EBD7C9FFF1F38B5104D2B78013BDF
:109050001B0203F47063044643F41043000443F01E
:10906000090300F4FE00184305F0ECFC2868013801
:1090700060F06F00C0B204F013FD204604F010FD54
:109080000020BDE8384004F00BBD00BF7C9FFF1FEF
:1090900038B50E4D2B78013B1B0203F47063044678
:1090A00043F45043000443F00D0300F4FE00184362
:1090B00005F0C8FC2868013860F02F00C0B204F049
:1090C000EFFC2046BDE8384004F0EABC7C9FFF1F5F
:1090D00008B5002005F080FD0028FAD108BD00BFCA
:1090E00008B564210720FFF75FFF7F210B20BDE853
:1090F0000840FFF759BF00BF10B500217B20FFF7E4
:1091000053FF0024E0B2FFF79FFF0134022004F078
:1091100067FB802CF6D110BD10B504464FF44060BB
:1091200004F06EFC04F0C6FC2CB1102C044BA8BF5C
:1091300010241C6010BD024B01241C6010BD00BF38
:109140007C9FFF1F10B5044641F0E00004F0A8FC2E
:1091500004F07F0004F0A4FCC4F3C610BDE8104086
:1091600004F09EBC38B5134D2B78044641F6FF72CF
:10917000A0F50050824203F1FF33A8BF02461B0254
:1091800002F5005203F47063100443F4604343F0AB
:109190000E0300F4FE005204184302F0FE42104396
:1091A00005F050FC296801392046C9B2BDE83840B5
:1091B000FFF7C8BF7C9FFF1F38B504460D46F0205F
:1091C00004F06EFC35B1254414F8010B04F068FC82
:1091D000AC42F9D1F720BDE8384004F061BC00BFD3
:1091E00000B50B4B83B00246998818680090032A9B
:1091F000ADF8041002D903B05DF804FB68460621FF
:109200008DF80520FFF7D8FF03B05DF804FB00BF21
:109210000032010000B50B4B024683B018689988F4
:109220000090131F4C2BADF8041002D903B05DF869
:1092300004FB684606218DF80520FFF7BDFF03B04B
:109240005DF804FB08320100030203F4FE43C0F39F
:10925000C6101843704700BF03784078DB0103F461
:109260007E5300F07F001843704700BF82B002AA0F
:10927000114642F8040D002012F8013B03F07F0371
:10928000914243EA0020F7D102B07047003210B497
:1092900003884FF0010404FA01F418BF012202FA16
:1092A00001F123EA04020A43028010BC704700BFA8
:1092B00070B5CEB20C46054603F024FE864203D0BC
:1092C0003146284603F038FE0135284603F01AFEE1
:1092D000240A844205D021462846BDE8704003F0A8
:1092E0002BBE70BD38B5054603F00CFE4FF00004F0
:1092F00060F30704681C03F005FE60F30F24A0B2BE
:1093000038BD00BFF8B504460020FFF7EBFF002C86
:1093100000F051854FF4AF610220FFF7C9FF4FF411
:109320007A610420FFF7C4FF4FF496610620FFF72F
:10933000BFFF4FF4FA610820FFF7BAFF4FF4FA615C
:109340000A20FFF7B5FF40F6B8310C20FFF7B0FF59
:109350004FF42F612220FFF7ABFF40F6AC512420E1
:10936000FFF7A6FF7D212A20FFF7A2FF0C210E2088
:10937000FFF79EFF01211020FFF79AFF0221122024
:10938000FFF796FF00211420FFF792FF002116201F
:10939000FFF78EFF02211820FFF78AFF01211A2014
:1093A000FFF786FF01211C20FFF782FF04211E200A
:1093B000FFF77EFF14212020FFF77AFF01212620EE
:1093C000FFF776FF03212820FFF772FF04212C20EE
:1093D000FFF76EFF14212E20FFF76AFF00213020D7
:1093E000FFF766FF0C213220FFF762FF00213420D7
:1093F000FFF75EFF00213620FFF75AFF00213820DB
:10940000FFF756FF00213A20FFF752FF00213C20D2
:10941000FFF74EFF00213E20FFF74AFF00214020CA
:10942000FFF746FF00214220FFF742FF1F214420A3
:10943000FFF73EFF13214620FFF73AFF0E21482099
:10944000FFF736FF11214A20FFF732FF0A214C2097
:10945000FFF72EFF00214E20FFF72AFF06215020A4
:10946000FFF726FF02215220FFF722FF0C21542094
:10947000FFF71EFF00215620FFF71AFF002158209A
:10948000FFF716FF01215A20FFF712FF08215C2089
:10949000FFF70EFF0A215E20FFF70AFF0021602080
:1094A000FFF706FF04216220FFF702FF012164207D
:1094B000FFF7FEFE00216620FFF7FAFE0B21682071
:1094C000FFF7F6FE7F216A20FFF7F2FE00216C20F5
:1094D000FFF7EEFE00216E20FFF7EAFE002170206C
:1094E000FFF7E6FE00217220FFF7E2FE0021742064
:1094F000FFF7DEFE1F217620FFF7DAFE132178202A
:10950000FFF7D6FE0E217A20FFF7D2FE11217C2034
:10951000FFF7CEFE0A217E20FFF7CAFE1F21802022
:10952000FFF7C6FE13218220FFF7C2FE0E21842022
:10953000FFF7BEFE11218620FFF7BAFE0A21882020
:10954000FFF7B6FE00218A20FFF7B2FE00218C2033
:10955000FFF7AEFE00219620FFF7AAFE002198201B
:10956000FFF7A6FE00219A20FFF7A2FE05219C200E
:10957000FFF79EFE06219E20FFF79AFE0021A02005
:10958000FFF796FE7F21A220FFF792FE40F2A46132
:10959000A420FFF78DFE4FF4E161A620FFF788FEBF
:1095A00028210020FFF784FE0220FFF79BFEB0F584
:1095B000805F034680F07485D24A04201380FFF751
:1095C00091FEB0F5805F034680F06185CE4A0620AB
:1095D0001380FFF787FEA0F52F739BB2B3F57A6F68
:1095E000024606D940F628210620FFF761FE40F624
:1095F0002822C64B08201A80FFF774FEA0F52F73AF
:109600009BB2B3F57A6F024606D940F6E4410820D2
:10961000FFF74EFE40F6E442BD4B0A201A80FFF7EA
:1096200061FEA0F5FA739BB240F6AC518B42024644
:1096300006D94FF4FA610A20FFF73AFE4FF4FA62B6
:10964000B44B0C201A80FFF74DFEA0F5FA739BB2C5
:1096500040F6AC518B42024606D940F6B8310C2098
:10966000FFF726FE40F6B832AB4B0E201A80FFF70C
:1096700039FE1828034600F20385A84A10201380FB
:10968000FFF730FE431E9BB20F2B024604D9012187
:109690001020FFF70DFE0122A14B12201A80FFF7C8
:1096A00021FE0A28034600F2E4849E4A1420138017
:1096B000FFF718FE0128034604D900211420FFF704
:1096C000F7FD0023984A16201380FFF70BFE7F2832
:1096D000034600F2C784954A18201380FFF702FE64
:1096E0000528034600F2B784914A1A201380FFF739
:1096F000F9FD0C28034600F2A7848E4A1C20138033
:10970000FFF7F0FD0428034600F297848A4A1E20E2
:109710001380FFF7E7FD0928034600F28784874A94
:1097200020201380FFF7DEFD4628034600F27784F1
:10973000834A22201380FFF7D5FDA0F5FA739BB270
:1097400040F6AC518B42024606D94FF42F612220DD
:10975000FFF7AEFD4FF42F627A4B24201A80FFF7FB
:10976000C1FDA0F5FA739BB240F6AC54A342024689
:1097700004D921462420FFF79BFD2246724B262068
:109780001A80FFF7AFFD7F28034600F241846F4A3D
:1097900028201380FFF7A6FD0628034600F2318437
:1097A0006B4A2A201380FFF79DFDA0F132039BB284
:1097B000B3F5967F024604D97D212A20FFF778FD74
:1097C0007D22644B2C201A80FFF78CFD0C28034669
:1097D00000F21084604A2E201380FFF783FD1E28BC
:1097E000034600F200845D4A30201380FFF77AFDC3
:1097F0000928034600F2F183594A32201380FFF70B
:1098000071FD1E28034600F2E283564A342013807D
:10981000FFF768FD7F28034600F2D383524C3620C1
:109820002380FFF75FFD7F28034600F2C4833820C2
:109830006380FFF757FD7F28034600F2B6833A2086
:10984000A380FFF74FFD7F28034600F2A8833C204A
:10985000E380FFF747FD7F28034600F29A833E200E
:109860002381FFF73FFD7F28034600F28C834020D1
:109870006381FFF737FD7F28034600F27E83422095
:10988000A381FFF72FFD394D28804420FFF72AFDE3
:109890003028034600F26B83354A46201380FFF7D9
:1098A00021FD3028034600F25C83324C482023809F
:1098B000FFF718FD3028034600F24D834A206380ED
:1098C000FFF710FD3028034600F23F834C20A380B1
:1098D000FFF708FD3028034600F231834E20E38075
:1098E000FFF700FD0128034604D900214E20FFF7B1
:1098F000DFFC0023204A50201380FFF7F3FC431EB7
:109900003CE000BFD89CFF1F9A9EFF1F8E9CFF1F4C
:10991000709EFF1F409EFF1F549CFF1F289CFF1F2F
:10992000F49DFF1F2C9EFF1FCA9CFF1F2C9CFF1F36
:10993000DE9CFF1F769CFF1F6E9CFF1F5C9CFF1F21
:10994000809EFF1FEC9DFF1FE89DFF1F049EFF1FD1
:109950004C9EFF1F949EFF1F3E9CFF1FC49CFF1F39
:10996000A49EFF1F729EFF1FB09DFF1F4C9CFF1FF8
:109970004E9CFF1F509EFF1F6C9CFF1F9BB20B2B2A
:10998000024604D906215020FFF792FC0622CF4B55
:1099900052201A80FFF7A6FC0428034600F2C98271
:1099A000CB4A54201380FFF79DFC431E9BB21D2B16
:1099B000024604D90C215420FFF77AFC0C22C54B37
:1099C00056201A80FFF78EFC0128034604D9002197
:1099D0005620FFF76DFC0023BF4A58201380FFF785
:1099E00081FC7F28034600F29E82BC4A5A201380E5
:1099F000FFF778FC431E9BB2092B024604D90121D4
:109A00005A20FFF755FC0122B54B5C201A80FFF766
:109A100069FC431E9BB2102B024604D908215C202E
:109A2000FFF746FC0822AF4B5E201A80FFF75AFC76
:109A3000431E9BB21D2B024604D90A215E20FFF76C
:109A400037FC0A22A84B60201A80FFF74BFC022843
:109A5000034600F26282A54A64201380FFF742FCAD
:109A60000128034604D901216420FFF721FC0123CA
:109A70009F4A62201380FFF735FCC31E9BB2012B67
:109A8000024604D904216220FFF712FC0422994BFC
:109A900066201A80FFF726FC7F28034600F23782F3
:109AA000954A68201380FFF71DFC7F28034600F2CB
:109AB0002882924A6A201380FFF714FC7F2803460D
:109AC00000F219828E4A6C201380FFF70BFC0428E9
:109AD000034600F20A828B4A6E201380FFF702FCD5
:109AE0001928034600F2FB81874A70201380FFF794
:109AF000F9FB0228034600F2EC81844A72201380AD
:109B0000FFF7F0FB0628034600F2DD81804A74204F
:109B10001380FFF7E7FB0428034600F2CE817D4A5D
:109B20008A201380FFF7DEFB0A28034600F2BF817C
:109B3000794A8C201380FFF7D5FB0428034600F2F6
:109B4000B081764A98201380FFF7CCFB01280346AA
:109B500004D900219820FFF7ABFB0023704A9A201C
:109B60001380FFF7BFFB0128034604D900219A2088
:109B7000FFF79EFB00236B4A96201380FFF7B2FB92
:109B80000B28034600F28781674A9C201380FFF769
:109B9000A9FB831E9BB2032B024604D905219C20FE
:109BA000FFF786FB0522614B76201A80FFF79AFBB0
:109BB0003028034600F269815D4A78201380FFF760
:109BC00091FB3028034600F25A815A4C7A202380B8
:109BD000FFF788FB3028034600F24B817C2063802E
:109BE000FFF780FB3028034600F23D817E20A380F2
:109BF000FFF778FB3028034600F22F818020E380B6
:109C0000FFF770FB3028034600F221814A4A822088
:109C10001380FFF767FB3028034600F21281474CA0
:109C200084202380FFF75EFB3028034600F2038187
:109C300086206380FFF756FB3028034600F2F5804C
:109C40008820A380FFF74EFB3028034600F2E78010
:109C5000A020E380FFF746FB0128034604D900213A
:109C6000A020FFF725FB0023354A9E201380FFF735
:109C700039FBC31E9BB20C2B024604D906219E2041
:109C8000FFF716FB06222F4BA2201A80FFF72AFBB4
:109C9000431E9BB27E2B024604D97F21A220FFF7F0
:109CA00007FB7F22284BA4201A80FFF71BFBA0F59F
:109CB000AF639BB2B3F5167F024647D940F2A46169
:109CC000A420FFF7F5FA40F2A4623FE0108AFF1FDC
:109CD0005A89FF1F128AFF1FB69CFF1F3A9EFF1F63
:109CE000249CFF1F608AFF1F5889FF1FE49DFF1FF0
:109CF000489EFF1F7C9CFF1F829EFF1FA89CFF1F8A
:109D0000609CFF1F189CFF1FCA9EFF1FD09DFF1F56
:109D1000A09EFF1F689EFF1FF69DFF1FDE9DFF1F79
:109D20005E9CFF1FBC9CFF1F349EFF1F429CFF1FB9
:109D3000569CFF1FC09DFF1F589CFF1FC89DFF1F03
:109D4000C09EFF1FBC89FF1F789EFF1FD94BA62016
:109D50001A80FFF7C7FAA0F5AF639BB2B3F5167F81
:109D600006D9A6204FF4E161FFF7A2FA4FF4E160B3
:109D70002B88DFF860E3D04FD04AD14DD14ED24C82
:109D8000D24903F0010CAEF800C0C3F3400EA7F8AF
:109D900000E0C3F380071780C3F3C007CC4A2F70DD
:109DA000C3F30017C3F34015C3F380133780258036
:109DB0000B801080F8BD4FF6FF7398423FF4AAAABB
:109DC00028283FF4F1AB17287FF6A4AA19287FF6BC
:109DD0000DAB1B287FF62AAB1C283FF43FAB1E2897
:109DE0007FF644AB1F283FF449AB20283FF462AB19
:109DF00021283FF46BAB22283FF470AB23283FF4BB
:109E000079AB24283FF4AAAB25283FF4AFAB262832
:109E10003FF4B0AB27287FF4C3ABFFF7B3BB0A21F5
:109E20008820FFF745FA0A2312E711218620FFF761
:109E30003FFA112304E70E218420FFF739FA0E239D
:109E4000F6E613218220FFF733FA1323E7E61F21FA
:109E50008020FFF72DFA1F23D8E60A217E20FFF786
:109E600027FA0A23CAE611217C20FFF721FA1123E1
:109E7000BCE60E217A20FFF71BFA0E23AEE6132173
:109E80007820FFF715FA13239FE61F217620FFF7AE
:109E90000FFA1F2390E600219620FFF709FA00230E
:109EA00072E600218C20FFF703FA002349E6002127
:109EB0008A20FFF7FDF900233AE600217420FFF71E
:109EC000F7F900232BE600217220FFF7F1F90023B8
:109ED0001CE600217020FFF7EBF900230DE60021BE
:109EE0006E20FFF7E5F90023FEE500216C20FFF767
:109EF000DFF90023EFE57F216A20FFF7D9F97F23FF
:109F0000E0E50B216820FFF7D3F90B23D1E5002111
:109F10006620FFF7CDF90023C2E500216020FFF79E
:109F2000C7F9002397E500215820FFF7C1F9002366
:109F30005BE502215220FFF7BBF9022330E50A213D
:109F40004C20FFF7B5F90A23C8E411214A20FFF796
:109F5000AFF91123BAE40E214820FFF7A9F90E2327
:109F6000ACE413214620FFF7A3F913239DE41F213E
:109F70004420FFF79DF91F238EE400214020FFF7C6
:109F800097F900237BE400213E20FFF791F900239D
:109F90006DE400213C20FFF78BF900235FE40021F2
:109FA0003A20FFF785F9002351E400213820FFF71C
:109FB0007FF9002343E400213620FFF779F90023DD
:109FC00035E400213420FFF773F9002326E40C2147
:109FD0003220FFF76DF90C2317E400213020FFF742
:109FE00067F9002308E414212E20FFF761F91423F8
:109FF000FFF7F9BB04212C20FFF75AF90423FFF7E0
:10A00000E9BB03212820FFF753F90323FFF7C8BB5F
:10A0100001212620FFF74CF90123FFF7B8BB1421DB
:10A020002020FFF745F91423FFF782BB04211E20EF
:10A03000FFF73EF90423FFF772BB01211C20FFF755
:10A0400037F90123FFF762BB01211A20FFF730F92E
:10A050000123FFF752BB02211820FFF729F9022341
:10A06000FFF742BB00211620FFF722F90023FFF77C
:10A0700032BB02211220FFF71BF90223FFF715BBA9
:10A080000C210E20FFF714F90C23FFF7F6BA4FF45A
:10A090007A610420FFF70CF94FF47A63FFF796BA60
:10A0A0004FF4AF610220FFF703F94FF4AF63FFF7FE
:10A0B00083BA00BFDC9CFF1F8C9CFF1FC69CFF1F48
:10A0C000D49DFF1FE69DFF1F4A9EFF1FFA9DFF1FA5
:10A0D0005C9EFF1F369EFF1FF8B5B92006F0C8FB37
:10A0E000204B214A054603CB1368C5F803001A0C20
:10A0F000A820C5F807102B80AA70FFF7A5F82E46F8
:10A10000002426F80B0FA0B2FFF7ECF8FFF79CF83D
:10A110000234A82C26F8020FF5D16C1E05F1B40606
:10A120004FF0FF3014F8013F082758400F4B40F321
:10A1300000017A1E0B4012F0FF0783EA5000F5D1B0
:10A14000B442EFD1C043FFF791F83A46C5F8B500E5
:10A15000B921284604F0C4FC2846BDE8F84006F0C2
:10A160008FBB00BF14320100103201002083B8ED14
:10A17000F0B50E4B0E4C054693E8070085B02468F9
:10A180002E88AD7801AB83E80700270C1846002223
:10A190000B21ADF804408DF80670ADF80C608DF819
:10A1A0000E5004F09DFC05B0F0BD00BF2032010050
:10A1B00010320100F0B5124B124D1E68124F0FCD38
:10A1C00087B06C460FC495E8030044F8040B386868
:10A1D0003B79CDF80D00320C282021808DF802202B
:10A1E0008DF81130ADF80060FFF72EF80022ADF8C1
:10A1F0000B001221684604F073FC07B0F0BD00BFED
:10A20000103201002C320100342B0100002004F038
:10A21000E3BC00BF02F02EBE70B5124C82B0002528
:10A22000402306462946204600930195802320229C
:10A2300001F072FE20222946204602F031FA204623
:10A24000012102F037FA304607F09AF8314602460B
:10A25000204602F0BFFB204602B0BDE8704001F08E
:10A2600041BC00BFF89EFF1FF0B5B82983B075D977
:10A270000546441E00F1B4064FF0FF3014F8012FDC
:10A2800008275040404A40F300017B1E0A4013F06B
:10A29000FF0782EA5000F5D1B442EFD1C043FEF788
:10A2A000E5FF0146D5F8B5000190019A914202D030
:10A2B000B2F17F2F0BD105F10B00FEF7CDFFA828DF
:10A2C0000BD03248FFF7A8FF002003B0F0BD3048A4
:10A2D000FFF7A2FF384603B0F0BD05F10D00FEF711
:10A2E000BBFF282840D1002440F6AC5613E00428D8
:10A2F0001AD0062821D008281FD00A2828D00C28D8
:10A3000022D1A1F5FA7292B2B24201D8FEF7D0FF83
:10A310000234A82C0ED004F10D002844FEF79CFF57
:10A32000022C0146A0B2E2D1B1F5805FEED3023437
:10A33000A82CF0D1012003B0F0BDA1F52F7292B28C
:10A34000B2F57A6FE4D8E1E7222801D0242811D1B0
:10A35000A1F5FA7292B2B242DAD8D7E70D48FFF708
:10A360005BFF002003B0F0BD0B48FFF755FF002056
:10A3700003B0F0BD2A28C9D1A1F1320292B2B2F5E0
:10A38000967FC5D8C2E700BF2083B8ED70320100C8
:10A390005C320100443201008432010003290CD9EF
:10A3A00070B5461C82B005460C46304603222A4949
:10A3B00007F054F810B102B070BD70470B2C05D9EE
:10A3C00005222649281D07F049F840B12448FFF727
:10A3D00023FF244802B0BDE87040FFF7C9BE05F175
:10A3E0000901032201A807F089F801A803221E49E8
:10A3F00007F034F8D8B103221C4901A807F02EF861
:10A4000008B301A803221A4907F028F8B0B919487F
:10A41000FFF702FFA11E89B23046FFF725FF002893
:10A42000C9D0154802B0BDE87040FFF7F5BE13482B
:10A43000FFF7F2FEFFF750FE1148F3E71148FFF770
:10A44000EBFE1148C6E71148FFF7E6FE02B0BDE893
:10A450007040FFF7AFBE00BF103201009C32010018
:10A46000A4320100B8320100BC320100E432010024
:10A47000FC3201000033010014330100C03201003E
:10A48000D4320100283301003C330100E8320100DE
:10A490002DE9F043174D2B6883B081460F46904657
:10A4A000F3B1154E34880A1992B21846114632801B
:10A4B00006F05CFD28603A464946204402F06CFDF7
:10A4C000B8F1000F09D031882868FFF767FF2868C6
:10A4D00006F0D6F900232B60338003B0BDE8F0838B
:10A4E000054E01930846318006F0C2F9019B2860B1
:10A4F0001C46E0E7849FFF1F809FFF1F10B51F4C85
:10A500004FF4FA70FBF7E6FF204601F0DFF9002276
:10A510001146204602F0C4F82046012102F0CAF894
:10A520002046002102F0C0F80B221549204602F017
:10A5300051FA204602F064FA0F221249204602F036
:10A5400049FA204602F05CFA0F490722204602F041
:10A5500041FA204602F054FA204601F0C3FA0B4BB0
:10A560000B4A1A604FF4FA70FBF7B4FFFFF722FEB4
:10A570000848BDE81040FFF74FBE00BFF89EFF1F20
:10A58000403301004C3301005C3301003CA1FF1F4C
:10A5900091A40000643301000020704790F8392036
:10A5A00090F83800101A704790F8383090F8392039
:10A5B0009A4205D95A1C034480F83820187E704707
:10A5C0004FF0FF30704700BF90F8383090F83920D6
:10A5D0009A4286BF1B18187E4FF0FF30704700BFAD
:10A5E000704700BF38B50546B0F85E0090B195F8E9
:10A5F0005D301446C3F1210294420CD805F13B00B2
:10A600001844224602F0C8FC95F85D30234485F8D2
:10A610005D30204638BD012014462871EEE700BFAA
:10A62000B0F85E306BB190F85D30202B07D8C218BF
:10A63000013380F85D30012082F83B107047012320
:10A6400003710020704700BF0023426980F8383052
:10A6500080F8393080F85C3080F85D3080F85E300A
:10A6600080F85F3006CA30B40D68046943662A4337
:10A6700083660A60A370426990F8613016491468D5
:10A6800013441D7A5B7B01EBC5051B026D6803F467
:10A69000E06343F064032B6090F8623013449D7CC8
:10A6A000DB7D01EBC5011B02496803F4E06343F065
:10A6B00064030B6021685368194205D0036927229F
:10A6C0005A70036904229A71036920225A7103693E
:10A6D00080229A7030BC7047983E010043690CCBD1
:10A6E00012681A420CD0094B99420AD9084B994278
:10A6F000036994BF1A220D225A70036904229A71C9
:10A700007047036927225A70F7E700BF7F1A0600D7
:10A710003F420F0010B50269D378DBB2D906044678
:10A720003DD510215806D17038D503F0040303F04D
:10A73000FF02002B51D03D49626E00230B7084F85C
:10A740005D30002A5BD0904794F85D30002B56D0E6
:10A750002369D0229A70236994F83B201A712369E7
:10A76000012284F85C200222DA7010BD304B84F89C
:10A7700060009C424AD02F4B9C4252D094F8391032
:10A7800013791F29DBB207D82848007820B1601858
:10A79000013184F8391003760223D37010BD5906B5
:10A7A000C3D4917801F0100101F0FF000029DDD041
:10A7B00013F001031ED194F85C1094F85D008842F8
:10A7C00081BF4B1C091984F85C3091F83B30137140
:10A7D0002369D0229A702269DEE7236984F8392040
:10A7E000C0229A702369114A19790121117002223D
:10A7F000DA7010BDC023937022691379CCE701226F
:10A80000002384F85D2084F83B30A1E7626994F866
:10A810006130094913440322187A02F043FD22698A
:10A82000ACE7626994F861300449F3E7889FFF1F41
:10A83000F890FF1F6491FF1F9DA80000A9A80000C9
:10A840000369DB7803F0200373B190F860300133C3
:10A85000DBB2012B80F860301AD9426990F8613080
:10A860001344187A02F09ABD70B5426903F0FF05EF
:10A8700090F8613013440446187A02F08FFDA36EFD
:10A880005BB184F8385094F83900BDE8704018473F
:10A8900090F85F30002BE0D0704770BD0148FFF7A3
:10A8A000CFBF00BFF890FF1F0148FFF7C9BF00BF2F
:10A8B0006491FF1F2DE9F047374FDFF8E0903B68C8
:10A8C000026982B006460093DDF800800021A025D1
:10A8D000D3789B065BD53B680193019BC8EB0303D0
:10A8E0000F2BF5D949B1102BF2D0002090703369AD
:10A8F00080229A7002B0BDE8F087726996F86130E4
:10A9000013440521187A02F043FF726996F861300A
:10A910001344012193F812A0504602F039FF092494
:10A920000021504602F020FF2B46013BFDD10121C2
:10A93000504602F019FF2B46013BFDD1013CEFD1FF
:10A94000706996F8611001444FF4A0720C7A4B7B49
:10A9500009EBC4011B02496803F4E06343F064039C
:10A960000B6096F862300344997CDB7D09EBC101F2
:10A970001B02496803F4E06343F064030B60013A8F
:10A98000FDD13269D3789B064FF00101A3D4012099
:10A9900002B0BDE8F08700BFB09FFF1F983E0100E6
:10A9A000F0B503691222DA700269937803F020038C
:10A9B00085B004460D46002B5ED0B42393703C490D
:10A9C00022690B680093009E05E00B680193019BD0
:10A9D0009B1B042B42D8D37803F0200303F0FF0025
:10A9E000002BF2D094F85D30002B31D04FF0000EE8
:10A9F0004FF0020C04EB0E0393F83B3013710B681D
:10AA00000393039F206907E09B060DD50B68029313
:10AA1000029BDB1B052B28D8C378DBB203F00202B4
:10AA200002F0FF06002AEFD080F803C02669F37811
:10AA3000DBB2DF0632462DD49F062BD5DB0731D49F
:10AA40000EF1010E94F85D305FFA8EFE7345D1D899
:10AA500000201DBB002384F85E3004E09070236961
:10AA600080229A70042005B0F0BD86702369802290
:10AA700004209A7005B0F0BD03F0FF06FFF71AFF3F
:10AA800010B9042005B0F0BD236984F85F60B022DE
:10AA90009A7094E78023B3700420DAE72669802354
:10AAA000B370D7E7BEF1000F0CBF02200320F6E71A
:10AAB000B09FFF1F2DE9F04106690025122780F89D
:10AAC000385080F83950F770D0F810C09CF802E088
:10AAD0000EF0200E88B00446884615461E46BEF18C
:10AAE000000F49D0B4238CF80230784B21691A68E2
:10AAF0000092DDF800E006E01A6801920198CEEBC2
:10AB00000000042830D8C87800F0200000F0FF07CB
:10AB10000028F1D04FEA480242F00102D2B20A7195
:10AB20001A680292DDF808E0206906E01A680392CC
:10AB30000399CEEB010105292AD8C17801F0020161
:10AB400001F0FF070029F1D04FF0020C80F803C09C
:10AB50002269D17811F0110722D12DBB002E0CBF34
:10AB6000A0238023937003E08F70236980229A7062
:10AB7000384608B0BDE8F0810EF0FF07FFF79AFEF7
:10AB80000028F5D0236984F85F70B0229A70ACE792
:10AB900087702369802238469A7008B0BDE8F0813A
:10ABA000802393700027E3E7012D75D0A0219170D9
:10ABB00021690A79BE4667464FF0A80C1A680492CC
:10ABC000049805E01A680592059A121A052A4AD8CF
:10ABD000CA7802F0020202F0FF08002AF2D0CF7019
:10ABE0002169CA78D2B212F0100F08465AD19206E3
:10ABF00058D5013DEDB2012D49D0BEF11F0F3BD913
:10AC00000A79012DDAD11A680692069D05E01A68C4
:10AC10000792079A521B052A46D8C27802F0020210
:10AC200002F0FF01002AF2D00223C3702269D37818
:10AC3000DBB2D9063AD49B0634D5B023BEF11F0F40
:10AC400093703FD8226904EB0E0312791A760EF145
:10AC5000010E5FFA8EFE16B1236980229A7084F885
:10AC600039E0774684E781F80280236980229A7070
:10AC7000774684F839E07BE704EB0E0291F8048014
:10AC800082F818800EF1010E5FFA8EFEB9E781F8A6
:10AC900002C021690846B0E7A82191702069BE462C
:10ACA0000279B0E7774663E78170DEE71021A023E1
:10ACB000D170013BFDD12269937803F0F703774609
:10ACC000937055E723691B79C5E700BFB09FFF1F4D
:10ACD0000148FFF71FBD00BFF890FF1F0148FFF7B5
:10ACE00019BD00BF6491FF1F704700BF38B5144CF9
:10ACF000037801225B000546204684F83B3084F847
:10AD00005E2084F85D20FFF78BFC20460021FFF7D2
:10AD100047FE0B4C2978012320461A46FFF7CAFE4E
:10AD20000128F6D194F8383094F839209A4205D9A0
:10AD3000E218013384F83830107E38BDFF2038BD6A
:10AD4000F890FF1F38B51B4C037801225B000546C5
:10AD5000204684F83B3084F85E2084F85D20FFF7BD
:10AD60005FFC20460021FFF71BFE124C297820468D
:10AD700001230222FFF79EFE0228F6D194F8382024
:10AD800094F839108A420FD2531CDBB2A0189942B2
:10AD900084F83830007E0AD9234402321B7E84F8BE
:10ADA000382040EA032038BD4FF6FF7038BD40F42C
:10ADB0007F4038BDF890FF1F0C2901D90020704753
:10ADC0000231490001F0FE01FFF7BCBF70B50C4C29
:10ADD0000378164601255B00204684F83B3084F852
:10ADE0005E5084F85D50FFF71BFC31462046FFF7AC
:10ADF00017FC29462046BDE87040FFF7D1BD00BFD3
:10AE0000F890FF1FF8B505460F4616464124214627
:10AE10003A462846FFF7DAFF611C0234C9B23246CF
:10AE20002846E4B2FFF7D2FF592CF0D1F8BD00BF9D
:10AE300038B504460D463548FFF706FC63228021ED
:10AE400020462570FFF7C2FF012002F0C9FC204612
:10AE500000225E21FFF7BAFF20465D21FFF746FF83
:10AE6000242801D0002038BD204606220C21FFF7FF
:10AE7000C9FF204601222B21FFF7A8FF204601220F
:10AE80002C21FFF7A3FF20460E222D21FFF79EFF66
:10AE9000204600222E21FFF799FF204601222F2174
:10AEA000FFF794FF204605223021FFF78FFF204651
:10AEB00001223121FFF78AFF204600223221FFF7CD
:10AEC00085FF204600223321FFF780FF2046002225
:10AED0003421FFF77BFF204600223521FFF776FF64
:10AEE000204600225B21FFF771FF204610225C21E3
:10AEF000FFF76CFF204620225D21FFF767FF204609
:10AF00008F225E21FFF762FF012038BDF890FF1FFE
:10AF100010B4047F4160022CC26002D010BC01F06A
:10AF2000D7BB836810BC184790E80C00F0B41C68CD
:10AF300059682568164F174E29432160164D174949
:10AF40001760D66015611160417A154A5C180A31A4
:10AF500094F8244053F8215002EBC40149680D6075
:10AF6000017A5C1803EB8101247ECD6902EBC401F8
:10AF700049680D60817A581803EB810390F830001E
:10AF8000596B02EBC002F0BC53681960704700BFF8
:10AF900001401F00011000380110007800001F80E0
:10AFA000983E0100704700BFF0B50C1EBDF814605C
:10AFB00034DBB0F906701919B942C4BF3B1B1BB290
:10AFC000002BA6461CDD002A1146B8BFD11D02F099
:10AFD0000705CC10826A012007FB04E1A840012E7E
:10AFE0000A44C0B21ED00CD3022E09D1013B12FA82
:10AFF00083F3013A12F8011F41409A421170F9D1CE
:10B00000F0BDC043013B12FA83F3C0B2013A12F81B
:10B01000011F014093421170F9D1F0BD23441BB2CE
:10B020000024C6E7013B12FA83F3013A12F8011F2C
:10B0300001439A421170F9D1F0BD00BFF8B50D1E61
:10B040000EDB14461F46064601F03AFBA84207DD18
:10B05000002C05DB304601F037FBA04201DCF8BDD7
:10B06000F8BD304601F02AFB022853D003284BD00C
:10B07000012806D16540F3886C406540013B5D1BAB
:10B080002DB2012F03D02AD3022F14D0F8BD002CEB
:10B090002246B6F90630B06AB8BFE21D42F3CF02CD
:10B0A00002FB035504F00704435D012101FA04F497
:10B0B0001C434455F8BD002C2246B6F90630B06A50
:10B0C000B8BFE21D42F3CF0202FB035504F00704B0
:10B0D000435D012101FA04F45C404455F8BD002CA5
:10B0E0002246B6F90630B06AB8BFE21D42F3CF027D
:10B0F00002FB035504F00704435D012101FA04F447
:10B1000023EA04044455F8BD3389013B591B254605
:10B110000CB2B6E7F18832890139013A4D1B141B94
:10B120002DB224B2ADE700BF2DE9F041079E9DF995
:10B130001880089D04461F4600F0C0FF0D4B0E48C6
:10B140000E4984F83380FF22002F08BF1F4684F881
:10B150002F20002384F8302084F8312084F8322016
:10B160002060A665E565676261652362A36220468B
:10B17000BDE8F081F890FF1FF033010001100138A5
:10B1800010B50446806A034B236008B105F078FBD4
:10B19000204610BDF0330100F8B5436ADBB190F8EA
:10B1A0002C200125AA4083F83B2083F85E5083F8C9
:10B1B0005D500446406A03680E461B6800219847AC
:10B1C000606A036831461B6898472946606ABDE893
:10B1D000F840FFF7E5BBC26BC56C1368046A23EA4D
:10B1E000050313604CB122684FF00043D3625163F2
:10B1F000D36A002BFCDA936BF8BD836B466B082592
:10B20000802410E03768426C3A4332601F68826CD9
:10B210003A431A601A68876C013D22EA07024FEA36
:10B2200054041A6007D02142ECD13268476C22EAFC
:10B2300007023260EAE7F8BD70B50446406A0D4681
:10B2400000282BD0A16DFFF749FA002D20460CBF36
:10B25000A621A721FFF7A0FF606A20B1E16DBDE83C
:10B260007040FFF73BBA216C226D0868236A0243E5
:10B270000A6093B1DA7A82B1D00703D5224A99697C
:10B280001160DA7A910703D5204AD9691160DA7A18
:10B29000520702D51E4A1B6A136070BD236A002B39
:10B2A0002BD0D97A626DE1B172B6D97ACE0706D5C4
:10B2B0001848D9680668314099610160D97A8807D1
:10B2C00006D51548196906683140D9610160D97AF7
:10B2D0004E0705D511485969066831401962016069
:10B2E00062B61B68D968914207D00D4818600D49B5
:10B2F000DA6042F0804018611960226C216D136899
:10B3000023EA01031360A0E700E100E004E100E0AC
:10B3100008E100E080E100E084E100E088E100E095
:10B3200001403F0000003F80436A2DE9F04105469F
:10B330000E469046002B3ED090F82C100124A140E0
:10B3400083F83B1083F85E4083F85D40406A0368F1
:10B3500000211B6808F1FF379847FFB2B8F1000FD2
:10B3600023D03744A046013E686A16F8011F0368DF
:10B370001B6898470134B742E4B216D0202CF3D1B1
:10B380000121686AFFF70CFB95F82C206B6A5200CC
:10B3900083F83B2083F85E8083F85D80686A0368E9
:10B3A00000211B6898470124DEE7686A0121BDE897
:10B3B000F041FFF7F5BAC26BC16C136823EA0103D1
:10B3C00006EB080413604FF00048A6420ED02B6A2B
:10B3D00016F801EB63B11A68C2F82C80C2F834E0A9
:10B3E000D36A002BFCDAA642936BF0D1BDE8F08162
:10B3F000AB6BD5F834C008208021DCF800206F6CDE
:10B400001EEA010F14BF3A43BA43CCF800201A6871
:10B41000AF6C3A431A601A68AF6C013822EA07022F
:10B420004FEA51011A60E8D1CFE700BF70B504467A
:10B43000406A0D46002828D0A16DFFF74FF920463D
:10B440002946FFF7A9FE606A20B1E16DBDE87040B2
:10B45000FFF744B9216C226D0868236A02430A6031
:10B4600093B1DA7A82B1D00703D5234A9969116082
:10B47000DA7A910703D5214AD9691160DA7A52073D
:10B4800002D51F4A1B6A136070BD236A002B2BD0A4
:10B49000D97A626DE1B172B6D97ACE0706D519486C
:10B4A000D9680668314099610160D97A880706D564
:10B4B0001548196906683140D9610160D97A4E078B
:10B4C00005D512485969066831401962016062B6B3
:10B4D0001B68D968914207D00D4818600D49DA60A1
:10B4E00042F0804018611960226C216D136823EAD4
:10B4F00001031360A3E700BF00E100E004E100E006
:10B5000008E100E080E100E084E100E088E100E0A3
:10B5100001403F0000003F802DE9F041044686B025
:10B52000806A9DF830801E460F461546B4F90830F3
:10B53000002800F04281DA1D48BF03F10E02B4F981
:10B540000630D21003FB02F2002105F0BDFCB4F975
:10B550000820202A00F39280B4F90610A34B0120A2
:10B56000203A733902EBD27201EBD1714FF0200E09
:10B57000029073208DE8014042F34F0241F34F01E6
:10B58000204600F051FE606A84F82D70002800F01B
:10B590004D81002D40F08A80B4F90830202B14BF73
:10B5A0003D253C2584F82C50B8F1000F40F08580F3
:10B5B00006B394F93300002818DBC0B2012102F071
:10B5C000E7F8012194F8330002F0CEF8012002F0F0
:10B5D00007F9002194F8330002F0C6F80A2002F0BF
:10B5E000FFF8012194F8330002F0BEF8606A0028E9
:10B5F00000F08280A16DFFF771F804227C4920469B
:10B60000FFF792FE217A0139C9B22046FFF7C4FD47
:10B61000784904222046FFF787FE94F92D30012B4C
:10B6200014BF142110212046FFF7B6FD04227249F1
:10B630002046FFF779FEB4F90630802B00F09280A7
:10B64000602B00F0A680D9212046FFF7A5FD94F9D4
:10B650002D30012B14BFF12122212046FFF79CFD44
:10B66000204606226549FFF75FFE606A50B3E16D30
:10B67000FFF734F8012006B0BDE8F081B4F90610F8
:10B680005F4B0120403A52394FF0400E029002EBDE
:10B69000D272522001EBD1718DE8014042F34F028A
:10B6A00041F34F01204600F0BFFD6CE76DB284F816
:10B6B0002C50B8F1000F3FF47BAFFEF7C5FF002E12
:10B6C00094D076E7216C226D0868236A02430A60F1
:10B6D00073B1DA7A62B1D00703D54A4A9969116029
:10B6E000DA7A91077CD4520702D5474A1B6A136065
:10B6F000012006B0BDE8F081236A002B2BD0D97A57
:10B70000626DE1B172B6D97ACF0706D53F48D968E4
:10B710000568294099610160D97A8E0706D53C48B1
:10B72000196905682940D9610160D97A4D0705D5A5
:10B7300038485969056829401962016062B61B687A
:10B74000D968914207D0344818603449DA6042F031
:10B75000804018611960226C216D136823EA01038F
:10B7600013604AE7B4F90830202B00F08680402BA4
:10B770007FF469AF2A4920460322FFF7D5FD94F9EB
:10B780002D30012B14BFCF219F212046FFF704FD50
:10B7900059E7B4F90830102B7FF455AF2149204602
:10B7A0000322FFF7C1FD94F92D30012B14BFAF2107
:10B7B00010212046FFF7F0FC45E7DA1D48BF03F1F2
:10B7C0000E02B4F90630D21003FB02F210460592C5
:10B7D00005F04EF8A06200283FF44DAF059AB3E69D
:10B7E000114AD9691160DA7A7DE700BF4834010057
:10B7F000283601002C3601003036010034360100B5
:10B800003C36010000E100E008E100E080E100E0FA
:10B8100084E100E088E100E001403F0000003F805B
:10B8200044340100FC38010004E100E0012194F8F7
:10B830003100244F01F0ACFF94F83200012101F0F7
:10B84000A7FF94F9312094F9323057F83220E2639F
:10B8500057F83330206A23640125E56425651A68AA
:10B860002A431A6078B1B8F1000F3FF428AFFFF710
:10B870005BFB002E3FF4BAAE9BE604221249204641
:10B88000FFF752FDDFE6294694F82F0001F080FF14
:10B89000294694F8300001F07BFF94F92F2094F9A9
:10B8A000303057F83220626357F833306564A5644E
:10B8B0001A68A36322F001021A60002E3FF496AECC
:10B8C00077E600BF983E010040340100B0F908203F
:10B8D000D31D48BF02F10E03B0F90620806ADB10C9
:10B8E00002FB03F2002105F0EFBA00BFF0B500291A
:10B8F000BDF814502EDBB0F90660B1422ADA002AF6
:10B9000059DBB0F9087014461C44BC42C4BFBB1AD2
:10B910001BB2002B1EDDD2B2D408D0F828E016FBF3
:10B92000041112F00702DBB20EEB010421D0C2F1C8
:10B930000807FAB2374F9342BF5C0CD2C3EB020C3C
:10B94000FF2646FA0CF6012D07EA06073FD005D37D
:10B95000022D36D0F0BD012D39D030D21EF8016055
:10B9600026EA07070EF801709342F3D3B0F90610E8
:10B970000C449A1AD2B2072A10D9022D36D0002DC3
:10B9800014BFFF26002613462670083BB0F90610A8
:10B99000DBB2072B0C44F7D802F00702002AD9D0FB
:10B9A0001D4B012D9B5C1DD017D3022DD2D12278C7
:10B9B00053402370F0BD13441BB20022A1E7022DB7
:10B9C00025D11EF8016077400EF80170CCE71EF813
:10B9D000016037430EF80170C6E7227822EA0303BC
:10B9E0002370F0BD227813432370F0BD11462378F5
:10B9F000DB4323700839B0F90630C9B207291C446B
:10BA0000F5D812F00702A5D0034B9B5CCFE7344476
:10BA1000AFE700BFE0330100D033010070B4C47D54
:10BA2000BDF80C50022C18D0032C1FD0012C0BD0C9
:10BA3000002A03DBB0F90840944201DC70BC704777
:10BA4000039570BCFFF7B0BAC4880395013CA41AF3
:10BA50000A4621B270BCFFF749BF0689C488013E7F
:10BA6000641AB21AE41A12B221B2E1E7048903950A
:10BA7000E41A641A114622B270BCFFF737BF00BF48
:10BA800070B4C57DBDF80C60022D1AD0032D12D004
:10BA9000012D03D0039670BCFFF728BFC488E41AB9
:10BAA000A41A0A4621B2002A03DBB0F908409442E6
:10BAB00013DC70BC70470489013C641A114622B241
:10BAC000F1E7C48805890396013CAD1AED1A621AA4
:10BAD00011B22AB270BCFFF709BF039670BCFFF722
:10BAE00063BA00BF2DE9F8430446406A002863D0DA
:10BAF000A16DFEF7F3FD052274492046FFF714FC03
:10BB0000A1790139C9B22046FFF746FBB4F90820F4
:10BB1000E588A66AD31D48BF02F10E03DB10626AF6
:10BB200015FB03F51FFA85F8002A7BD094F82C301A
:10BB30000125AB4082F83B3082F85E5082F85D50C0
:10BB4000606A036840211B6808F1FF379847BFB25D
:10BB5000B8F1000F23D03744A846013E606A16F8BA
:10BB6000011F03681B6898470135B742EDB216D034
:10BB7000202DF3D10121606AFEF712FF94F82C20EA
:10BB8000636A520083F83B2083F85E8083F85D800F
:10BB9000606A036840211B6898470125DEE70121A0
:10BBA000606AFEF7FDFE606A002800F08D80E16D9E
:10BBB000BDE8F843FEF792BD236A002B2BD0D97A5B
:10BBC000626DE1B172B6D97ACE0706D54048D96820
:10BBD0000568294099610160D97A8D0706D53D48ED
:10BBE000196905682940D9610160D97A480705D5E6
:10BBF00039485969056829401962016062B61B68B5
:10BC0000D968914207D0354818603549DA6042F06A
:10BC1000804018611960226C216D136823EA0103CA
:10BC2000136068E7E26BE36C1168276A0B4306EB6D
:10BC3000080913604FF0004E4E450DD016F801CBA9
:10BC40002FB33A68C2F82CE0C2F834C0D36A002B94
:10BC5000FCDA4E45936BF1D1226C236D11680B43D6
:10BC6000136097B1FB7A83B1D90703D51D4BBA692D
:10BC70001A60FB7A9A0703D51B4BFA691A60FB7AA4
:10BC80005B0702D5194B3A6A1A60BDE8F883A36BCB
:10BC9000D4F8348008208021D8F80020656C1CEA94
:10BCA000010F14BF2A43AA43C8F800201A68A56CE4
:10BCB0002A431A601A68A56C013822EA05024FEA85
:10BCC00051011A60E8D1B7E7276AC5E7D833010008
:10BCD00080E100E084E100E088E100E001403F0015
:10BCE00000003F8000E100E004E100E008E100E046
:10BCF0002DE9F04F85B09946BDF93870BDF83CA0EC
:10BD0000BB1AC1EB090B002BB8BF5B42BBF1000FA4
:10BD1000B8BFCBF1000B5B450D461646009380463D
:10BD200048DC4D453A4633464CDC194613460A4634
:10BD3000C5EB09019B1A89B2002B0CB2B8BF5B425C
:10BD400004EBD474BE42ACBF4FF0FF3201224D452C
:10BD5000039102924FEA640429DC9BB201930DE047
:10BD6000D8F80070BF69B847019BE41AA3B21CB2AF
:10BD70000135002C2DB211DBA94518DB009B5B457A
:10BD80002A46534631464046EADCD8F8002053465E
:10BD90009769294632464046B847E5E7029A164475
:10BDA000039AA94502EB030436B224B2E6DA05B0E1
:10BDB000BDE8F08F4A462B46B94635464D451746F5
:10BDC0001E46B2DD304629463E464D460746894668
:10BDD000AEE700BF10B404682469A44610BC6047F5
:10BDE00030B40468BDF808500295A46BA44630BC7A
:10BDF000604700BF30B40468BDF808500295E46B9A
:10BE0000A44630BC604700BF70B40468BDF90C6044
:10BE1000BDF8105003960495246CA44670BC60478E
:10BE2000704700BF10B582B0B0F90C2001910168D5
:10BE3000009200220C6CB0F90A301146A04702B003
:10BE400010BD00BF704700BF01F003010129C1759B
:10BE500006D0032904D0C2880389428183817047B8
:10BE60000289C38842818381704700BF2DE9F04178
:10BE70000568134E6F6986B0B7420446BDF830803E
:10BE800010D1013B13441BB20093CDF804800B4644
:10BE9000AD6A2046A8472368DB6AB3420AD106B0E0
:10BEA000BDE8F081059304920391B84703A9256882
:10BEB0000EC9E6E7204606B0BDE8F041184700BFCE
:10BEC00021BE00002DE9F0410568124E6F6986B071
:10BED000B7420446BDF830800FD1013BCDF8048055
:10BEE0000B4400921BB2AD6A2046A8472368DB6A68
:10BEF000B3420AD106B0BDE8F081059304920391E4
:10BF0000B84703A925680EC9E7E7204606B0BDE893
:10BF1000F041184721BE00002DE9F04F0568DFF819
:10BF200058B06F6985B05F450646BDF93890BDF8D9
:10BF30003CA00C46904615D11F19BC420CDACDF836
:10BF400000A0214601342D6A4B464246304624B2B9
:10BF5000A847BC423568F2DBEB6A5B4507D105B008
:10BF6000BDE8F08F0393B8473568039BE4E730469C
:10BF700005B0BDE8F04F184721BE00002DE9F043A1
:10BF800087B099420546BDF93840BDF83C6025D0E0
:10BF9000A24212D00768DFF88080D7F81490C1451C
:10BFA00032D18DE850002846BC6AA0472B68DB6A76
:10BFB000434524D107B0BDE8F083994202DD08462D
:10BFC0001946034628680E96C46B01335B1A1BB2F0
:10BFD0002846A44607B0BDE8F0436047A24202DD10
:10BFE000134622461C4628680E96631C846B9B1AD7
:10BFF0001BB22846A44607B0BDE8F0436047284678
:10C0000007B0BDE8F0431847059304920391C84771
:10C0100003A92F680EC9C4E721BE00002DE9F04F27
:10C02000D0F800E0DFF89090DEF814B083B0CB4594
:10C030000446BDF93080BDF834A00D4617461E46B3
:10C0400031D1CDF800A0DEF824B0294633463A4677
:10C050002046D8472368CDF800A008F1FF323A44C3
:10C06000D3F824B0294612B233462046D847236875
:10C07000CDF800A02946D3F820B03A4643462046E2
:10C08000D8472068CDF800A0711E29444346056AB0
:10C0900009B23A462046A8472368DB6A4B4506D1D9
:10C0A00003B0BDE8F08FD847D4F800E0C9E72046D8
:10C0B00003B0BDE8F04F184721BE0000F0B40024E3
:10C0C00001264FF6FF75094F07600471C475C481DE
:10C0D00004824476C4618675067685824582C18075
:10C0E000028141818281F0BC704700BF08390100A4
:10C0F0002DE9F04F85B00668BDF84450BDF9388091
:10C10000CDF8008004460195D6F848B00392BDF9F9
:10C110003C60BDF9407089469A46D847236801952E
:10C12000009742465146D3F8488020463346C047E0
:10C130002068039B0E930F95856C4B463A4631461B
:10C140002046AC4605B0BDE8F04F60472DE9F04F02
:10C1500087B01746BDF9404000912546E91D05937B
:10C1600044BF2B4603F10E010268BDF848605369D5
:10C170000294C91003912B49BDF9444001968B42AA
:10C18000824645D1002C3CDD029B3C445E1EB6B28B
:10C190004FF0000923B2049301364D46029B002B59
:10C1A00028DD059B002403EB090806E0EDB22B0611
:10C1B00004F1010411D4A6421CD0A1B211F0070F62
:10C1C00023B24FEA4505F1D1002BB8BF0733DB108E
:10C1D000013418F803502B06EDD5009BD2F818B0A7
:10C1E00019443A4609B2019B5046D847A642DAF8AC
:10C1F0000020E2D1039B01379944049B3FB2BB422C
:10C20000CCD1D36A074A934206D107B0BDE8F08F7C
:10C210009847DAF80020B5E7504607B0BDE8F04F80
:10C22000184700BF21BE000070B4BDF90C60BDF915
:10C230001050BDF8144003960495059470BCFFF7A8
:10C2400085BF00BF2DE9F04F93B090460591C169BD
:10C250001090BDF870000790BDF874909DF878A01C
:10C260000493002900F0CD800A7A0AC9894604990E
:10C270008A1AD2B203EBC203BAF1010FDA780B9239
:10C2800093F905201E8893F802B00F9293F90640A7
:10C2900079D913B2099323B20C93109B1A68A94B56
:10C2A0001193194653698B4240F0A6800B9B002BDB
:10C2B00055D01FFA88F300210D93C8462344DDF8BA
:10C2C000409006910E930F460C46BBF1000F3FD0F5
:10C2D000BDF818100C9B03971FFA8AF0CB1813FBBC
:10C2E00000F304900E9801440D98034409B21BB268
:10C2F0000A910893002505E00135EBB264009B45E7
:10C30000E4B222D9039B2B44590703D1731C18F8BC
:10C3100006409EB22306EFD5099BBDF81000E91830
:10C3200011FB00F10598BAF1010F0FFA8AF30144ED
:10C330001CD0079801900093D26909B2174648466D
:10C34000089AB847D9F80020D6E7039F5F44FFB2A8
:10C35000069B0B9901330693DBB29942B5D8D36A99
:10C36000119A934243D113B0BDE8F08F0F9B191877
:10C3700093690A9A29441F4609B2079B4846B84761
:10C38000D9F80020B8E700230C93099385E70A9AAF
:10C390000D9B0132013B52B213F0FF030A920D9341
:10C3A0006FD1DDF81890079BDDF83C80DDF820A008
:10C3B0004B4517D0BAF1010F00F0C8800B9A109DC1
:10C3C000CDF804900BEB8B014FEACB030A440093AA
:10C3D0001146DEF81C405346424609B22846A047A3
:10C3E000D5F800E0DEF82C30119A9342BBD01098BB
:10C3F00013B0BDE8F04F1847109D284698472A68AB
:10C4000054E7109A0598B2F90A308342ABDDB2F9CD
:10C410000C304345A7DD062313FB0A03002BA2DDE6
:10C4200008EBCA03002B9EDD537E2BB9049BAF2B78
:10C4300002D90133DBB20493109BD3F800E0414BE7
:10C4400011931A46DEF81430934240F08E801FFAA2
:10C4500088F30E9308339BB2BDF81420059305238F
:10C460000D9300230A93CDF83C800FFA8AF3DDF890
:10C470004080CDF818900B921FFA8AFBCDF820A0CF
:10C4800099460A9ABDF810000B9C0E9D052319468B
:10C4900011FB00232C481146C75C039702FB0B429B
:10C4A00014FA81F312B21BB209920C932C462E4659
:10C4B0001CE0089B0999012B2AB24B4640462DD01F
:10C4C000079F0197CDF80090DEF81CA0D047D8F860
:10C4D00000E0039B5B0801340393059BA4B25D4419
:10C4E0005E44A342ADB2B6B23FF451AF039BD8074E
:10C4F000DFD4079B069A9342EBD0089B012B16D002
:10C50000069B0193CDF80090DEF81CA009994B46DC
:10C5100032B24046D047D8F800E0DAE7DEF818A09B
:10C52000079B0C9922B2D047D8F800E0D1E7DEF89B
:10C5300018A00C991346404622B2D047D8F800E024
:10C54000C7E700BF21BE0000583901000B99109DBC
:10C55000CDF800900531DEF8204009B242460823AC
:10C560002846A047D5F800E03CE7109C20469847B5
:10C57000D4F800E06BE700BFF0B5C36985B00446AE
:10C580002BB30A2968D00D294AD01A7A914247D391
:10C59000587A884244D35D688A1A05EBC205AA78A6
:10C5A000002A50D0E87800284DD0207E00283AD0CC
:10C5B00095F905E0B4F90E00A67DB4F90A7072444D
:10C5C00006FB0202BA4262DCB4F9102030E00A290C
:10C5D00056D00D2924D0027E002A4BD0B0F90E008F
:10C5E000A57DB4F90A60062212FB0502B2423EDDC7
:10C5F000228AE38102EBC50212B218462282A78A80
:10C60000668A02950B468DE8C00001462046FFF77A
:10C6100019FEA37DE28903EB430302EB4303E381AD
:10C62000012005B0F0BDA67DB4F90E00B4F91020CC
:10C63000B4F814E0678A02960B468DE88040014604
:10C640002046FFF7FFFD2979E389A27D012001FB48
:10C650000233E38105B0F0BD0022C2819A7A817D68
:10C66000038A01FB02330382012005B0F0BDB4F957
:10C670001020C4E7857DB4F91020B0F90E00BEE7A4
:10C68000028A817DC38102EBC1030382C8E70020D7
:10C69000E0819B7A228A03FB062212B22282C7E73C
:10C6A000C1810282704700BF002908BF0121817546
:10C6B000704700BF81824182704700BFC07D7047D4
:10C6C000B0F90A00704700BFB0F90C00704700BF16
:10C6D00010B4EFF3108272B6437F33B9017F0129A2
:10C6E00007D003290FD00123437702B962B610BCEB
:10C6F0007047124C2168A1B1114943610B688361F5
:10C7000008605861EFE70F4C216881B10E49436121
:10C710000B688361086058610C4B4FF080511960C1
:10C72000E1E7074B4161816120601860DBE7064B60
:10C730004161816120601860EEE700BF9C9FFF1F90
:10C74000989FFF1F8C9FFF1F909FFF1F04ED00E02D
:10C7500070B5EFF3108272B60C4C206880B10C4EAD
:10C7600000254369236073B19D6102B962B64577C4
:10C7700083689847EFF3108272B620680028F0D1E2
:10C7800002B962B670BD3360EFE700BF8C9FFF1F38
:10C79000909FFF1FFFF7DCBF184A30B41468002CCD
:10C7A00027D0036821688B420ED2CB1A0021846007
:10C7B000C1602360E06010600223037530BC7047E5
:10C7C00011688B42144608D3A2685B1A0360002AE2
:10C7D000F6D18260C460A060EEE7D268C260846077
:10C7E000E060C568CB1A0222A8602360027530BCE5
:10C7F00070478460C4601060DEE700BF949FFF1F35
:10C80000F8B5224E34682CB32368002B3AD1204F60
:10C810001D4604E03468ECB12368002B32D1A368D4
:10C8200003B1DD6020693360036825751B68BB4276
:10C8300021D1037F4560022BC46020D0FFF748FF61
:10C840006368002BE6D023602046FFF7A5FF34681D
:10C85000002CE1D1EFF3108372B60E4A002110686C
:10C86000116003B962B628B18468FFF795FF2046CE
:10C870000028F9D1F8BD224600219847E0E78368F7
:10C880009847DDE7013B2360E4E700BF949FFF1F6B
:10C8900011AF0000A49FFF1F024A13680133136009
:10C8A000FFF7AEBFB09FFF1F704700BF0368F0B433
:10C8B000FBB1002501249D60DC601B4C1A601C4408
:10C8C000241104F144056A11032692009E60174F5B
:10C8D0000679174B47F8241002F1604202F56142D5
:10C8E00005F01F05012000FA05F5E6541560F0BCBF
:10C8F0007047104C236843F40003236000BF0E4BC5
:10C900000E4DA4F58734A4F59E7401261E602346BF
:10C9100004609C68002CD0D01033AB420360F8D187
:10C92000002303601846E2E7008FFCBFD091FF1F91
:10C9300044E400E03C800440007003404071034048
:10C940000168A9B10B4BF0B40B441B110A4E0B4FFD
:10C950000B4D46F8237003F1440202F01F0401233B
:10C960005211A340002445F822308C600460F0BCD2
:10C97000704700BF008FFCBFD091FF1FA9C8000007
:10C9800080E100E0024A034B012111601B68184757
:10C990000C710340D091FF1F024A034B012111602B
:10C9A0005B6818471C710340D091FF1F024A034B7C
:10C9B000012111609B6818472C710340D091FF1F23
:10C9C000024A034B01211160DB6818473C710340A8
:10C9D000D091FF1FF8B50E4671B17AB107461446E3
:10C9E00000253B6816F8011B1B6838469847013C38
:10C9F0000544F6D12846F8BD0846F8BD1046F8BDF6
:10CA000000B5064A036812885B6883B001A9ADF8D7
:10CA100004200222984703B05DF804FB583E010051
:10CA2000F0B507468BB0002A33D0012A08BF0A228E
:10CA300051B3212400E0F4B2B1FBF2F502FB151171
:10CA4000C8B2092900F1300198BFC8B20AA988BF4D
:10CA50003730214488BFC0B201F8240C661E294635
:10CA6000002DE8D133B1013CE4B20AAB23442D22BE
:10CA700003F8242C3B6801AA11195B683846C4F1FD
:10CA8000220298470BB0F0BD30228DF825202124DA
:10CA9000E8E70368C9B21B6898470BB0F0BD00BF58
:10CAA0000029BABF49422D2300230A22FFF7B8BF4D
:10CAB000374A384913681B06FCD40B6813F080030F
:10CAC000F8D172B634490A78002A5FD0334A344824
:10CAD000F0B4344C176806682568D4680C303E44BE
:10CAE000143200681268304F35442C44204402440C
:10CAF000C2F34E022D4E2E482E4D2F4C42F40042D2
:10CB00003A60376806682D682C4A24680C303E4429
:10CB1000006812682A4F35442C4420440244C2F372
:10CB20004E02284E2848294D294C42F400423A60D2
:10CB3000376806682D68274A24680C303E44006830
:10CB40001268254F35442C4420440244C2F34E025F
:10CB5000224E2348234D244C42F400423A60376869
:10CB600006682D68214A24680C303E44006812682B
:10CB700035442C4420440244C2F34E021C4842F483
:10CB8000004202600B7062B6F0BC704762B670473C
:10CB900024B0034024B00B40A99FFF1F38B00340CE
:10CBA0003CB0034040B003402CB0034058B00340B9
:10CBB0005CB0034060B0034064B003406CB003401D
:10CBC00030B0034038B00B403CB00B4040B00B409D
:10CBD00044B00B404CB00B402CB00B4058B00B4055
:10CBE0005CB00B4060B00B4064B00B406CB00B40CD
:10CBF00030B00B4030B42948294A2A4B2A4D6024D2
:10CC0000E121047011701B78284C082B30D00A2BBE
:10CC10002748284937D00C2B0CBF35223D22122340
:10CC20002A60236002600B60234B24491B78244A4E
:10CC3000BBB101230B601360224B23491B78234AAD
:10CC4000012B26D9042B0FD9082B1ED9102B94BFEA
:10CC5000862387230B6013601D4B01221A7030BCA2
:10CC600070470B601360E7E784230B601360F3E702
:10CC700000F58E200F490830012213232A6023601B
:10CC800002600B60D0E73922F7E785230B60136061
:10CC9000E2E780230B601360DEE700BF004007403F
:10CCA00001400740E091FF1F08B003400CB0034073
:10CCB00008B00B400CB00B40AC9FFF1F20B00340EE
:10CCC00020B00B40E191FF1F24B0034024B00B4083
:10CCD000A99FFF1F0C2830B417D91023984228BFF2
:10CCE00018461C46104A114D1178181A8C422870AB
:10CCF00018D00F4913700B7823B10E490E4A002348
:10CD00000B60136030BCFFF775BF0A2802D90C23F3
:10CD10001C46E7E7082802D90A231C46E2E7082355
:10CD20001C46DFE730BC7047E091FF1FA89FFF1F44
:10CD3000A99FFF1F24B0034024B00B4028282FD800
:10CD4000334B2DE9F0411E5CFF2E2BD0314B1B786D
:10CD5000002B2AD132062CD472B62F4D2F4C2F46E1
:10CD6000012326602B7062B672B623681B060CD4B2
:10CD70003B781BB9F4E72B78002BF1D062B602F0B8
:10CD80009BF972B623681806F5D5254B1B6800225F
:10CD90002A7062B6234A107843FA00F0BDE8F081A9
:10CDA000002070470020BDE8F081FFF781FE3206C9
:10CDB000D2D572B61C4DDFF87C801C4C06F04007C3
:10CDC000FFB206F03F06D8F80030DFB123F01003C1
:10CDD000C8F8003001232660134A2B7062B672B681
:10CDE000236819060CD413781BB9ECE72B78002BB9
:10CDF000E9D062B602F060F972B623681B06F5D579
:10CE00000B4BC3E743F01003C8F80030E2E700BF64
:10CE10005C3E0100A99FFF1FAB9FFF1F00B00340B6
:10CE200010B00340A89FFF1FAA9FFF1F00B00B4038
:10CE300010B00B400CB00B400A4A0B49136843F486
:10CE4000805313600B7843B9084BC0221A70084B0B
:10CE500080F30C0000B218807047044B80221A70D7
:10CE6000F5E700BF2C800440AC9FFF1F21C00C40A1
:10CE700000C00C40F0B51B4B1B4E596818689A68EF
:10CE8000DB6885B06C460FC4337899071DD5174A07
:10CE9000174C1378174913F0700318BF1370164A14
:10CEA000164B8027177000263320032226706D460C
:10CEB00008701A7072B6043C45F001052046A84778
:10CEC00062B6237813F0700309D10D4B064901E0D7
:10CED000013B02D00A78D207FAD505B0F0BD237025
:10CEE00005B0F0BD883E0100010002400000024094
:10CEF000040002400B000240070002400A0002400A
:10CF0000410D0300B0F5006F0AD210B5094B1B7834
:10CF1000DB07044606D504F1A0500078C0B210BD6E
:10CF200000207047FFF7A6FF04F1A0500078C0B2C0
:10CF300010BD00BF01000240B0F5006F17D238B538
:10CF40000F4B1B78DA070D46044611D504F1A050AB
:10CF50000378AB420AD00B4A137813F0700318BF62
:10CF60001370074A05701378DB07FCD538BD70478E
:10CF7000FFF780FF04F1A0500378AB42EBD1F5E757
:10CF8000010002400000024008B5F4F773FDF5F718
:10CF90001DFC02F091F8FAE7844641EA000313F021
:10CFA00003036DD1403A41D351F8043B40F8043BB0
:10CFB00051F8043B40F8043B51F8043B40F8043B73
:10CFC00051F8043B40F8043B51F8043B40F8043B63
:10CFD00051F8043B40F8043B51F8043B40F8043B53
:10CFE00051F8043B40F8043B51F8043B40F8043B43
:10CFF00051F8043B40F8043B51F8043B40F8043B33
:10D0000051F8043B40F8043B51F8043B40F8043B22
:10D0100051F8043B40F8043B51F8043B40F8043B12
:10D0200051F8043B40F8043B403ABDD2303211D3B2
:10D0300051F8043B40F8043B51F8043B40F8043BF2
:10D0400051F8043B40F8043B51F8043B40F8043BE2
:10D05000103AEDD20C3205D351F8043B40F8043BB2
:10D06000043AF9D2043208D0D2071CBF11F8013BB0
:10D0700000F8013B01D30B8803806046704700BF76
:10D08000082A13D38B078DD010F003038AD0C3F185
:10D090000403D21ADB071CBF11F8013B00F8013B67
:10D0A00080D331F8023B20F8023B7BE7043AD9D326
:10D0B000013A11F8013B00F8013BF9D20B780370FB
:10D0C0004B7843708B7883706046704708B5104C7E
:10D0D00008E0236859050DD423681A050FD4236886
:10D0E000DB0411D423685803F3D500F08DFE2368C8
:10D0F0005905F1D502F044F823681A05EFD502F07E
:10D10000D5F82368DB04EDD500F0F0FCEAE700BFBA
:10D110003480044008B5FFF7D9FF00BF014B10224F
:10D120001A80704700200540704700BF094908B5C4
:10D130000B6830B16A461844A2F58052904202D280
:10D140000860184608BD03F065FB0C2303604FF030
:10D15000FF3008BDE491FF1FFEE700BFEFF313802F
:10D1600070B9EFF310836BB9EFF305825AB94FF43E
:10D170008070EFF311832BB1984228BF1846704797
:10D180004FF0FF3070470F2A01D81846F1E7014BE6
:10D19000D05CEEE7F0E300E0F0B44D1E2E46002434
:10D1A00000E00134B0FBF2F302FB1300092800F1A8
:10D1B00030078ABF3730F8B2C0B206F8010F184600
:10D1C000002BEED10A1953704CB1107815F8016F8D
:10D1D00028700133E01A834202F80169F5DB084642
:10D1E000F0BC7047704700BF10B40F4B53F83020AD
:10D1F00092F880422CB1012369B182F8803010BCD2
:10D20000704703EBC0035B681A6841B922F0020261
:10D210001A6010BC704782F8003110BC704742F0B1
:10D2200003021A6010BC7047983E01001C4A02EBD2
:10D23000C00301295B6811D004291BD052F83000CB
:10D24000002280F8802229B1022920D0032922D08F
:10D250001A6070474FF480721A60704752F83000BD
:10D260004FF4A27280F880121A601A6822F020022D
:10D270001A60704752F830104FF4A272012081F802
:10D2800080021A601A6842F020021A60704740F269
:10D2900003121A6070474FF481721A60704700BF22
:10D2A000983E0100212848D8F8B5042A44D8DFE880
:10D2B00002F0484B4E0345004FF410262B4B03EB76
:10D2C000C0030D465C68216811F4E06148D0284B2A
:10D2D000284A2949C3F89C2104F140422748C3F851
:10D2E000A411A2F59221264FC3F8A0017C2925485C
:10D2F000C3F8A871C3F8AC012CD9A2F594237C2BF8
:10D300002AD9A2F596237C2B28D9A2F598237C2B29
:10D3100029D9A2F59A227C2A27D81B4872B62368FD
:10D3200023F4702343F08072C4F384011643236016
:10D3300040F82150266062B6F8BD70474FF43026A1
:10D34000BCE74FF40026B9E74FF44026B6E74FF4A8
:10D350002026B3E70D48E1E70D48DFE70D48DDE79C
:10D36000FFF764FFB3E70C48D8E7F8BD983E01002B
:10D370000082FF1FF188FF1F9988FF1FC588FF1FCC
:10D380006D88FF1F4188FF1FC092FF1FE891FF1F9C
:10D390002092FF1F7092FF1FA092FF1F1A4B03EBFA
:10D3A000C00010B4426802F14043A3F592217C29E9
:10D3B00023D9A3F594217C290DD9A3F596217C29A5
:10D3C0001FD9A3F598217C2919D9A3F59A237C2B81
:10D3D00011D80E4C00E00E4C72B613680D4823F0C5
:10D3E0008773C2F3840123F4803343F080731360A6
:10D3F00044F8210062B610BC7047074CECE7074CBC
:10D40000EAE7074CE8E700BF983E0100C092FF1F23
:10D410002092FF1FE5D10000E891FF1FA092FF1F9F
:10D420007092FF1F30B4054B054D064C00221021B1
:10D430001A602A602060196030BC704714D0034025
:10D4400004D0034000D00340282838B52ED000294E
:10D4500004464FDD5F4B1B78012505FA03F28A4233
:10D4600002D8212837D938BD0338C2B2012A3AD9A7
:10D47000202C4AD0192C48D0574A126802FB0112BE
:10D4800022FA03F31D2800F29B80DFE800F0928B64
:10D49000847D9999766F99999999999999999968AB
:10D4A000615A53994C99999999999945494B1B7887
:10D4B0000B2B08D90C2B1CBF0C3B19410846BDE8AF
:10D4C0003840FFF7B9BCC3F10C0399400846BDE8EA
:10D4D0003840FFF7B1BC2946FFF786FE2946BDE874
:10D4E0003840FFF7A3BE3D4A126802FB011222FA40
:10D4F00003F3C7E72128B6D80021FFF775FE2046C1
:10D500000121BDE83840FFF791BE354A126802FBA1
:10D51000011222FA03F3B5E73249334A0B604FF4A4
:10D520005173136038BD3149314A0B604FF4517368
:10D53000136038BD2F49304A0B6040F244431360FA
:10D5400038BD2E492E4A0B6040F24443136038BD6B
:10D550002C492D4A0B6040F24443136038BD2B49DF
:10D560002B4A0B6040F24443136038BD29492A4AD4
:10D570000B6040F24443136038BD2849284A0B60D1
:10D5800040F24443136038BD2649274A0B6040F2FD
:10D590004443136038BD2549254A0B6040F244439B
:10D5A000136038BD2349244A0B604FF45173136054
:10D5B00038BD2249224A0B604FF45173136038BDC5
:10D5C000212C3FF650AF7F29D4BF002101212046F6
:10D5D00093E700BFC892FF1F0880034008900340F4
:10D5E00008800B4010800B4048A0044018800B407E
:10D5F0004CA004401880034008B004401080034051
:10D6000004B004404080034018C004403880034008
:10D6100014C004402880034010B004402080034020
:10D620000CB004403080034010C0044048800340E8
:10D630001CC00440189003403490044010900340F4
:10D640003090044038B1102828BF1020044AC3B2DB
:10D65000107813707047024A0123107813707047D6
:10D66000C892FF1F2DE9F8430E4680463249334DDC
:10D67000304603F055F847F6122300281ABF1D461E
:10D680004FF002094FF00109002425FA04F002F0DE
:10D6900051FE4FF05E51074602F0A4FE01463046AF
:10D6A00003F052F830B90134072CEED1E80902F04A
:10D6B00041FE07463146384602F048FF4FF07C51A4
:10D6C00002F086FD03F07AF84FF6FF729042A8F15F
:10D6D000030328BF1046012B29D9B8F1170F17D81B
:10D6E000174B23FA08F303F0010383F0010223B977
:10D6F000B8F1190F0FD0BDE8F883124B124D134942
:10D700001A6044EAC9042A6008601C60BDE8F88316
:10D71000B8F1200FECD10E4B0E4D0F49002244EA18
:10D72000C9041A602A6008601C60BDE8F8830B4BCE
:10D730000B4D0C49F2E700BF001BB740006CDC0248
:10D740006006F0000080034004800340088003402E
:10D7500000800B4004800B4008800B400090034089
:10D760000490034008900340212801D8FFF73CBDF6
:10D77000704700BF212806D8044B53F8303093F887
:10D780000002C0B270470020704700BF983E010001
:10D79000212801D8FFF74ABD704700BF72B60C4977
:10D7A0000C4B0D4A1B680868126862B6520102D51C
:10D7B000322B88BF01300949C3F5BB334FF47A726D
:10D7C000FF33A1FB031302FB00F000EB9310704743
:10D7D000B09FFF1F18E000E004ED00E0ABAAAAAA8A
:10D7E0002DE9F843054672B6204F214B214A1B68AC
:10D7F0003C68126862B6520102D5322B88BF0134F0
:10D8000095B3C3F5BB331C4EDFF86490DFF864803A
:10D81000FF334FF47A72A6FB031302FB04F404EB0C
:10D82000931472B6D9F800103A68D8F800E062B6DE
:10D83000C1F5BB33FF33A6FB03031EF0806FC4EBBF
:10D8400093134FF47A7002D0322988BF013200FB63
:10D850000233B3F57A7F04D3013D05D004F57A7421
:10D86000DFE701F029FCDCE7BDE8F883B09FFF1F8C
:10D8700018E000E004ED00E0ABAAAAAAF8B52D4B31
:10D880002D49DFF8D0E0DFF8D0C02C4E2C4D2D4CC8
:10D890002D4A2E4F4FF4000018604FF08070186032
:10D8A0004FF0007018604FF0806018604FF000601B
:10D8B00018600020086028234BF6FF71CCF8001098
:10D8C000CEF80030336013602B6023603B60B3629E
:10D8D0009362092245F8242CC4F8D80F05F57F651A
:10D8E000C7F8D41F07F5FF2707F5FA67C6F8F83F12
:10D8F0002B6006F5FF26C4F8D42F05F5FD2504F5A9
:10D90000FF24386006F2F4761148316005F5FF65B2
:10D9100004F5FD642B6023600260FFF76BF91920AA
:10D92000FFF75EFF00F0B6FF40F21310BDE8F840CD
:10D93000FFF756BF08E100E0048003401480034075
:10D94000248003402C8003401C800340348003402B
:10D9500000800B400C800340088003402DE9F84F05
:10D96000214B1B6807460BB101221A70DFF8889023
:10D970001E4D99F80040DFF884801D4E0134272C9D
:10D980008ABF4FF0000A5FFA84FA5446AB462B7800
:10D99000A34216D1FFF7E2FB40281FDC33791B06B8
:10D9A000F5D59BF800300133272B86BF00221346A4
:10D9B000DAB218F80330DBB2F3712A702B78A34285
:10D9C000E8D00C490A4BFFB208F804700120AC22E1
:10D9D000087089F800A0DA70BDE8F88FFF28D6DD5E
:10D9E00001F06AFBD3E700BF28A0FF1F25A0FF1F9F
:10D9F00000C0064024A0FF1F2CA0FF1FBC9FFF1FDC
:10DA00001C4BDFF894C01A681B49F0B542F48052F1
:10DA10001A4D1A60DFF884E0194F1A4E1A4C002391
:10DA20008CF800304FF451722B701F2840F21335E0
:10DA30008EF800303B70337025600A6012D81946AA
:10DA40000124124A124D11701248547000212C27E3
:10DA5000402693724FF4003491701174D7702E7079
:10DA60000460F0BDC0F34431C0F3471400F01F035D
:10DA7000E7E700BF348004400CC00440B99FFF1F9B
:10DA800025A0FF1F24A0FF1F08C0044000C00640BF
:10DA900031E400E004E100E0B89FFF1F2CA0FF1F6D
:10DAA000034B1B68DB0401D5FFF758BF704700BF6D
:10DAB0003480044010B5044C237823B101F0FCFA03
:10DAC0002378002BFAD110BD24A0FF1F054A064B76
:10DAD00010781B78C0B2DBB2984238BF4030C01A11
:10DAE000704700BFB89FFF1FB99FFF1F30B42B4B7B
:10DAF0001A7994061FD52A48DA790378294901331F
:10DB00003F2B0978C8BF00238B42D2B203D0264CEA
:10DB1000D9B2E2540170254A116861B1244A1278E1
:10DB2000D2B2934236BFC2F140029B1A9B18272BF8
:10DB3000C4BF01230B70194AD378DBB2180611D485
:10DB40005A060DD5154B1B795B0609D5194B1A4999
:10DB50001B6800220A7003B11A70104B2C22DA7075
:10DB600030BC704711790906EAD5144910480C7881
:10DB70000178C9B28C420DD04A1C272A84BF0021EB
:10DB80000A460F4D054C98BFD1B2AA5CD2B2E271E1
:10DB90000170D5E76C21D170D2E700BF00C006400C
:10DBA000B89FFF1FB99FFF1FE49FFF1FB49FFF1F78
:10DBB00025A0FF1F28A0FF1F24A0FF1F2CA0FF1FD0
:10DBC000BC9FFF1F21282FD8184B195CFF292BD091
:10DBD000174B184ADFF870C003EBC000F0B543687C
:10DBE000DFF868E0144F154D154E00241C60DEF878
:10DBF0000030012043F020038840CEF8003014604C
:10DC00004FF4A07338602E60C2F800C0013BFDD114
:10DC100013689B05FCD42023013BFDD1094B09B2BD
:10DC200033F8110080B2F0BD00207047A83F01001A
:10DC3000983E010000500440085004400450044045
:10DC4000000002030051044080014A003880044073
:10DC5000431E032B14D872B60A4951F8230068B149
:10DC600070B4094C058834F81320466841F82360E5
:10DC7000521B24F8132062B670BC704762B670471E
:10DC80000020704788A0FF1FCCA2FF1F0138032887
:10DC90000BD872B6074B53F8203043B100205B68B5
:10DCA0000130002BFBD162B6704700207047184648
:10DCB000F9E700BFDCA0FF1F30B472B62B4A13781F
:10DCC0001D0706D52A4B196A002936D0996A002902
:10DCD00041D053781C0706D5254B196C00293ED03E
:10DCE000996C002939D09378190705D5204B196E06
:10DCF000002936D0996E89B1D3781B0707D51C4B04
:10DD0000D3F880207AB3D3F8882011213AB162B6D3
:10DD1000184B00221A7030BC00F04ABE0D21154C81
:10DD2000154D227843F8315003EBC1030830013A16
:10DD30005860227062B630BC704704220D4C0F4D03
:10DD4000217843F8325003EBC20308304A1E586072
:10DD5000227062B6EFE70521E1E70921DFE708223B
:10DD6000ECE70C22EAE71022E8E700BFCC3F010015
:10DD70000080FF1F05A1FF1FC80040008800400071
:10DD8000431E032B1DD81B4A400140F0100030B445
:10DD9000104472B6184CE25C032A1BD8DFE802F08C
:10DDA0000212151703220D88E25410F0080F14BF59
:10DDB000C823882343EA054308310360416062B603
:10DDC00030BC704708300222EDE70522EBE708304F
:10DDD0000422E8E7094A52F8230038B1084A52F809
:10DDE0002300416042F8231062B6E9E742F82310AD
:10DDF000034AF7E70080FF1F14A1FF1FDCA0FF1FED
:10DE0000ECA0FF1F00BE70472DE9F04FDFF818B3FC
:10DE1000DFF818A387B044E0AD4F4FEA930807EB53
:10DE2000C809013ED9F8042003F00803F6B2A2F1B4
:10DE3000080003F0FF04002B40F0018157F8383050
:10DE40001B0C99B222F8081C002B00F0EF80A14BAC
:10DE500022F8064C42F8044C53F82620002A00F021
:10DE6000CF819D4D55F8263058609C4C45F82600D2
:10DE700034F81630194424F8161000F079FD002803
:10DE800000F0C281964A974B19F0080F00F1080084
:10DE900018BF1346C9F8040047F8383008238BF838
:10DEA00000309BF80040E4B265071CD58E4B1B7810
:10DEB000B3B18E490A7802F0FF0322B1013BDBB215
:10DEC0000B7003B900BE8A490A7802F0FF032AB139
:10DED000013BDBB20B70002B00F0688100F066FEA6
:10DEE00004238BF8003004F0080303F0FF02002B3A
:10DEF00000F0C9809AF80030DBB21E098CD19A0874
:10DF0000DFF8CC9159F8321009EBC200C1F383015C
:10DF1000013940680C2900F28580DFE801F07A7A47
:10DF20008383838383834683838307000168714DE2
:10DF30004068714F714E6860296088B240F281611B
:10DF40000024674B49F832304FF0010E88423C60A4
:10DF5000C9F81040C9F8184086F800E05C4A00F2A1
:10DF6000E780B0F5D06F80F01B82B0F5817F00F0C4
:10DF7000D98100F26981802800F02A82822840F04D
:10DF8000D781A98801F07F01042900F2D1815C4882
:10DF90005C4A890008441470547001788C0740F181
:10DFA000608382F800E0022173E1534F3A682AB39C
:10DFB000554B524E554819883478057840298E467D
:10DFC00045F0020828BF4FF0400E002C84F00104F9
:10DFD0003470CEEB01010CBF8824C82409EBC806BD
:10DFE00089B285F0010544EA0E447260198049F84F
:10DFF000384072440570002965D03A603D4B1A885C
:10E00000B2F5A06F0ED100219A785970404B1A706A
:10E0100008E038493F4C0D68A54200F0988030492F
:10E0200049F832103C4A0123137037E72C4A2D4B34
:10E0300019F0080F18BF134647F838302EE700F0E4
:10E04000B7FC364A364952F82630002B00F0E38000
:10E0500058688C5D42F8260003F10802C9F80420D4
:10E06000032C05D8DFE804F02C02292602228A5569
:10E070001A8819F0080F0CBF8823C82343EA02430B
:10E0800047F838300AE7E00700F19380210600F1F5
:10E09000D180A20706D5234A234913780220DBB298
:10E0A00013700870E30602D51F4B10221A7007B0D8
:10E0B000BDE8F08F04228A55DAE705228A55D7E7B2
:10E0C00003228A55D4E7BEF1400F18BF002294E71F
:10E0D0000080FF1F88A0FF1F34A0FF1FCCA2FF1FDE
:10E0E000C80040008800400010A1FF1F99A0FF1F3A
:10E0F00084A1FF1FFCA0FF1F30A0FF1F98A0FF1FDF
:10E10000C020074008A1FF1F44A0FF1F04A1FF1F5C
:10E11000982007402109000394200740DCA0FF1F3E
:10E1200014A1FF1F8820074080200740902007404F
:10E13000B0F5106F00F07C8140F2A38040F6211210
:10E14000904240F07B82A54A012313706AE74C6835
:10E15000A3498C427FF463AF0178A9297FF45FAFB4
:10E16000417845297FF45BAF8178C2297FF457AFAE
:10E17000C1786B297FF453AF9A489B4E017834786D
:10E1800081F00105002C41F0020105700CBF8820D0
:10E19000C82084F0010449F8310009EBC10193481B
:10E1A0003470002505244D60047038E700F064FFEA
:10E1B00094E68F4B89488B491A614FF0020E80F824
:10E1C00000E08C4F0A708C49196099608B4E8C4D21
:10E1D0008C4C9A610D213970FF213170DFF84CE2CF
:10E1E00029702270884D894A8EF800109F270124DB
:10E1F00006F8047C5D600470DA6007B0BDE8F08F5B
:10E2000043F82600824D30E6824A47F838001378FA
:10E210000133137042E68B5D032B00F2BA8001A23A
:10E2200052F823F09DDE00009DDE00007DE200003C
:10E2300077E200006F49724B80220D2008701A703F
:10E24000A2077FF52FAF26E740F20232904240F05E
:10E25000ED81AA8802F07F02042A69D86D88002D1A
:10E2600066D16449CDF804E0920011440A7842F086
:10E2700002020A70C1E101238B550FE600238B5582
:10E280000CE6B0F5086F53D16349644A0978117000
:10E290007146ED888D4280F0E88252480478402D26
:10E2A000AE4644F0020C28BF4FF0400E02EB0E03C6
:10E2B00009EBCC01029301234A604FEA0E48CEEBF2
:10E2C000050101930025C82242EA080384F00102F7
:10E2D00049F83C3035700270DFF814C1424BDFF86A
:10E2E000048149BBBEF1400F7FF42DAF42F0020C18
:10E2F00009EBCC03029ADFF8F8E05A608DBB0D04FD
:10E3000045F088059DF804304EF83C500A443370BF
:10E310000470134640297FF416AF0021404A3B6049
:10E32000118010E7AA8802F07F02042A40F28B8154
:10E33000304A0F23137006E74029D7D942F0020272
:10E340000CEBC200029E4660BDB19DF804503548FA
:10E350001D703346403988F8004040334CF8320095
:10E36000DCE79DF8043033700D04029B047045F027
:10E37000C8050B444EF83C50CCE79DF804501D7086
:10E38000029B1D4888F80040403940334CF8320069
:10E39000C4E719F0080F0CBF022303238B557DE55A
:10E3A00021494A68002AC3D06C88B5F804E003E02C
:10E3B0000C314A68002ABBD00B88A342F8D14B88A5
:10E3C0007345F5D1240A032C0CBF1178098960E745
:10E3D000124A0221147054705BE700BF942007407A
:10E3E0000100040004A1FF1F98A0FF1F99A0FF1FB8
:10E3F0000080FF1FC02007408800400088200740A1
:10E40000802007409820074048A0FF1F9CA0FF1FC6
:10E4100034A0FF1F05A1FF1F10A1FF1F08A1FF1FB0
:10E4200044A0FF1FC8004000D03F01008C200740DF
:10E43000B248116AAC7804700C0600F19881D9F8E2
:10E440002820AF49100600F1DB81D9F83020AC4913
:10E45000120600F1D081D9F83820A949130600F13D
:10E46000C581D9F84020A649150600F1BA81D9F82E
:10E470004820A349140600F1AF81D9F85020A049E3
:10E48000100600F1A481D9F858209D49120600F128
:10E490009981D9F860209A49130600F18E81D9F844
:10E4A00068209749150600F18381D9F870209449B6
:10E4B000140600F17881D9F878209149100600F10E
:10E4C0006D81D9F880208E49120600F16181D9F85A
:10E4D00088208B49130600F15581D9F8902088498E
:10E4E000150600F14981D9F898208549140600F1F4
:10E4F000FF808448844A854901908548854D864C33
:10E50000049700230596029580460F4616461D4641
:10E510000394306828B1446800F04AFA2046002C81
:10E52000F9D100233360029B38681A46002342F871
:10E53000253028B1446800F03BFA2046002CF9D180
:10E5400000223A60019A98F800301146002241F802
:10E55000042B039A0191023B4FF0000122F81510A1
:10E56000032B07D8DFE803F05D025D024FF00103E3
:10E5700088F800300135042D06F1040607F1040780
:10E5800008F10108C5D1654C654D2278654B049FA3
:10E59000059E0021100729701A7000F192806249CF
:10E5A00062780A700021C9F83010C9F838101107D4
:10E5B000DFF84C816ED4A2785C49DFF844810A70A0
:10E5C00000211207C9F85010C9F858104BD4E2784E
:10E5D00057494B4C0A7013074FF00001C9F87010EF
:10E5E000C9F8781000F1AE8033780193002283F0EF
:10E5F0000105C9F89020C9F89820002102918846A9
:10E600008E460A464B48047844F0020C09EBCC03D2
:10E610000393019B002B039B5A600CBF8822C822E6
:10E6200052E64FF0000388F80030A3E7B0F5A06F82
:10E630007FF47EAE012300250193DEE740F6212220
:10E640009042F7D074E66D88002D7FF471AE3A49A0
:10E65000CDF804E0920011440A7822F002020A7018
:10E66000CBE7022115E600F083F9002800F0EB80EB
:10E670000830324AC8F86400C8F8602000F078F921
:10E68000002800F0DA8008302D4AC9F86C00C9F87B
:10E6900068209CE700F06CF9002800F0E08008306A
:10E6A000264AC8F84400C8F8402000F061F9002864
:10E6B00000F0CF800830224AC9F84C00C9F8482041
:10E6C00079E700F055F9002800F0A58008301B4AD2
:10E6D000C9F82400C9F8202000F04AF9002800F009
:10E6E00094800830164AC9F82C00C9F8282056E74B
:10E6F000D1F89C00083800F05BF9FAE610A1FF1F82
:10E700000080FF1FECA0FF1F88A0FF1FDCA0FF1FE1
:10E7100014A1FF1F34A0FF1FCCA2FF1FCC3F01009C
:10E7200005A1FF1FC4200740C8200740CC20074098
:10E73000D020074004A1FF1FC020074088004000F0
:10E74000C800400000F014F9002870D008304F4A8B
:10E75000C4F88400C4F8802000F00AF9002860D0D2
:10E7600008304B4AC9F88C00C9F888203CE7506A49
:10E77000083800F01DF962E6D1F89400083800F07E
:10E7800017F9B0E6D1F88C00083800F011F9A4E6CA
:10E79000D1F88400083800F00BF998E6C86F083803
:10E7A00000F006F98DE6486F083800F001F982E6BE
:10E7B000C86E083800F0FCF877E6486E083800F0BC
:10E7C000F7F86CE6C86D083800F0F2F861E6486DBD
:10E7D000083800F0EDF856E6C86C083800F0E8F8A4
:10E7E0004BE6486C083800F0E3F840E6C86B0838A0
:10E7F00000F0DEF835E6486B083800F0D9F82AE674
:10E80000C86A083800F0D4F81FE62A78C9F828004A
:10E8100001322A70C3E62A78C9F8200001322A7032
:10E820005AE72A78C9F8880001322A70DCE62A788B
:10E83000C4F8800001322A708EE72A78C9F868008F
:10E8400001322A70C3E62A78C8F8600001322A70C3
:10E8500014E72A78C9F8480001322A70ABE62A7812
:10E86000C8F8400001322A701FE740298E4628BFB1
:10E870004FF0400E02EB0E0302930123CEEB010199
:10E880004FEA0E4800250193BCE600BF8800400017
:10E89000C8004000F8B500F08FFD294B29482A4CEC
:10E8A0002A4F2B4DDFF8BCC0DFF8BCE0294E002218
:10E8B0001A605A609A60DA601A615A619A61DA6184
:10E8C0001A625A629A62DA621A635A639A63DA6364
:10E8D0001A645A649A64DA641A655A659A65DA6544
:10E8E0001A665A669A66DA661A675A679A67DA6724
:10E8F000C3F880200168C3F8842041F480210160BE
:10E90000C3F307212170C3F30740134938701B0E6E
:10E910002B70FF238CF80030104D8EF8003010481B
:10E920000B700123337084F8642070264FF4007458
:10E93000102207F82C3C2E70046081F8F820F8BDF6
:10E940000080FF1F348004409C200740B020074017
:10E95000B4200740942007401020074049E400E01D
:10E9600008E100E08020074088200740704700BF92
:10E9700072B60D480268B2FA82F30F2B10DC4FF02A
:10E980000041D94022EA0102026062B6074803EB67
:10E99000C303DB00C2180021C1501046516070470C
:10E9A00062B60020704700BFCC92FF1FBC83FF1FE0
:10E9B0000D4B0E4AC31AA2FB03231B090F2B0CD8C5
:10E9C0000B4A127852B972B60A484FF000410268F9
:10E9D00021FA03F31A43026062B67047064A1278BE
:10E9E000002AF0D0FFF768B9BC83FF1F398EE338E7
:10E9F00005A1FF1FCC92FF1F10A1FF1F38B50E4BC2
:10EA00000E4C1B68218805468BB1B1F5917F05D26C
:10EA10000B4A4B1C55549BB2238038BD002208483A
:10EA200098470021064A55540123238038BDB1F58B
:10EA3000917FEDD338BD00BF3CA1FF1FD6A2FF1FC1
:10EA4000DCA2FF1F2DE9F843214E224F316801233C
:10EA500080463B70B1B1204D4B8801EB83020133FE
:10EA600000240F2BC2F808802C7004D84B800023A0
:10EA70003B70BDE8F88340230B800320FFF780F94B
:10EA80003460F4E7DFF8549099F80030002BF0D0B0
:10EA9000114D45F6215408E0013C12D02B7883B982
:10EAA00000F00AFB99F800307BB10320FFF7EEF885
:10EAB0000528F1D8FFF75CFF014630600028EBD055
:10EAC000CAE701232B70BDE8F883BDE8F88300BFD7
:10EAD00058A1FF1F2CA1FF1F5CA1FF1F10A1FF1F4A
:10EAE0001201F8B5D5B2A1B3012943D04378044649
:10EAF00000781B0643EA004040F4704045F00406ED
:10EB00008F1E3043FFF79EFF022F04F1020314D93A
:10EB1000053414F8023C14F8032C14F8010C1B04FF
:10EB200043EA0223334343EA0060033FFFF78AFFCF
:10EB3000022F234604F10304EBD8022F23D0012F28
:10EB40000DD045F4774040F00500BDE8F840FFF7F0
:10EB500079BF14482843BDE8F840FFF773BF187821
:10EB600045F4770545F0060545EA0020BDE8F84084
:10EB7000FFF768BF03780C4845EA03452843BDE822
:10EB8000F840FFF75FBF1A78587845F0774545F0B1
:10EB9000070545EA022545EA0040BDE8F840FFF7D1
:10EBA00051BF00BF06F0F70007F000F738B5084B7B
:10EBB0001C7824B9074D296809B14B8803B938BDC1
:10EBC0009B000B800320FFF7DBF82C6038BD00BFF3
:10EBD0002CA1FF1F58A1FF1F2DE9F041AD4E336856
:10EBE0000746002B00F092801D885A88910803EB9D
:10EBF00081010432AA428C6842D25A8004F00F0686
:10EC00004FEA1428A449A6F1080208F00F00C4F343
:10EC10000313062A00F101050B701AD9B31E012B4C
:10EC20005FFA88F04ED9052E48D0042E00F0A4815A
:10EC3000731F022B7FD90F2E0ED1F72842D8F02850
:10EC400002D0964B1B883BB1FFF7D8FE0020BDE8F1
:10EC5000F08127B1BD4202D00020BDE8F081082E2E
:10EC6000C4F3033300F08780092E11D00A2E40F040
:10EC700094800A2BF0D18A4B8A4A1B68A02181E03C
:10EC80001846FFF795FE0420FEF7E2FF3060B5E777
:10EC9000092BE1D1270E00F07B81834B814A1B6851
:10ECA0009021C4F307461170EDB2FCB2002B00F0C6
:10ECB0009D80224631462846984797E0F02843D960
:10ECC000F72841D0F1380E28C6D801A353F820F018
:10ECD00087EE00006BEE000059EE000059EC0000DA
:10ECE00059EC00004BEE000059EC00002BEF000047
:10ECF00059EC0000F5EE00000FEF000033EE0000CD
:10ED000059EC00001BEE0000FFED0000674B1B7884
:10ED1000002BA1D00420FEF79BFF034630600028A3
:10ED20009AD00588002D7FF460AFFFF741FE356073
:10ED30002846BDE8F081FFF761FEC4F30740FFF706
:10ED40005DFE072E02D1200EFFF758FE534B584AA6
:10ED5000198858481468584D524A017000270E0A05
:10ED6000F0201F802E7010700CB301225348A04772
:10ED70000120BDE8F081082B7FF46EAF504B494A6B
:10ED80001B688021C4F307461170EDB2240E6BB3EB
:10ED9000284622463146984728E00B2E11D10B2BEE
:10EDA0007FF45AAF474B3F4A1B68B021EAE7464B16
:10EDB0001B68002B00F0FB80404898470120BDE80D
:10EDC000F0810C2E40F000810C2B7FF445AF3F4BBF
:10EDD000344A1B68C0211170EDB2C4F30746002B02
:10EDE00000F0C88028463146240E98473849314AF9
:10EDF000314B0D7016701C700120BDE8F081354B51
:10EE00001B68002B00F0D6809847C4F30746254BBB
:10EE1000EDB2240E83F80080E8E72F4B1B68002B2F
:10EE2000F2D12E4B1B68A3B1FE209847C4F30746CE
:10EE3000EDE72B4B1B68002BE6D1284B1B6843B139
:10EE4000FC209847C4F30746E1E7264B1B68002BDC
:10EE5000DAD1C4F30746DAE7234B1B68C4F307464D
:10EE6000002BD4D030469847D1E7204B1A68002AAF
:10EE7000EFD0260C630C06F07F0003F47E5318439A
:10EE8000F6B29047C3E71A4B1B68C4F30746002B42
:10EE9000E8D1BCE764A1FF1FDAA2FF1FD6A2FF1FC3
:10EEA00040A1FF1FD4A2FF1F74A1FF1F10A1FF1FCD
:10EEB0003CA1FF1FD8A2FF1FD9A2FF1FDCA2FF1F8A
:10EEC0006CA1FF1F70A1FF1F54A1FF1F30A1FF1FE6
:10EED000DBA2FF1F1CA1FF1F20A1FF1F24A1FF1FFA
:10EEE00060A1FF1F50A1FF1F68A1FF1F38A1FF1FD6
:10EEF0004CA1FF1F3F4B1B68002B85D13E4B1B686D
:10EF0000002BA6D0FA209847C4F307467FE73B4B77
:10EF10001B68002B7FF478AF374B1B68002B98D011
:10EF2000FB209847C4F3074671E7354B1B68002B5D
:10EF30007FF46AAF304B1B68002B8AD0F8209847CB
:10EF4000C4F3074663E70E2B7FF486AE2D4A2E4BA3
:10EF50001268E0211970002A47D0260C610C06F0D7
:10EF60007F0301F47E511943EDB2A1F5005128460B
:10EF70009047F6B2240E39E7FFF740FDC4F307408F
:10EF8000FFF73CFD200EFFF739FD0020BDE8F081C2
:10EF90001E4B1D4A1B6880211170EDB2C4F3074659
:10EFA00083B1314628463A4698473C461EE7012041
:10EFB000BDE8F081104B1B68002B3FF44AAFFF20E7
:10EFC000984746E71C4611E70D2EBCD10D2B7FF468
:10EFD00043AE0F4B0C4A1B68D0211170EDB2C4F345
:10EFE0000746002B7FF4FEAEC4E7C4F30746EDB23C
:10EFF000240EFBE648A1FF1F24A1FF1F28A1FF1F2D
:10F0000018A1FF1F34A1FF1FD4A2FF1F6CA1FF1F77
:10F0100044A1FF1F38B5164D2868E0B10188448827
:10F02000A14213DD03191B7A83B104F10803C2184E
:10F030000C1B002302E012F8011F21B10133A3428F
:10F04000F9D1204638BD1C46204638BDFFF7B0FC3C
:10F050000020286038BD074B1B780BB9002038BD55
:10F060000220FEF7F5FD28600028D7D1F6E700BFA3
:10F0700080A1FF1F10A1FF1F0D4B1B78BBB910B55E
:10F080000C4C216803F0FF024B883F2B07DC073351
:10F090000B4401F1470003F8012F8342FBD14023C9
:10F0A0000B800120FEF76CFE0023236010BD70472B
:10F0B00078A1FF1F7CA1FF1F38B5224C237803B134
:10F0C00038BD01232370FFF7A5FF70BB00F048F89F
:10F0D00040BB00F0DBF810BBFEF7F8FCE0B9002302
:10F0E0002370EFF30583002BEAD1EFF3108172B6A2
:10F0F000154B1868E0B1154C2278CAB945691D60F6
:10F1000001232370C5B1AA6101B962B60025457714
:10F11000836898472570D3E700F020F8DFE700F018
:10F120001BF8D9E700F016F8D3E7FFF71FFCCDE78F
:10F130000029C5D162B638BD054B1D600029E5D157
:10F14000E3E700BF85A1FF1F9C9FFF1FA09FFF1F3C
:10F15000989FFF1F704700BF704700BF704700BFF8
:10F16000054A064B10781B78C0B2DBB2984238BF14
:10F170004030C01A704700BF8CA1FF1F8DA1FF1F38
:10F18000F0B4384B1A7912F0300F2CD072B6997D4A
:10F1900001F0FF0200293DD062B6334F3349387881
:10F1A0000D78334E1C46C0B2EDB2431C402BE179C2
:10F1B00028BF0023AB4202F1FF32C9B21CBFF15499
:10F1C000184612F0FF02F0D12A4B1B68C2B23A7007
:10F1D0004BB1A84236BFC5F14005401B4019272856
:10F1E000C4BF01221A701F49CA78D2B2150616D4BC
:10F1F00052060DD51B4B1B795B0609D51E4B1F49CB
:10F200001B6800220A7003B11A70164B3C22DA7098
:10F21000F0BC70474022D9795A7462B6E3E70B79A3
:10F220001C06E5D5164B174E1C783378E4B2DBB2DA
:10F230009C420ED0144D01E0A3420AD00133402B72
:10F2400028BF00230879E85CC0B2C871087D072890
:10F25000F2D9DBB2034933700B79180644BF7C2323
:10F26000CB70C5E700A006408CA1FF1F8DA1FF1F3A
:10F27000D0A1FF1F88A1FF1F14A2FF1F10A2FF1F14
:10F2800018A2FF1F11A2FF1F90A1FF1F054A064BE6
:10F2900010781B78C0B2DBB2984238BF4030C01A39
:10F2A000704700BF8CA2FF1F21A2FF1FF0B4384B94
:10F2B0001A7912F0300F2CD072B6997D01F0FF024E
:10F2C00000293DD062B6334F334938780D78334E3C
:10F2D0001C46C0B2EDB2431C402BE17928BF00238D
:10F2E000AB4202F1FF32C9B21CBFF154184612F012
:10F2F000FF02F0D12A4B1B68C2B23A704BB1A84250
:10F3000036BFC5F14005401B40192728C4BF012264
:10F310001A701F49CA78D2B2150616D452060DD5F6
:10F320001B4B1B795B0609D51E4B1F491B6800222E
:10F330000A7003B11A70164B3C22DA70F0BC7047A9
:10F340004022D9795A7462B6E3E70B791C06E5D5F9
:10F35000164B174E1C783378E4B2DBB29C420ED0C9
:10F36000144D01E0A3420AD00133282B28BF00230B
:10F370000879E85CC0B2C871087D0728F2D9DBB211
:10F38000034933700B79180644BF7C23CB70C5E763
:10F3900000B006408CA2FF1F21A2FF1F4CA2FF1F3E
:10F3A0001CA2FF1F90A2FF1F20A2FF1F94A2FF1FFD
:10F3B0008DA2FF1F24A2FF1F70B584B072B6194B37
:10F3C000194D1A48702241260F2480211A702E7080
:10F3D0001A460470197013781B06FCD5144B186874
:10F3E00062B6144B144C984298BF00EB800001A900
:10F3F00098BF40000A22FDF7CFFE01A92046002356
:10F4000011F8012B01333AB10A2B20F8022FF7D162
:10F410001623237004B070BD5B00DBB2237004B010
:10F4200070BD00BF0000024007000240060002401D
:10F43000080002407F9698009893FF1FFFFFFFFF90
:10F440002DE9F043DFF8EC808BB006460F4600F064
:10F4500073F898F90030013304460D4637D0304632
:10F46000394600F0DFF9002831D02BA3D3E900237F
:10F470003046394600F026FE814668BB28A3D3E912
:10F4800000233046394600F0FFFD00B398F9003004
:10F49000254ACDF82090042400200021022BCDE93C
:10F4A0000467CDE9026700940192CDE906012CD0F2
:10F4B000684600F0BDF940B3089B1BB101F0AAF902
:10F4C000089B0360DDE906010BB0BDE8F083204630
:10F4D00029460BB0BDE8F083134A98F90030019239
:10F4E00003210022CDE90467CDE90267009108926B
:10F4F0002BB90E4B4FF06042CDE90623D8E70C49FB
:10F500000020022BCDE90601D2D101F083F922239C
:10F510000360D1E7AFF30080EF39FAFE422E864058
:10F5200051302DD5104987C03C400100FFFFEF4707
:10F530000000F07FAE93FF1F2DE9F04FB04F21F098
:10F540000042BA4283B00C464FEAD17605460DD947
:10F55000AC4FBA4225D9C1F31303034340F0EF8007
:10F560000EB10020014603B0BDE8F08FA64B9A42D1
:10F5700000F2CC80A54B9A4200F2DE808AA3D3E948
:10F58000002300F05DF90022A14B00F09BFD002854
:10F5900000F005812846214600229D4B00F050F9DD
:10F5A000E1E783A3D3E9002300F08CFD002840F0BD
:10F5B000CB802846214680A3D3E9002300F064FDD8
:10F5C0000028CED1934B284603EBC60821467CA3E6
:10F5D000D3E9002300F0E6FAD8E9002300F030F97F
:10F5E00000F07AFD804600F077FA77A3D3E9002394
:10F5F00006460F4600F0D6FA02460B46284621463C
:10F6000000F01CF972A3D3E90023CDE900013046D4
:10F61000394600F0C7FA82468B4652465B46DDE922
:10F62000000100F00BF905460C462A462346284601
:10F63000214600F0B7FA68A3D3E9002306460F4637
:10F6400000F0B0FA66A3D3E9002300F0F7F83246E1
:10F650003B4600F0A7FA64A3D3E9002300F0F0F8DA
:10F6600032463B4600F09EFA61A3D3E9002300F046
:10F67000E5F832463B4600F095FA5FA3D3E9002354
:10F6800000F0DEF832463B4600F08CFA02460B46AC
:10F690002846214600F0D2F806460F462846214665
:10F6A00032463B46B8F1000F56D000F07BFA3246A6
:10F6B00004460D463B4600204FF0804100F0BEF866
:10F6C00002460B462046294600F096FB02460B46B2
:10F6D0005046594600F0B2F8DDE9002300F0AEF8DC
:10F6E0000B4602464A49002000F0A8F86FF47F73E9
:10F6F00098454FDA08F57A7801EB085100224FF06F
:10F70000B87300F04FFA03B0BDE8F08F424B9A4255
:10F710003FF658AF414BF4002344D3E9002300F0F7
:10F720008DF83F4BC6F101081C44CDE90001D4E936
:10F7300000ABC6EB080870E74FF0000875E702461B
:10F740000B4600F07DF80EE717A3D3E9002310461F
:10F75000194600F027FA06E700F024FA0022804656
:10F7600089464FF080433046394600F067F802463C
:10F770000B464046494600F03FFB2A46234600F030
:10F780005DF802460B460020214900F057F803B00F
:10F79000BDE8F08F01EB085103B0BDE8F08F804663
:10F7A00043E700BFAFF300809C7500883CE4377EE0
:10F7B000EF39FAFE422E864051302DD5104987C0D0
:10F7C000FE822B654715F73F0000E0FE422EE63F24
:10F7D000763C7935EF39EA3DD0A4BE726937663E92
:10F7E000F16BD2C541BDBB3E2CDE25AF6A56113F41
:10F7F00093BDBE166CC1663F3E5555555555C53F28
:10F80000412E8640FFFFEF7F422ED63FFFFF2F3E67
:10F810000000F03F40400100B1A2F03F6040010015
:10F820005040010041F0004101F58010C00F7047C9
:10F830000020704781F0004102E000BF83F00043E8
:10F8400030B54FEA41044FEA430594EA050F08BF7B
:10F8500090EA020F1FBF54EA000C55EA020C7FEA3F
:10F86000645C7FEA655C00F0E2804FEA5454D4EBBC
:10F870005555B8BF6D420CDD2C4480EA020281EA86
:10F88000030382EA000083EA010180EA020281EABE
:10F890000303362D88BF30BD11F0004F4FEA013110
:10F8A0004FF4801C4CEA113102D0404261EB41011F
:10F8B00013F0004F4FEA03334CEA133302D05242A5
:10F8C00063EB430394EA050F00F0A780A4F1010461
:10F8D000D5F1200E0DDB02FA0EFC22FA05F280189B
:10F8E00041F1000103FA0EF2801843FA05F3594181
:10F8F0000EE0A5F120050EF1200E012A03FA0EFC00
:10F9000028BF4CF0020C43FA05F3C01851EBE37129
:10F9100001F0004507D54FF0000EDCF1000C7EEB46
:10F9200000006EEB0101B1F5801F1BD3B1F5001F84
:10F930000CD349085FEA30004FEA3C0C04F10104A3
:10F940004FEA445212F5800F80F09A80BCF1004FCC
:10F9500008BF5FEA500C50F1000041EB045141EA4E
:10F96000050130BD5FEA4C0C404141EB010111F44F
:10F97000801FA4F10104E9D191F0000F04BF0146FA
:10F980000020B1FA81F308BF2033A3F10B03B3F1D8
:10F9900020020CDA0C3208DD02F1140CC2F10C0268
:10F9A00001FA0CF021FA02F10CE002F11402D8BFC6
:10F9B000C2F1200C01FA02F120FA0CFCDCBF41EA92
:10F9C0000C019040E41AA2BF01EB0451294330BD61
:10F9D0006FEA04041F3C1CDA0C340EDC04F114043E
:10F9E000C4F1200220FA04F001FA02F340EA030015
:10F9F00021FA04F345EA030130BDC4F10C04C4F15B
:10FA0000200220FA02F001FA04F340EA030029463A
:10FA100030BD21FA04F0294630BD94F0000F83F484
:10FA2000801306BF81F480110134013D4EE77FEA67
:10FA3000645C18BF7FEA655C29D094EA050F08BFB3
:10FA400090EA020F05D054EA000C04BF1946104694
:10FA500030BD91EA030F1EBF0021002030BD5FEAD8
:10FA6000545C05D14000494128BF41F0004130BD00
:10FA700014F580043CBF01F5801130BD01F0004554
:10FA800045F0FE4141F470014FF0000030BD7FEAC7
:10FA9000645C1ABF194610467FEA655C1CBF0B46C2
:10FAA000024650EA013406BF52EA033591EA030FD9
:10FAB00041F4002130BD00BF90F0000F04BF0021D1
:10FAC000704730B54FF4806404F132044FF0000504
:10FAD0004FF0000150E700BF90F0000F04BF00217D
:10FAE000704730B54FF4806404F1320410F00045E3
:10FAF00048BF40424FF000013EE700BF42004FEADE
:10FB0000E2014FEA31014FEA02701FBF12F07F435A
:10FB100093F07F4F81F06051704792F0000F14BF57
:10FB200093F07F4F704730B54FF4607401F000459B
:10FB300021F0004120E700BF50EA010208BF7047F2
:10FB400030B54FF000050AE050EA010208BF7047E7
:10FB500030B511F0004502D5404261EB41014FF450
:10FB6000806404F132045FEA915C3FF4DCAE4FF054
:10FB700003025FEADC0C18BF03325FEADC0C18BF3B
:10FB8000033202EBDC02C2F1200300FA03FC20FA8C
:10FB900002F001FA03FE40EA0E0021FA02F11444D9
:10FBA000C1E600BF70B54FF0FF0C4CF4E06C1CEAEE
:10FBB00011541DBF1CEA135594EA0C0F95EA0C0F63
:10FBC00000F0DEF82C4481EA030621EA4C5123EAD6
:10FBD0004C5350EA013518BF52EA033541F4801105
:10FBE00043F4801338D0A0FB02CE4FF00005E1FBB8
:10FBF00002E506F00042E0FB03E54FF00006E1FB02
:10FC000003569CF0000F18BF4EF0010EA4F1FF0444
:10FC1000B6F5007F64F5407404D25FEA4E0E6D4184
:10FC200046EB060642EAC62141EA55514FEAC52095
:10FC300040EA5E504FEACE2EB4F1FD0C88BFBCF511
:10FC4000E06F1ED8BEF1004F08BF5FEA500E50F1C2
:10FC5000000041EB045170BD06F0004646EA010188
:10FC600040EA020081EA0301B4EB5C04C2BFD4EBBA
:10FC70000C0541EA045170BD41F480114FF0000EB3
:10FC8000013C00F3AB8014F1360FDEBF002001F021
:10FC9000004170BDC4F10004203C35DA0C341BDC9B
:10FCA00004F11404C4F1200500FA05F320FA04F06D
:10FCB00001FA05F240EA020001F0004221F00041A1
:10FCC00010EBD37021FA04F642EB06015EEA430E14
:10FCD00008BF20EAD37070BDC4F10C04C4F1200544
:10FCE00000FA04F320FA05F001FA04F240EA0200F7
:10FCF00001F0004110EBD37041F100015EEA430EC8
:10FD000008BF20EAD37070BDC4F1200500FA05F2E7
:10FD10004EEA020E20FA04F301FA05F243EA020366
:10FD200021FA04F001F0004121FA04F220EA020075
:10FD300000EBD3705EEA430E08BF20EAD37070BDBB
:10FD400094F0000F0FD101F00046400041EB01019B
:10FD500011F4801F08BF013CF7D041EA060195F07D
:10FD6000000F18BF704703F00046520043EB030337
:10FD700013F4801F08BF013DF7D043EA0603704724
:10FD800094EA0C0F0CEA135518BF95EA0C0F0CD02F
:10FD900050EA410618BF52EA4306D1D181EA030175
:10FDA00001F000414FF0000070BD50EA410606BF6F
:10FDB0001046194652EA430619D094EA0C0F02D1B4
:10FDC00050EA013613D195EA0C0F05D152EA0336F9
:10FDD0001CBF104619460AD181EA030101F0004117
:10FDE00041F0FE4141F470014FF0000070BD41F060
:10FDF000FE4141F4780170BD70B54FF0FF0C4CF43A
:10FE0000E06C1CEA11541DBF1CEA135594EA0C0F58
:10FE100095EA0C0F00F0A7F8A4EB050481EA030EA5
:10FE200052EA03354FEA013100F088804FEA03338C
:10FE30004FF0805545EA131343EA12634FEA02225A
:10FE400045EA111545EA10654FEA00260EF000411B
:10FE50009D4208BF964244F1FD0404F5407402D26D
:10FE60005B084FEA3202B61A65EB03055B084FEAFE
:10FE700032024FF480104FF4002CB6EB020E75EBFB
:10FE8000030E22BFB61A754640EA0C005B084FEA23
:10FE90003202B6EB020E75EB030E22BFB61A7546A0
:10FEA00040EA5C005B084FEA3202B6EB020E75EBEB
:10FEB000030E22BFB61A754640EA9C005B084FEA63
:10FEC0003202B6EB020E75EB030E22BFB61A754670
:10FED00040EADC0055EA060E18D04FEA051545EA5F
:10FEE00016754FEA06164FEAC30343EA52734FEA08
:10FEF000C2025FEA1C1CC0D111F4801F0BD141EA81
:10FF000000014FF000004FF0004CB6E711F4801FE5
:10FF100004BF01430020B4F1FD0C88BFBCF5E06FC5
:10FF20003FF6AFAEB5EB030C04BFB6EB020C5FEAD5
:10FF3000500C50F1000041EB045170BD0EF0004E2A
:10FF40004EEA113114EB5C04C2BFD4EB0C0541EA5C
:10FF5000045170BD41F480114FF0000E013C90E659
:10FF600045EA060E8DE60CEA135594EA0C0F08BF1D
:10FF700095EA0C0F3FF43BAF94EA0C0F0AD150EA1C
:10FF800001347FF434AF95EA0C0F7FF425AF1046AF
:10FF900019462CE795EA0C0F06D152EA03353FF4D7
:10FFA000FDAE1046194622E750EA410618BF52EA54
:10FFB00043067FF4C5AE50EA41047FF40DAF52EA28
:10FFC00043057FF4EBAE12E74FF0FF3C06E000BFC5
:10FFD0004FF0010C02E000BF4FF0010C4DF804CDD2
:10FFE0004FEA410C7FEA6C5C4FEA430C18BF7FEA92
:10FFF0006C5C1BD001B050EA410C0CBF52EA430CC0
:020000021000EC
:1000000091EA030F02BF90EA020F0020704710F13F
:10001000000F91EA030F58BF994208BF90422CBFCE
:10002000D8176FEAE37040F0010070474FEA410CC7
:100030007FEA6C5C02D150EA013C07D14FEA430CE5
:100040007FEA6C5CD6D152EA033CD3D05DF8040B56
:10005000704700BF8446104662468C461946634688
:1000600000E000BF01B5FFF7B7FF002848BF10F15F
:10007000000F01BD4DF808EDFFF7F4FF0CBF0120A4
:1000800000205DF808FB00BF4DF808EDFFF7EAFF20
:1000900034BF012000205DF808FB00BF4DF808EDDB
:1000A000FFF7E0FF94BF012000205DF808FB00BFD0
:1000B0004DF808EDFFF7CEFF94BF012000205DF85A
:1000C00008FB00BF4DF808EDFFF7C4FF34BF012067
:1000D00000205DF808FB00BF4FEA410212F5001254
:1000E00015D211D56FF47873B3EB625212D94FEA7F
:1000F000C12343F0004343EA505311F0004F23FA69
:1001000002F018BF404270474FF00000704750EABD
:10011000013005D111F0004008BF6FF0004070477A
:100120004FF00000704700BF4FEA4102B2F1E043D8
:1001300024BFB3F5001CDCF1FE5C0DD901F0004CCE
:100140004FEAC0024CEA5070B2F1004F40EB83001E
:1001500008BF20F00100704711F0804F21D113F14A
:100160003872BCBF01F00040704741F480114FEA83
:100170005252C2F11802C2F1200C10FA0CF320FA0C
:1001800002F018BF40F001004FEAC1234FEAD32329
:1001900003FA0CFC40EA0C0023FA02F34FEA430393
:1001A000CCE77FEA625307D150EA01331EBF4FF01C
:1001B000FE4040F44000704701F0004040F0FE4037
:1001C00040F40000704700BF80F0004002E000BF34
:1001D00081F0004142001FBF5FEA410392EA030F32
:1001E0007FEA226C7FEA236C6AD04FEA1262D2EB7C
:1001F0001363C1BFD218414048404140B8BF5B4281
:10020000192B88BF704710F0004F40F4000020F019
:100210007F4018BF404211F0004F41F4000121F02F
:100220007F4118BF494292EA030F3FD0A2F1010279
:1002300041FA03FC10EB0C00C3F1200301FA03F1B7
:1002400000F0004302D5494260EB4000B0F5000FDA
:1002500013D3B0F1807F06D340084FEA310102F199
:100260000102FE2A51D2B1F1004F40EBC25008BF4B
:1002700020F0010040EA03007047490040EB000015
:1002800010F4000FA2F10102EDD1B0FA80FCACF144
:10029000080CB2EB0C0200FA0CF0AABF00EBC25043
:1002A00052421843BCBFD0401843704792F0000F31
:1002B00081F4000106BF80F400000132013BB5E784
:1002C0004FEA41037FEA226C18BF7FEA236C21D0FA
:1002D00092EA030F04D092F0000F08BF084670475F
:1002E00090EA010F1CBF0020704712F07F4F04D12D
:1002F000400028BF40F00040704712F100723CBF40
:1003000000F50000704700F0004343F0FE4040F469
:10031000000070477FEA226216BF08467FEA236327
:100320000146420206BF5FEA412390EA010F40F412
:10033000800070474FF0000304E000BF10F000435E
:1003400048BF40425FEA000C08BF704743F0964345
:1003500001464FF000001CE050EA010208BF704760
:100360004FF000030AE000BF50EA010208BF7047E7
:1003700011F0004302D5404261EB41015FEA010CFC
:1003800002BF84460146002043F0B64308BFA3F1F4
:100390008053A3F50003BCFA8CF2083AA3EBC253D6
:1003A00010DB01FA02FC634400FA02FCC2F12002F5
:1003B000BCF1004F20FA02F243EB020008BF20F02C
:1003C0000100704702F1200201FA02FCC2F1200292
:1003D00050EA4C0021FA02F243EB020008BF20EA87
:1003E000DC7070474FF0FF0C1CEAD0521EBF1CEAB5
:1003F000D15392EA0C0F93EA0C0F6FD01A4480EAA3
:10040000010C400218BF5FEA41211ED04FF000638B
:1004100043EA501043EA5111A0FB01310CF00040B7
:10042000B1F5000F3EBF490041EAD3715B0040EADD
:10043000010062F17F02FD2A1DD8B3F1004F40EBAD
:10044000C25008BF20F00100704790F0000F0CF080
:10045000004C08BF49024CEA502040EA51207F3A44
:10046000C2BFD2F1FF0340EAC250704740F400001F
:100470004FF00003013A5DDC12F1190FDCBF00F010
:1004800000407047C2F10002410021FA02F1C2F1BE
:10049000200200FA02FC5FEA310040F1000053EA5A
:1004A0004C0308BF20EADC70704792F0000F00F0A8
:1004B000004C02BF400010F4000F013AF9D040EAAE
:1004C0000C0093F0000F01F0004C02BF490011F442
:1004D000000F013BF9D041EA0C018FE70CEAD15340
:1004E00092EA0C0F18BF93EA0C0F0AD030F0004CC0
:1004F00018BF31F0004CD8D180EA010000F0004074
:10050000704790F0000F17BF90F0004F084691F031
:10051000000F91F0004F14D092EA0C0F01D142026B
:100520000FD193EA0C0F03D14B0218BF084608D134
:1005300080EA010000F0004040F0FE4040F400007E
:10054000704740F0FE4040F4400070474FF0FF0C11
:100550001CEAD0521EBF1CEAD15392EA0C0F93EA58
:100560000C0F69D0A2EB030280EA010C49024FEAAA
:10057000402037D04FF0805343EA111143EA101363
:100580000CF000408B4238BF5B0042F17D024FF41B
:10059000000C8B4224BF5B1A40EA0C00B3EB510FF6
:1005A00024BFA3EB510340EA5C00B3EB910F24BFDF
:1005B000A3EB910340EA9C00B3EBD10F24BFA3EB64
:1005C000D10340EADC001B0118BF5FEA1C1CE0D12C
:1005D000FD2A3FF650AF8B4240EBC25008BF20F0DF
:1005E000010070470CF0004C4CEA50207F32C2BF33
:1005F000D2F1FF0340EAC250704740F400004FF0D0
:100600000003013A37E792F0000F00F0004C02BF00
:10061000400010F4000F013AF9D040EA0C0093F0CA
:10062000000F01F0004C02BF490011F4000F013B24
:10063000F9D041EA0C0195E70CEAD15392EA0C0F8C
:1006400008D142027FF47DAF93EA0C0F7FF470AFC4
:10065000084676E793EA0C0F04D14B023FF44CAF07
:1006600008466EE730F0004C18BF31F0004CCAD19C
:1006700030F000427FF45CAF31F000437FF43CAFD8
:100680005FE700BF4FF0FF3C06E000BF4FF0010CFA
:1006900002E000BF4FF0010C4DF804CD4FEA4002DC
:1006A0004FEA41037FEA226C18BF7FEA236C11D026
:1006B00001B052EA530C18BF90EA010F58BFB2EBD9
:1006C000030088BFC81738BF6FEAE17018BF40F059
:1006D000010070477FEA226C02D15FEA402C05D10D
:1006E0007FEA236CE4D15FEA412CE1D05DF8040B92
:1006F000704700BF844608466146FFE70FB5FFF725
:10070000C9FF002848BF10F1000F0FBD4DF808EDDC
:10071000FFF7F4FF0CBF012000205DF808FB00BFCD
:100720004DF808EDFFF7EAFF34BF012000205DF827
:1007300008FB00BF4DF808EDFFF7E0FF94BF012074
:1007400000205DF808FB00BF4DF808EDFFF7D2FF71
:1007500094BF012000205DF808FB00BF4DF808EDB4
:10076000FFF7C8FF34BF012000205DF808FB00BF81
:100770004FEA4002B2F1FE4F0FD34FF09E03B3EBAE
:1007800012620DD94FEA002343F0004310F0004FEE
:1007900023FA02F018BF404270474FF00000704744
:1007A00012F1610F01D1420205D110F0004008BFE3
:1007B0006FF0004070474FF00000704742000ED2CB
:1007C000B2F1FE4F0BD34FF09E03B3EB126209D48C
:1007D0004FEA002343F0004323FA02F070474FF042
:1007E0000000704712F1610F01D1420202D14FF0B7
:1007F000FF3070474FF00000704700BF0B460146C6
:10080000184600F001B800BF13460A460146022010
:1008100000F0A8BE014B1868704700BFD897FF1FB3
:1008200070B50F4E0F4D761BB61018BF002405D0C3
:10083000013455F8043B9847A642F9D10A4E0B4DB6
:10084000761B03F017FCB61018BF002406D0013445
:1008500055F8043B9847A642F9D170BD70BD00BF62
:100860008040010080400100944001008040010070
:10087000024B0146186800F00BB800BFD897FF1F65
:10088000024B0146186800F031BF00BFD897FF1F28
:100890002DE9F04F01F10B05162D83B0064640F20D
:1008A0009F8035F0070500F1BF80A94200F2BC80AF
:1008B00000F058FBB5F5FC7FC0F09C826B0A00F09D
:1008C000BA80042B00F28381A80900F1390E4FEAA7
:1008D0004E033830C44F07EB8303A3F108015C6873
:1008E000A14207D1ACE0002A80F2AC80E468A142CA
:1008F00000F0A680636823F003035A1B0F2AF2DD81
:10090000B9493C6901F1080E744500F0B381636890
:1009100023F003035A1B0F2A00F39981002AC1F820
:1009200014E0C1F810E080F29E80B3F5007F80F003
:100930006781DB0803F1010C01229B1002FA03F32B
:100940004A6851F83C80C4F8088001EBCC091A438E
:10095000A9F10803E3604A6041F83C40C8F80C4044
:10096000831001249C40944200F28A80144206D1F4
:1009700020F003006400144200F10400FAD007EBF9
:10098000C009CC468046DCF80C108C4507D173E1D9
:10099000002A80F28181C9688C4500F06D814B6826
:1009A00023F003035A1B0F2AF2DD0C46D1F80CC0CA
:1009B00054F8088F4B1945F001054D6042F00101D4
:1009C000C8F80CC03046CCF808807B613B61C3F8A6
:1009D0000CE0C3F808E059609A5000F0C5FA1FE037
:1009E000102921D800F0BEFA1025062302207E4FE0
:1009F00007EB8303A3F108025C68944200F0458191
:100A00006368E168A56823F00303234430465A680D
:100A1000E96042F001028D605A6000F0A5FA0834E6
:100A2000204603B0BDE8F08F00240C23204633603D
:100A300003B0BDE8F08F80234FF0400E3F2049E720
:100A400070465DE72344E1685A68A56842F00102F8
:100A5000E96030468D605A6000F086FA083420461E
:100A600003B0BDE8F08F234430465A6842F00102DB
:100A70005A6000F079FA0834204603B0BDE8F08FE0
:100A8000BC68636823F00308A84504D3C5EB0803DA
:100A90000F2B00F38C80554BDFF860911A68D9F862
:100AA000003001332A4404EB080A00F0608102F5AB
:100AB00080520F3222F47F6222F00F02114630463C
:100AC000019200F04BFCB0F1FF3F8346019A00F029
:100AD0005881824500F2FC80454B1968DA45114483
:100AE000196000F05381D9F80000DFF810E10130FF
:100AF0001BBFCAEB0B0A5144CEF800B019601BF0C3
:100B0000070100F01781C1F10800C1F5805183444D
:100B100008315A44C2F30B02C2EB01094946304680
:100B2000019300F01BFC431C019B00F03F81CBEBC9
:100B300000024A4442F001021968C7F808B049446B
:100B4000BC42CBF804201960DFF8A49016D0B8F1AD
:100B50000F0F40F2FD806268A8F10C0323F0070339
:100B6000E01802F001024FF0050E1A430F2B6260ED
:100B7000C0F804E0C0F808E000F21C811D4BBC681E
:100B80001A68914288BF19601B4B1A6891426268CB
:100B900088BF196022F003029542A2EB050301D839
:100BA0000F2B04DC304600F0DFF9002438E762192F
:100BB00043F0010345F0010565603046BA605360BB
:100BC00000F0D2F90834204603B0BDE8F08F142BB2
:100BD00071D9542B00F2A480280B00F16F0E4FEA5C
:100BE0004E036E3076E600BFDC97FF1FA0A2FF1F0A
:100BF000A4A2FF1F9CA2FF1F98A2FF1FE89BFF1F3C
:100C00005A0A042A5ED9142A00F2B38002F15C0168
:100C100049005B3207EB810C57F82110DFF8DC81CB
:100C2000ACF1080C8C4500F088804A6822F0030281
:100C3000934202D289688C45F7D1D1F80CC07A680A
:100C4000C4F80CC0A160CCF80840CC6088E66319F9
:100C500042F0010745F00105656030464B610B61CC
:100C6000C3F80CE0C3F808E05F609A50083400F065
:100C70007BF9D5E64A6873E608F1010818F0030F1E
:100C80000CF1080C7FF47FAE30E0DC68A34208BFB3
:100C900002303FF435AEB3E60B440C465A68C968DF
:100CA00054F8085F42F001025A603046E9608D60F6
:100CB00000F05AF9B4E603F15C0E03F15B004FEA71
:100CC0004E0307E69A0902F1390149003832A1E7DB
:100CD000BC424A4B3FF400AF9C68626822F00302BA
:100CE0005AE759F80839994540F0828010F0030F0F
:100CF00000F1FF30F5D17B6823EA04037B606400D8
:100D00009C423FF6BDAE002C3FF4BAAE1C424046BA
:100D10007FF435AE64001C4200F10400FAD02EE6E8
:100D2000B3F5AA7F18D8E80B00F1780E4FEA4E030E
:100D30007730CFE54FF48051EBE60121D8F804304D
:100D4000921001FA02F21A43C8F80420614677E7CC
:100D50000123CBF8043025E740F25452934220D8C7
:100D6000A80C00F17D0E4FEA4E037C30B2E5103244
:100D7000A4E6542A26D81A0B02F16F0149006E32FC
:100D800048E7BC68626822F0030205E7CAF30B007B
:100D900000287FF4A8AE4244BB6842F001025A60CA
:100DA000ECE6FE234FF07F0E7E2093E501224FF00C
:100DB0000009C1E604F10801304600F097FCD9F8BB
:100DC0000010DBE6B2F5AA7F05D8DA0B02F1780154
:100DD000490077321EE740F254518A4205D89A0CF6
:100DE00002F17D0149007C3214E7FE217E2211E7E9
:100DF0007B6884E7E808431C5B00F8E5DC97FF1F8D
:100E00008842F0B50DD98B1898420AD28118002A71
:100E100051D09A1A13F8014D01F8014D9342F9D1BE
:100E2000F0BD0F2A48D941EA00039B0746D100F1E3
:100E3000100401F11003154653F8106C44F8106CBF
:100E400053F80C6C44F80C6C53F8086C44F8086CBC
:100E5000103D53F8046C44F8046C0F2D03F110039B
:100E600004F11004E8D8A2F1100323F00F0302F0FC
:100E70000F0E1033BEF1030F1944034421D91E1F76
:100E80000D467446043C55F8047B46F8047F032C59
:100E9000F8D8AEF1040424F00304043423442144BC
:100EA00002F0030262B1013B0A4411F8014B03F85E
:100EB000014F8A42F9D1F0BD0346F3E70346F2E75A
:100EC000F0BD7246EEE700BF70B4840746D0541EF2
:100ED000002A41D0CDB2034602E0621EE4B31446BC
:100EE00003F8015B9A07F8D1032C2ED9CDB245EA5D
:100EF00005250F2C45EA054519D903F110022646B0
:100F0000103E0F2E42F8105C42F80C5C42F8085C70
:100F100042F8045C02F11002F2D8A4F1100222F0AF
:100F20000F0204F00F041032032C13440DD91E4697
:100F30002246043A032A46F8045BFAD8221F22F01C
:100F400003020432134404F003042CB1C9B21C445C
:100F500003F8011BA342FBD170BC70471446034643
:100F6000C2E700BF704700BF704700BF024B0A4690
:100F70000146186800F002B8D897FF1F2DE9F04F1E
:100F8000174683B0002900F0C1800E46814607F164
:100F90000B05FFF7E7FF56F804EC162D2EF00304BF
:100FA000A6F1080840D810221546AF4241D8944215
:100FB00075DAC94B996808EB04008842416800F073
:100FC000D98021F0010303445B68DB077DD51EF067
:100FD000010F35D039464846FFF75AFC0746E0B1C5
:100FE00056F8043C23F001034344A0F108029A425E
:100FF00000F04481221F242A00F23181132A00F2DA
:10100000048103463246116819605168596092683C
:101010009A603146484600F069FB4846FFF7A4FF56
:10102000384603B0BDE8F08F25F00705002D2A46AD
:10103000BBDA0C230020C9F8003003B0BDE8F08F04
:1010400056F8083CC3EB080ADAF8043023F0030C26
:1010500004EB0C039342BDDB5746DAF80C1057F84B
:10106000080F221F242AC160886000F21781132A0A
:1010700040F212813168CAF808107168CAF80C1081
:101080001B2A00F22B8108360AF110023168116028
:1010900071685160B16891603E461C46D046631B42
:1010A0000F2B1DD8D8F8043003F001032343444428
:1010B000C8F80430636843F0010363604846FFF7F3
:1010C00053FF304603B0BDE8F08F21F00301214407
:1010D000914221DBC36882680C46D3609A60DEE7E8
:1010E000D8F8042008EB050102F00102154343F093
:1010F00001020B44C8F804504A605A6842F00102E9
:1011000008315A60484600F0F1FAD7E7114603B0BB
:10111000BDE8F04FFFF7BCBB1EF0010F7FF45AAFE4
:1011200056F8083CC3EB080ADAF8043023F0030C45
:1011300001EB0C0E96458BDBC36882685746D36083
:101140009A6057F8081FDAF80C30CB60221F242A67
:10115000996000F29980132A62D93368CAF808307E
:101160007368CAF80C301B2A00F2A08008360AF116
:10117000100356E021F0030BA34405F11000834552
:1011800059DA1EF0010F7FF425AF56F8081CC1EBA9
:10119000080ADAF8041021F0030CE34458453FF73D
:1011A00057AF5746DAF80C1057F8080F221F242AB9
:1011B000C160886000F2B480132A40F2A5803168D3
:1011C000CAF808107168CAF80C101B2A00F2AF8028
:1011D00008360AF110023168116071685160B16817
:1011E00091600AEB0501C5EB0B0242F00102996028
:1011F0004A60DAF8043003F001031D434846CAF898
:101200000450FFF7B1FE38465CE73368036073684B
:1012100043601B2A27D800F1080306F10802F2E612
:101220003B4632681A6072685A60B2689A603E46FD
:101230007446D04633E708EB0501C5EB0B0B4BF0CA
:10124000010299604A6056F8043C03F001031D4313
:10125000484646F8045CFFF787FE304632E73146E1
:10126000FFF7CEFDD5E6B3688360F368C360242A38
:1012700028D000F1100306F11002C4E650F8043C37
:1012800023F003031C440AE7314638467446D0462F
:10129000FFF7B6FD3E4602E73A46F7E631463846E6
:1012A0001C46D046FFF7ACFD3E46F8E6B368CAF8E8
:1012B0001030F368CAF81430242A1BD010360AF113
:1012C0001803AEE7336903617369436106F11802DD
:1012D00000F1180397E600BFDC97FF1FB168CAF85A
:1012E0001010F168CAF81410242A0FD010360AF131
:1012F0001802CBE63369CAF818307369CAF81C3093
:1013000018360AF120038CE73A4664E73269CAF8D6
:1013100018207269CAF81C2018360AF12002B5E6B6
:10132000314638460193FFF76BFD019B59E7B168E1
:10133000CAF81010F168CAF81410242A03D0103625
:101340000AF1180247E73269CAF818207269CAF828
:101350001C2018360AF120023DE700BF38B5074CC3
:101360000023054608462360FBF7E0FE431C00D03F
:1013700038BD2368002BFBD02B6038BD00A4FF1FB5
:1013800090F800F06DE9024520F007016FF0000CC5
:1013900010F0070491F820F040F049804FF000046D
:1013A0006FF00700D1E9002391F840F000F1080048
:1013B00082FA4CF2A4FA8CF283FA4CF3A2FA8CF380
:1013C0004BBBD1E9022382FA4CF200F10800A4FAE7
:1013D0008CF283FA4CF3A2FA8CF3E3B9D1E904233B
:1013E00082FA4CF200F10800A4FA8CF283FA4CF372
:1013F000A2FA8CF37BB9D1E9062301F1200182FA2C
:101400004CF200F10800A4FA8CF283FA4CF3A2FA31
:101410008CF3002BC6D0002A04BF04301A4612BA3F
:10142000B2FA82F2FDE8024500EBD2007047D1E942
:10143000002304F00305C4F100004FEAC50514F0D1
:10144000040F91F840F00CFA05F562EA05021CBFA2
:1014500063EA050362464FF00004A9E7002A41D081
:1014600040EA010313F00303F0B425D1032A23D982
:1014700004680D68AC421FD1043A35D0A4F101359F
:1014800025EA040414F0803F31D1071D0D1D0DE045
:1014900057F8043B0E68A3F10134B34224EA030475
:1014A0000AD1043A20D014F0803F23D1032A2946E0
:1014B000384605F10405EBD803780C789C4202F11C
:1014C000FF320CD182B114B916E06AB17BB110F8C9
:1014D000013F11F8014FA34202F1FF32F5D0181B72
:1014E000F0BC7047104670471046F0BC7047184675
:1014F000F0BC70470020F3E72046F1E740EA010323
:101500009B0770B42BD1032A29D90C4603462146E8
:1015100054F8046BA6F1013525EA060515F0803F65
:1015200006D1043A032A43F8046B2146EFD8A2B14E
:101530000C781C70013A013301313CB16AB111F8E9
:10154000014B03F8014B013A002CF7D12AB11A44A0
:10155000002103F8011B9A42FBD170BC704703467F
:10156000E5E700BF2DE9F047254C2568D5F848414F
:101570000646884692469946C4B360681F2817DC21
:10158000431C76B104EB80050122C5F888A0D4F88D
:10159000881182401143022EC4F88811C5F80891C1
:1015A0001ED00230636044F820800020BDE8F08740
:1015B000144B03B34FF4C870FFF75AF90446D0B187
:1015C000D5F84831002780E88800C5F848413846FA
:1015D0000123C4F88871C4F88C71002EE1D0D1E7E2
:1015E000D4F88C110A43C4F88C21DAE705F5A67407
:1015F000C5F84841C1E74FF0FF30BDE8F08700BFB4
:101600007040010071080100024B13B1024800F064
:1016100005B87047000000002916010000230146AC
:101620001A461846FFF79EBF38B5074D074C2C1BCE
:10163000A41005D0013C55F8043D9847002CF9D181
:10164000BDE8384002F026BD0000000000000000A8
:10165000F8B5234F0C460646FFF784FCBB685D686F
:1016600025F00305291B01F6EF7121F47F6121F0BC
:101670000F01A1F58054B4F5805F07DB00213046EF
:10168000FFF76CFEBB682B44984204D03046FFF74E
:101690006BFC0020F8BD61423046FFF75FFE013071
:1016A0000DD0104BBA6819682D1B45F00105304666
:1016B000091B55601960FFF757FC0120F8BD002198
:1016C0003046FFF74BFEBA68831A0F2BDEDD064C5F
:1016D0000449246843F00103001B53600860D5E708
:1016E000DC97FF1FA4A2FF1FE89BFF1F002945D026
:1016F0002DE9F0410D468046FFF734FC55F8047C97
:101700006A4927F00103A5F10804E2188E685068C1
:10171000B24220F0030062D0FE0750600BD455F8AF
:10172000087CE41B01F1080EA56875453B446FD0A9
:10173000E768EF60BD6015186D68ED0742D543F0AE
:1017400001026260E350B3F5007F18D2DB085A1C37
:101750004D6851F83270A76001209B1000FA03F326
:1017600001EBC2001D430838E0604D6041F8324093
:10177000FC604046BDE8F041FFF7F6BB70475A0AEF
:10178000042A53D89A0902F139077F0002F138057B
:1017900001EB870051F827204449083890424DD08A
:1017A000516821F003018B4202D292689042F7D136
:1017B000D068E060A2608460D4604046BDE8F0413B
:1017C000FFF7D2BB95683A4FBD4203443FD0D06883
:1017D000E86043F0010285606260E350B3E7FF0711
:1017E000034407D455F8082CA41A1344A068E268EF
:1017F000C26090602F4A126843F00100934260601B
:101800008C60B6D32C4B40461968FFF721FFB0E738
:1018100011184968C90744D49168D268CA60034462
:1018200043F0010091606060E350A2E7142A17D8EA
:1018300002F15C077F0002F15B05A9E7AA104B6883
:10184000012505FA02F213434B600246B1E743F06B
:1018500001024C610C61E560A5606260E35088E7BD
:10186000542A06D81A0B02F16F077F0002F16E05A9
:101870008EE7B2F5AA7F06D8DA0B02F178077F006F
:1018800002F1770584E740F25450824206D89A0C60
:1018900002F17D077F0002F17C0579E7FE277E25B6
:1018A00076E743F001026260E35062E7DC97FF1FD6
:1018B000E497FF1FE49BFF1FA0A2FF1F0000780515
:1018C0003408540B800C3C0F5C12E015FA19141EFE
:1018D0006022AC265C2B0C30BC34023AFF3FFFFF89
:1018E000FDFFFFFFFBFFFFFFF8FFFFFFFDFFFFFF17
:1018F000FBFFFFFFF8FFFFFFFDFFFFFFFAFFFFFF0A
:10190000F7FFFFFFFDFFFFFFFBFFFFFFF7FFFFFFFD
:10191000FCFFFFFFFBFFFFFFF7FFFFFFFDFFFFFFE8
:10192000FAFFFFFFF7FFFFFFFDFFFFFFFBFFFFFFDA
:10193000F8FFFFFFFDFFFFFFFBFFFFFFF8FFFFFFCB
:10194000FDFFFFFFFAFFFFFFF7FFFFFFFCFFFFFFB9
:10195000FBFFFFFFF7FFFFFFFDFFFFFFFBFFFFFFA9
:10196000F7FFFFFFFDFFFFFFFAFFFFFFF7FFFFFF9E
:10197000FDFFFFFFFBFFFFFFF7FFFFFFFDFFFFFF87
:10198000FBFFFFFFF7FFFFFFFDFFFFFFFAFFFFFF7A
:10199000F7FFFFFFFDFFFFFFFAFFFFFFF8FFFFFF6D
:1019A000FDFFFFFFFAFFFFFFF7FFFFFFFDFFFFFF58
:1019B000FAFFFFFFF7FFFFFFFDFFFFFFFAFFFFFF4B
:1019C000F8FFFFFFFDFFFFFFFAFFFFFFF8FFFFFF3C
:1019D000FDFFFFFFFAFFFFFFF7FFFFFFFCFFFFFF29
:1019E000FBFFFFFFF7FFFFFFFDFFFFFFFAFFFFFF1A
:1019F000F7FFFFFFFDFFFFFFFAFFFFFFF7FFFFFF0E
:101A0000FEFFFFFFFBFFFFFFF8FFFFFFFEFFFFFFF3
:101A1000FBFFFFFFF8FFFFFFFDFFFFFFFAFFFFFFE8
:101A2000F7FFFFFFFCFFFFFFFAFFFFFFF7FFFFFFDE
:101A3000FCFFFFFFFAFFFFFFF7FFFFFFFDFFFFFFC8
:101A4000FAFFFFFFF7FFFFFFFDFFFFFFF9FFFFFFBB
:101A5000F7FFFFFFFDFFFFFFF9FFFFFFF7FFFFFFAE
:101A6000FDFFFFFFFAFFFFFFF7FFFFFFFDFFFFFF97
:101A7000FAFFFFFFF7FFFFFFFDFFFFFFFAFFFFFF8A
:101A8000F6FFFFFFFDFFFFFFFAFFFFFFF7FFFFFF7E
:101A9000FEFFFFFFFBFFFFFFF7FFFFFFFEFFFFFF64
:101AA000FBFFFFFFF7FFFFFFFDFFFFFFFAFFFFFF59
:101AB000F7FFFFFFFDFFFFFFFBFFFFFFF8FFFFFF4B
:101AC000FDFFFFFFFBFFFFFFF8FFFFFFFDFFFFFF35
:101AD000FAFFFFFFF7FFFFFFFCFFFFFFF9FFFFFF2C
:101AE000F7FFFFFFFCFFFFFFF9FFFFFFF7FFFFFF1F
:101AF000FDFFFFFFFAFFFFFFF7FFFFFFFDFFFFFF07
:101B0000FAFFFFFFF7FFFFFFFDFFFFFFF9FFFFFFFA
:101B1000F6FFFFFFFDFFFFFFFAFFFFFFF7FFFFFFED
:101B2000D0210100AC2101008821010064210100C5
:101B3000BC1C0100781B01009C1B0100C01B0100A4
:101B4000981C0100541B0100E01F0100BC1801009B
:101B5000101E01000000580246056608540BD80EFE
:101B60005C127017FC21F82A70305834DC37663A62
:101B70008C3C803EFF3FFFFF000058024605660890
:101B8000540BD80E5C12E015FA19141E6022AC2614
:101B90005C2B0C30BC34023AFF3FFFFF0000900189
:101BA00020031405D0075A0AAC0DCC10B4146A18DF
:101BB000E81C342180252A2B70301437FF3FFFFFAB
:101BC0000000C800F4018403140508072E091C0C4A
:101BD000D80EF811AE159619401F1C25F22B58345B
:101BE000FF3FFFFFFBFFFFFFF8FFFFFFF4FFFFFFDB
:101BF000FAFFFFFFF7FFFFFFF4FFFFFFFDFFFFFF0F
:101C0000F9FFFFFFF4FFFFFFFAFFFFFFF7FFFFFF02
